:100000000C94580C0C94890C0C94890C0C94890C4D
:100010000C94890C0C94890C0C94890C0C94890C0C
:100020000C94890C0C94890C0C94890C0C94890CFC
:100030000C94890C0C94890C0C94890C0C94890CEC
:100040000C94890C0C941F650C94890C0C94890CED
:100050000C94890C0C94890C0C94AF360C941935C3
:100060000C94890C0C94BA640C94890C0C94890C33
:100070000C94890C0C94890C0C94890C0C94890CAC
:100080000C94890C0C94890C0C94890C0C94890C9C
:100090000C94890C0C94890C0C94890C0C94890C8C
:1000A0000C94890C0C94890C0C94890C0C94890C7C
:1000B0000C94890C0C94890C0C94890C0C94890C6C
:1000C0000C94890C0C94890C0C94890C0C949190D0
:1000D0000C9467900C94890C0C94890C0C94890CEA
:1000E0000C94890CFA32FD32EC32F032F6323433B1
:1000F000013305330B330F33133319331D332133DE
:10010000343327332B332F3335343A343F344934A7
:100110005334CC345D3465346D34773481348B346E
:100120009A34A434CC34AE34B834C23414372137C2
:100130003D374A37643771378B378D37084AD73B9D
:100140003BCE016E84BCBFFDC12F3D6C74319ABDA6
:1001500056833DDA3D00C77F11BED9E4BB4C3E91CA
:100160006BAAAABE000000803F05A84CCDB2D44EB9
:10017000B93836A9020C50B9918688083CA6AAAABB
:100180002ABE000000803F004E414E494E4954595E
:10019000494E46CDCCCC3D0AD7233C17B7D1387752
:1001A000CC2B329595E6241FB14F0A000020410068
:1001B00000C84200401C4620BCBE4CCA1B0E5AAEB2
:1001C000C59D7400407A10F35A00A0724E180900C1
:1001D00010A5D4E80000E87648170000E40B5402AC
:1001E0000000CA9A3B000000E1F5050000809698E7
:1001F00000000040420F000000A086010000001037
:100200002700000000E80300000000640000000078
:10021000000A00000000000100000000002C76D859
:1002200088DC674F0823DFC1DFAE59E1B1B796E53F
:10023000E3E453C63AE651997696E8E6C28426EBA3
:10024000898C9B62ED407C6FFCEFBC9C9F40F2BAB6
:10025000A56FA5F490055A2AF75C936B6CF9676D4E
:10026000C11BFCE0E40D47FEF520E6B500D0ED90A3
:100270002E0300943577050080841E080000204E70
:100280000A000000C80C333333330F986E12831109
:1002900041EF8D2114893BE65516CFFEE6DB18D1E0
:1002A000844B381BF77C1D901DA4BBE424203284B2
:1002B000725E228100C9F124ECA1E53D272F005395
:1002C00044207072696E74696E672062797465206B
:1002D000004E6F74205344207072696E74696E67AB
:1002E000002E0044656C6574696F6E206661696CF0
:1002F00065642C2046696C653A200046696C65206F
:1003000064656C657465643A002E006F70656E20DC
:100310006661696C65642C2046696C653A20005002
:100320004944204175746F74756E652066696E6905
:1003300073686564212050757420746865204B7063
:100340002C204B6920616E64204B6420636F6E73B8
:1003500074616E747320696E746F20436F6E66698A
:100360006775726174696F6E2E6800504944204150
:1003700075746F74756E65206661696C65642120A3
:1003800074696D656F75740020403A006F6B20547E
:100390003A006F6B20423A00504944204175746F17
:1003A00074756E65206661696C6564212054656DA5
:1003B000706572617475726520746F6F206869670B
:1003C0006800204B643A2000204B693A2000204B03
:1003D000703A200020436C617369632050494420C7
:1003E000002054753A2000204B753A2000206D61A2
:1003F000783A2000206D696E3A200020643A20008F
:1004000020626961733A2000486F74656E64206FE2
:100410006666736574733A002200556E6B6E6F7773
:100420006E20636F6D6D616E643A202200486F74B8
:10043000656E64206F6666736574733A007A5F6DEB
:10044000696E3A2000795F6D696E3A2000785F6DC1
:1004500061783A2000785F6D696E3A20005A3A0060
:10046000593A0020436F756E7420583A2000453A7F
:10047000005A3A00593A00583A004649524D5741FD
:1004800052455F4E414D453A4D61726C696E205642
:10049000313B20537072696E7465722F6772626CA3
:1004A000206D617368757020666F722067656E36A7
:1004B000204649524D574152455F55524C3A687457
:1004C00074703A2F2F7777772E6D656E64656C2D7B
:1004D00070617274732E636F6D2050524F544F438E
:1004E0004F4C5F56455253494F4E3A312E302E30C5
:1004F000204D414348494E455F545950453A334495
:10050000205072696E7465722045585452554445A6
:10051000525F434F554E543A320A002042403A004F
:1005200020403A00202F0020423A00202F006F6B1D
:1005300020543A002569206D696E2C2025692073AE
:10054000656300456E642066696C65206C69737430
:1005500000426567696E2066696C65206C6973741A
:10056000005072696E7465722073746F7070656488
:100570002064756520746F206572726F72732E200F
:1005800046697820746865206572726F7220616EAA
:100590006420757365204D39393920746F20726578
:1005A00073746172742E202854656D706572617465
:1005B0007572652069732072657365742E205365AA
:1005C0007420697420616674657220726573746149
:1005D0007274696E6729004E6F204C696E65204EFB
:1005E000756D626572207769746820636865636BF6
:1005F00073756D2C204C617374204C696E653A20C4
:10060000004E6F20436865636B73756D2077697466
:1006100068206C696E65206E756D6265722C204C69
:10062000617374204C696E653A2000636865636B82
:1006300073756D206D69736D617463682C204C61F6
:100640007374204C696E653A20004C696E65204ECB
:10065000756D626572206973206E6F74204C6173D2
:1006600074204C696E65204E756D6265722B312C5D
:10067000204C617374204C696E653A20004D313115
:100680003000256920686F757273202569206D69B7
:100690006E7574657300446F6E65207072696E7458
:1006A000696E672066696C65005072696E74657268
:1006B0002073746F707065642064756520746F209A
:1006C0006572726F72732E20466978207468652097
:1006D0006572726F7220616E6420757365204D398A
:1006E000393920746F20726573746172742E2028FA
:1006F00054656D70657261747572652069732072DE
:10070000657365742E205365742069742061667466
:1007100065722072657374617274696E6729004E28
:100720006F204C696E65204E756D62657220776929
:10073000746820636865636B73756D2C204C6173FE
:1007400074204C696E653A20004E6F2043686563E3
:100750006B73756D2077697468206C696E65206EA7
:10076000756D6265722C204C617374204C696E65E6
:100770003A2000636865636B73756D206D69736DF6
:10078000617463682C204C617374204C696E653A07
:1007900020004C696E65204E756D6265722069732C
:1007A000206E6F74204C617374204C696E65204E0E
:1007B000756D6265722B312C204C617374204C690D
:1007C0006E653A20004572726F723A004D313130D9
:1007D000006572726F722077726974696E67207437
:1007E0006F2066696C6500205A3A0020593A002053
:1007F000583A00656E6473746F7073206869743A58
:1008000020006563686F3A00446F6E6520736176FF
:10081000696E672066696C652E006F6B004D32391A
:100820000053442063617264206F6B006F70656ECB
:10083000526F6F74206661696C656400766F6C75C9
:100840006D652E696E6974206661696C656400452A
:1008500072726F723A00534420696E697420666147
:10086000696C006563686F3A002200656E7175659A
:10087000696E672022006563686F3A004D3234006C
:100880004D3233202573006175746F25692E670022
:100890002020506C616E6E657242756666657242AC
:1008A000797465733A20002046726565204D656D48
:1008B0006F72793A20004A616E2031342032303232
:1008C0003100436F6D70696C65643A200054656E49
:1008D0006C6F6700207C20417574686F723A20004D
:1008E0004A616E20313420323032312030303A3398
:1008F000323A333500204C61737420557064617452
:1009000065643A2000312E302E3137004D61726C13
:10091000696E200020536F6674776172652052659E
:1009200073657400205761746368646F6720526553
:10093000736574002042726F776E206F7574205259
:1009400065736574002045787465726E616C205221
:100950006573657400506F776572557000737461CC
:1009600072740070012C0190012701B0012201C0B6
:10097000011D01F00118011002130130020E016087
:1009800002090190020401C002FF000003FA0040C6
:1009900003F5008003F000D003EB002004E60070B4
:1009A00004E100E004DC004005D700C005D20040AF
:1009B00006CD00D006C8008007C3003008BE00F096
:1009C00008B900C009B400B00AAF00B00BAA00D04B
:1009D0000CA500000EA000500F9B00C01096005008
:1009E00012910000148C00C0158700B0178200B06F
:1009F000197D00D01B7800001E730040206E00900F
:100A0000226900F024640040275F0090295A00E02A
:100A10002B5500102E500020304B0010324600E0C5
:100A200033410090353C001037370070383200A059
:100A3000392D00B03A2800A03B2300603C1E001076
:100A40003D1900903D1400103E0F00703E0A00C09A
:100A50003E0500003F00003A2045787472756465D9
:100A600072207377697463686564206F66662E20F0
:100A70004D415854454D50207472696767657265E1
:100A8000642021003A204578747275646572207381
:100A900077697463686564206F66662E204D494EE1
:100AA00054454D50207472696767657265642021F2
:100AB0000054656D7065726174757265206865615A
:100AC0007465642062656420737769746368656423
:100AD000206F66662E204D415854454D502074724B
:100AE000696767657265642021210054656D7065D2
:100AF00072617475726520686561746564206265F1
:100B000064207377697463686564206F66662E205D
:100B10004D494E54454D5020747269676765726542
:100B200064202121004572726F723A00000021009A
:100B3000240027002A002D003000330001010000AE
:100B4000040107010A0100002200250028002B00F3
:100B50002E003100340002010000050108010B01E4
:100B6000000020002300260029002C002F00320066
:100B7000000100000301060109010505050507053F
:100B800008080808020202020A0A08080404040409
:100B90000101010101010101030303030303030335
:100BA000040707070C0C0C0C0C0C0C0C02020202C4
:100BB00006060606060606060B0B0B0B0B0B0B0BAD
:100BC000010210202008081020401020408002015F
:100BD0000201080402010102040810204080804044
:100BE0002010080402018004020180402010080443
:100BF00002010804020101020408102040800102E1
:100C000004081020408000000A0B02090C0D0E0899
:100C100007030401000000000000000000000000C5
:100C200000000000000000000000000000000000C4
:100C30000000121110000000000000000000000081
:100C40000000000000000000000000005365747404
:100C5000696E67732053746F726564005A323A008C
:100C6000457874656E646572204F66667365743A84
:100C70000059323A00457874656E646572204F669B
:100C8000667365743A0058323A005365636F6E6458
:100C9000657279204D617820506F733A00204400CE
:100CA0002049002020204D3330312050005049444D
:100CB0002073657474696E67733A00205A00205976
:100CC0000020204D323036205800486F6D65206F6F
:100CD000666673657420286D6D293A0020450020F2
:100CE0005A0020580020420020540020204D32306D
:100CF00035205300416476616E63656420766172CD
:100D00006961626C65733A20533D4D696E2066657A
:100D100065647261746520286D6D2F73292C2054D1
:100D20003D4D696E2074726176656C206665656400
:100D30007261746520286D6D2F73292C20423D6DE2
:100D4000696E696D756D207365676D656E7420746D
:100D5000696D6520286D73292C20583D6D61786977
:100D60006D756D205859206A65726B20286D6D2F46
:100D700073292C20205A3D6D6178696D756D205A5C
:100D8000206A65726B20286D6D2F73292C202045F9
:100D90003D6D6178696D756D2045206A65726B20C7
:100DA000286D6D2F73290020540020204D323034DF
:100DB000205300416363656C65726174696F6E3ABC
:100DC00020533D616363656C65726174696F6E2C5D
:100DD00020543D7265747261637420616363656C55
:100DE00065726174696F6E00204500205A002059B9
:100DF0000020204D3230312058004D6178696D75EA
:100E00006D20416363656C65726174696F6E202843
:100E10006D6D2F7332293A00204500205A00205969
:100E20000020204D3230332058004D6178696D75B7
:100E30006D2066656564726174657320286D6D2F21
:100E400073293A00204500205A0020590020204DE7
:100E500039322058005374657073207065722075A4
:100E60006E69743A0053746F7265642073657474AC
:100E7000696E67732072657472696576656400488F
:100E8000617264636F6465642044656661756C7447
:100E90002053657474696E6773204C6F6164656478
:100EA000006563686F3A00473238205859000000E7
:100EB00048C200000000000000002200656E71754D
:100EC00065696E672022000000404000004040003D
:100ED00000003F20746F6F206C6F6E672065787420
:100EE000727573696F6E2070726576656E74656475
:100EF0000020636F6C6420657874727573696F6E1F
:100F00002070726576656E746564006563686F3A1B
:100F1000004E65772056616C756520457272200021
:100F200025730057726974696E6720746F20666953
:100F30006C653A20002E006F70656E206661696CEA
:100F400065642C2046696C653A20002E006F706540
:100F50006E206661696C65642C2046696C653A2078
:100F60000046696C652073656C6563746564002078
:100F700053697A653A200046696C65206F70656E2A
:100F800065643A20002E006F70656E206661696CA2
:100F900065642C2046696C653A20007C3C3E5E2BE3
:100FA0003D3F2F5B5D3B2C2A225C0024F4D4305063
:100FB000C38E20C2A24017828B7011127A910D81CC
:100FC0006CD90AA861E108C7586607615143061E3B
:100FD0004B5D05C145A7041A411104093D980371F1
:100FE0003931034036DB0265339102D4305402803C
:100FF0002E1D02632CEE01752AC501B028A0011038
:101000002781018F2564012B244B01E0223401ACA0
:10101000211F018D200D01801FFC00841EED009713
:101020001DDF00B81CD200E61BC600201BBC0064FC
:101030001AB200B219A8000A19A0006A189900D1C2
:1010400017910040178B00B516840031167E00B34F
:101050001579003A157300C7146F0058146A00EE32
:101060001366008813630025135E00C7125B006CD3
:1010700012570015125400C111510070114F002178
:10108000114B00D61049008D104700461044000255
:10109000104200C00F4000800F3E00420F3C00068F
:1010A0000F3B00CB0E3800930E37005C0E35002747
:1010B0000E3400F30D3200C10D3100900D30006090
:1010C0000D2E00320D2D00050D2C00D90C2B00AE7D
:1010D0000C2900850C29005C0C2700350C27000E1C
:1010E0000C2600E80B2400C40B2400A00B23007D79
:1010F0000B23005A0B2100390B2100180B2000F89C
:101100000A1F00D90A1E00BB0A1E009D0A1D00808E
:101110000A1D00630A1C00470A1B002C0A1B001151
:101120000A1A00F7091A00DD091900C4091900ABF1
:10113000091900920917007B091800630917004C70
:1011400009160036091600200916000A091500F5CF
:10115000081500E0081400CC081400B8081400A416
:10116000081400900813007D0812006B0813005843
:10117000081200460812003408110023081100125A
:1011800008110001081100F0071000E0071000D05E
:10119000071000C0071000B0070F00A10710009152
:1011A000070E0083070F0074070F0065070E005736
:1011B000070E0049070E003B070D002E070E00200A
:1011C000070D0013070D0006070D00F9060C00EDD2
:1011D000060D00E0060C00D4060C00C8060C00BC8E
:1011E000060C00B0060C00A4060B0099060C008D3E
:1011F000060B0082060B0077060B006C060B0061E5
:10120000060A0057060B004C060A0042060A003880
:10121000060A002E060A0024060A001A060A001012
:1012200006090007060A00FD050900F4050900EBA0
:10123000050900E2050900D9050900D0050900C724
:10124000050900BE050900B5050800AD050800A5A3
:101250000509009C050800940508008C0508008419
:101260000508007C050800740508006C050700658A
:101270000508005D050700560508004E05070047F4
:101280000507004005080038050700310507002A5A
:10129000050700230507001C050600160507000FBB
:1012A0000507000805060002050700FB040600F517
:1012B000040700EE040600E8040600E2040700DB71
:1012C000040600D5040600CF040600C9040600C3C6
:1012D000040600BD040600B7040600B1040500AC16
:1012E000040600A6040600A00405009B0406009561
:1012F000040500900406008A0405008504050080AA
:101300000406007A04050075040500700405006BEE
:1013100004050066040500610405005C040500572F
:10132000040500520405004D04050048040500436F
:101330000405003E0404003A0405003504050030AD
:101340000404002C04050027040400230405001EE7
:101350000404001A04040016040500110404000D1E
:10136000040400090405000404040000040400FC53
:10137000030400F8030400F4030400F0030400EC89
:10138000030400E8030400E4030400E0030400DCB9
:10139000030400D8030400D4030400D0030400CCE9
:1013A000030400C8030300C503030024F404D92088
:1013B0001BC40C5C0E9804C4095F0265077101F43C
:1013C00005F900FB04B30048048700C10369005815
:1013D00003550003034500BE023A00840231005366
:1013E000022A002902250004022000E4011C00C892
:1013F000011900AF01170098011400840113007156
:101400000110006101100051010E0043010D003672
:10141000010B002B010B0020010B00150109000C32
:1014200001090003010800FB000800F3000800EBBD
:10143000000700E4000600DE000600D8000600D227
:10144000000600CC000500C7000500C2000500BD75
:10145000000400B9000400B5000400B1000400ADB0
:10146000000400A9000400A5000300A20003009FDF
:101470000004009B00030098000300950002009305
:10148000000300900003008D0002008B0003008821
:101490000002008600020084000300810002007F39
:1014A0000002007D0002007B00020079000200774C
:1014B0000001007600020074000200720001007159
:1014C0000002006F0002006D0001006C0002006A63
:1014D000000100690002006700010066000100656C
:1014E0000001006400020062000100610001006070
:1014F0000001005F0002005D0001005C0001005B74
:101500000001005A00010059000100580001005775
:101510000001005600010055000100540001005375
:101520000000005300010052000100510001005072
:101530000001004F0001004E0000004E0001004D70
:101540000001004C0001004B0000004B0001004A6C
:101550000001004900010048000000480001004768
:101560000001004600000046000100450000004563
:10157000000100440001004300000043000100425C
:101580000000004200010041000000410001004055
:101590000001003F0000003F0001003E0000003E4F
:1015A0000001003D0000003D0001003C0000003C47
:1015B0000000003C0001003B0000003B0001003A3D
:1015C0000000003A00010039000000390001003835
:1015D000000000380000003800010037000000372C
:1015E0000001003600000036000000360001003522
:1015F0000000003500000035000100340000003418
:10160000000000340001003300000033000000330C
:101610000001003200000032000000320001003101
:1016200000000031000000310001003000000030F7
:10163000000000300001002F0000002F0000002FEC
:101640000000002F0001002E0000002E0000002EE0
:101650000001002D0000002D0000002D0000002DD5
:101660000001002C0000002C0000002C0000002CC9
:101670000001002B0000002B0000002B0000002BBD
:101680000001002A0000002A0000002A0000002AB1
:1016900000010029000000290000002900000029A5
:1016A0000000002900010028000000280000002898
:1016B000000000280000002800010027000000278B
:1016C000000000270000002700000027000100267E
:1016D0000000002600000026000000260000002672
:1016E0000001002500000025000000250000002565
:1016F0000000002500000025000100240000002457
:101700000000002400000024000000240001002349
:10171000000000230000002300000023000000233D
:10172000000000230000002300010022000000222E
:101730000000002200000022000000220000002221
:101740000001002100000021000000210000002114
:101750000000002100000021000000210001002005
:1017600000000020000000200000002000000020F9
:101770000000002000000020000000200001001FE9
:101780000000001F0000001F0000001F0000001FDD
:101790000000001F0000001F0001001E0000001ECE
:1017A0000000001E0000001E0000000080984300A2
:1017B00000A0430000B443000048C2000000000045
:1017C00000000020423A0020453A00543A00526599
:1017D00073656E643A20006F6B005072696E7465B9
:1017E000722068616C7465642E206B696C6C2829AA
:1017F0002063616C6C656421005072696E7465725F
:101800002073746F707065642064756520746F2038
:101810006572726F72732E20466978207468652035
:101820006572726F7220616E6420757365204D3928
:10183000393920746F20726573746172742E202898
:1018400054656D706572617475726520697320727C
:10185000657365742E205365742069742061667405
:1018600065722072657374617274696E67290020F5
:10187000573A0020453A00543A006563686F3A00D1
:10188000202D20496E76616C6964206578747275CC
:10189000646572206E756D626572202100FFFFFF26
:1018A0000080B1430000A0430000B4432BB806B849
:1018B00011241FBECFEFD1E2DEBFCDBF00E00CBFD1
:1018C0001BE0A0E0B2E0E4ECF3E901E00BBF02C0F2
:1018D00007900D92AA31B107D9F729E1AAE1BBE03F
:1018E00001C01D92A035B207E1F71CE0C7E5DCE0BE
:1018F00000E006C021970109802FFE010E944BC81D
:10190000C635D10780E00807A9F70E9480AE0C9485
:10191000D1C90C9400002F923F924F925F926F9228
:101920007F928F929F92AF92BF92CF92DF92EF926F
:10193000FF920F931F93CF93DF93CDB7DEB7C557B9
:10194000D1090FB6F894DEBF0FBECDBF2DB73EB79D
:10195000E2963FAF2EAFE2978091DD0B882341F0F6
:101960000E94E25610923F1010923E101092DD0B32
:1019700087E40E94E4AD782E882309F48CC00E948D
:101980000AAE0E94D8C56430710509F474C0E4F44D
:101990006230710509F45CC00CF062C077FF02C0D0
:1019A0000C94A121A0E8AA2EAFE4BA2EA3ECCA2E73
:1019B000A7ECDA2E86017501A6019501C601B501D5
:1019C0000E94195A0C94A1216A35710509F45AC074
:1019D0002CF56C31710511F00C94A1216FE672E1C8
:1019E00083E89AE30E9413AE6FE672E183E89AE31C
:1019F0000E9413AE6FE672E183E89AE30E9413AE91
:101A00006FE672E183E89AE30E9413AE60E070E053
:101A100080E090E00E9435A90C94A1216B357105FE
:101A2000A9F16C35710511F00C94A121F0E8AF2EED
:101A3000FFE4BF2EF3ECCF2EF7ECDF2E860175010D
:101A4000A6019501C601B5010E94C07E0C94A1219A
:101A500080910713811104C00E941E9A81E007C083
:101A600080910713811107C00E941E9A80E00E9496
:101A700083910C94732560E070E0CB010E9413AE5B
:101A80000C94A121109283180C94A12181E08093E1
:101A900083180C94A1218DE40E94E4AD882311F4F5
:101AA0000C9453210E940AAE0E94D8C5693C71056E
:101AB00011F40C945F180CF0E0C06035710511F45E
:101AC0000C948D150CF071C06731710509F401C4D7
:101AD0000CF041C06231710511F40C94A01524F58D
:101AE00077FF02C00C94A121623071050CF4D1C1C2
:101AF0006131710511F00C94A1215F9847988A9883
:101B00009FB7F894809108018E7F809308019FBF52
:101B10009FB7F894809108018B7F809308019FBF45
:101B20008D9812980C94A1216431710509F47AC33F
:101B30000CF4B5C16531710509F4C7C3663171058F
:101B400011F00C94A12110923F1010923E101092AF
:101B500040100C94A1216C31710509F453C484F434
:101B60006931710509F4E6C30CF4CEC36A3171051D
:101B700009F4E6C36B31710509F4F0C30C94A1219B
:101B80006F31710509F458C634F46E31710509F4EA
:101B90006FC40C94A1216032710509F4DBC56A326F
:101BA000710509F4A7C60C94A1216B36710509F4DF
:101BB000AEC754F56535710509F4FCC784F4623588
:101BC000710509F4B4C70CF4ACC76335710509F4A9
:101BD000B2C76435710509F4B3C70C94A121683606
:101BE000710509F4A2C634F46C35710509F4F9C71E
:101BF0000C94A1216936710509F4B0C66A367105E5
:101C000009F455C70C94A1216737710509F43DC14A
:101C1000ECF46237710511F40C94CF165CF46D3658
:101C2000710511F00C94A1218FEF9FEF0E94379F57
:101C30000C94A1216337710511F40C94AE1665372D
:101C4000710511F40C94BD160C94A121693771052E
:101C500011F40C94B21714F40C94AD176C38710590
:101C600009F46BC66E3B710511F00C94A1218FEF46
:101C70009FEF0E94917C0C94A121673E33E0730793
:101C800011F40C943B210CF076C06D3251E07507D5
:101C900011F40C941C1ADCF56E3C710511F40C94D3
:101CA0001919C4F46C3C710511F40C94971814F0D4
:101CB0000C94B9186B3C710511F00C94A12115EB33
:101CC000E12E12E1F12E07EC12E084E0D82ED00EC6
:101CD0000C9488186C3D710511F40C94FE193CF4B9
:101CE0006A3D710511F40C9437190C94A1216D3DD6
:101CF000710511F40C940D1A623E710511F00C94EB
:101D0000A12181E090E00E942B9B0C94A121653FD2
:101D100091E0790711F40C94671EC4F46F32B1E0BE
:101D20007B0711F40C94F81A14F40C94E41A60393B
:101D3000F1E07F0711F40C94641E643F714011F0D0
:101D40000C94A1210E94753E0C94A121673F31E0C3
:101D5000730711F40C946F1E14F40C946A1E6D3505
:101D600052E0750711F40C94721E603A734009F446
:101D70002AC50C94A121683F93E0790711F40C94D3
:101D80007B200CF04AC0633FB3E07B0711F40C9456
:101D9000941F6CF56A3EF3E07F0711F40C948C1FDE
:101DA0003CF4693E734011F40C94671F0C94A1211C
:101DB0006B3E43E0740711F40C94911F6C3E73402A
:101DC00011F00C94A121812C912C54017501640116
:101DD00000E010E020E030E040E050E060E070E043
:101DE000CB010E949942109248130C94A121653FA7
:101DF00083E0780711F40C940A2014F40C94CF1F9C
:101E0000663FA3E07A0711F40C944520673F7340C6
:101E100011F40C9460200C94A1216730E4E07E075B
:101E200011F40C940E21DCF46B3F23E0720711F4E3
:101E30000C94AE203CF4693F734011F40C94932051
:101E40000C94A1216D3F53E0750711F40C94D2203E
:101E50006E3F734011F40C94D8200C94A12169308A
:101E600094E0790711F40C940B2114F40C940821DC
:101E70006A30B4E07B0711F40C94032160317440A4
:101E800011F40C9413210C94A121E0EEF2E00C94D7
:101E9000BD1781E090E00E942B9B0C94A12183E56B
:101EA0000E94E4AD882341F00E940AAE0E94D8C58A
:101EB0007093350B6093340B85E990E19093941007
:101EC0008093931081E090E09093341280933312CA
:101ED000109236121092351240E050E0BA0189E9B2
:101EE00090E10E94F85C80919310909194102BE106
:101EF000FC013496DE01159601900D922A95E1F7CA
:101F0000DC0112968D919C9113979C838B838FEBB0
:101F100092E09A838983BE016F5F7F4F88E394E0EC
:101F20000E945B55CE0101960E949A72D0903512A4
:101F3000AD2CB090361280919C10882309F446C0D5
:101F40008250823030F48FE2809341101092421020
:101F50003DC06091A5107091A6108091A71090913E
:101F6000A81040E00E94EC72882381F12091A91012
:101F7000B0E22B9F90011124C9018259924F892B05
:101F800029F180E090E0E0E05EE2DC01A20FB31F07
:101F9000A259B24F4C91403289F08830910539F402
:101FA000AE2FB0E0A55CBF4E16965C93EF5FAE2FF0
:101FB000B0E0A55CBF4E16964C93EF5F01968B3058
:101FC000910519F7F0E0E55CFF4E16828091340B25
:101FD0009091350B892B59F489EF92E00E9411659D
:101FE00084E093E00E94116501E010E007C080E109
:101FF00093E00E9411658BE193E0F4CF87E293E0D8
:102000000E940F654AE0B801CE0101960E94DC8F64
:1020100089819A810E940F65CE0101960E947C8F72
:1020200082EB94E00E940F650E94036586E393E0D3
:102030000E940F654AE0B801CE0101960E94DC8F34
:1020400089819A810E940F65CE0101960E947C8F42
:1020500082EB94E00E940F650E9403650F5F1F4FA3
:102060000730110559F6E12CF12C00E010E075E97C
:10207000672E70E1772EDA942296DFAE2297EFEB8F
:102080008E2EE2E09E2EEA14FB0409F492C07092B8
:10209000941060929310E2E0F0E0F0933412E09339
:1020A000331222968FAD22978E1990E090933612BC
:1020B0008093351240E050E0BA0189E990E10E9436
:1020C000F85C8091931090919410FC013496DE019D
:1020D00015962BE101900D922A95E1F7DC011296FD
:1020E0008D919C9113979C838B839A828982BE01E8
:1020F0006F5F7F4F88E394E00E945B55CE010196AD
:102100000E949A7261E470E1CE01CB960E940F901A
:1021100080916910811145C021968EAD9FAD2197A8
:10212000892B09F43EC0BE01655C7F4FCE0101964C
:102130000E9407902DB63EB64D815E812A01F1E0E6
:102140004F1A51082DB73EB7241B350B0FB6F89424
:102150003EBF0FBE2DBF8DB79EB701966C014115D6
:10216000510541F0C114D10429F0B601CE01019608
:102170000E943855F601CF018C199D0984159505EB
:1021800014F40C94A421DD24D3940FB6F8943EBE2D
:102190000FBE2DBECE0101960E947C8FD1100C94F3
:1021A000AC21CE01CB960E947C8F5FEFE51AF50A39
:1021B0006ACF85E493E00E940F656091340B7091C3
:1021C000350B4AE0CE0101960E94DC8F89819A810D
:1021D0000E940F65CE0101960E947C8F0E940365CC
:1021E0008091340B9091350B019646E0489F900109
:1021F000499F300D11242017310754F08EE593E0EC
:102200000E9411658BE693E00E9411650C94A12158
:1022100089E793E00E94116586E893E00E941165CA
:102220000C94A121E1E5F5E08491882341F090919F
:10223000C00095FFFCCF8093C6003196F5CF80910A
:10224000C00085FFFCCF8AE08093C6001092341254
:102250001092331240E050E0BA0188E790E10E940A
:10226000F85C8BE1E8E7F0E1DE01159601900D9254
:102270008A95E1F780917610909177109C838B83FB
:102280008FEB92E09A838983BE016F5F7F4F88E373
:1022900094E00E945B55CE0101960E949A72E3E49D
:1022A000F5E08491882341F09091C00095FFFCCF28
:1022B0008093C6003196F5CF8091C00085FFFCCF9A
:1022C0008AE08093C6000C94A1210E94382A0C94C5
:1022D000A121E090C90BF090CA0B84E0E80EF11C3C
:1022E0006AE270E0C7010E947FC9009719F0FC0103
:1022F0003197108200E010E0980141E0B701C7017A
:102300000E94EE560C94A12180914010882331F058
:1023100081E090E090933F1080933E100E940D3535
:102320006093390B70933A0B80933B0B90933C0B6B
:102330000C94A12181E090E00E942B9B0C94A121A0
:1023400080914010882311F40C94A12183E50E9410
:10235000E4AD81110C9455220C94A1218091401080
:10236000882309F439C0EFEBF2E08491882341F02F
:102370009091C00095FFFCCF8093C6003196F5CFB9
:1023800060916C1070916D1080916E1090916F1033
:102390004AE00E94F626EDEBF2E08491882341F0BA
:1023A0009091C00095FFFCCF8093C6003196F5CF89
:1023B00060917010709171108091721090917310F3
:1023C0004AE00E94F6268091C00085FFFCCF8AE09B
:1023D0008093C6000C94A121E1EDF2E08491882362
:1023E00041F09091C00095FFFCCF8093C6003196DC
:1023F000F5CF8091C00085FFFCCF8AE08093C600B6
:102400000C94A1218091C90B9091CA0B6AE270E0F3
:1024100004960E947FC98C01892BE1F02091E00B8A
:102420003091E10B40E6429FC001439F900D112483
:102430006EE470E08651944F0E947FC960E270E0C4
:102440000E947FC901969093CA0B8093C90BF80133
:10245000319710828091C90B9091CA0B049600E0CD
:1024600010E0980140E0BC010E94EE560C94A121BE
:1024700080914010882311F40C94A1210E94E2560F
:102480008091C90B9091CA0B6AE270E004960E9499
:102490007FC98C01892BE1F02091E00B3091E10B99
:1024A00040E6429FC001439F900D11246EE470E00E
:1024B0008651944F0E947FC960E270E00E947FC9FC
:1024C00001969093CA0B8093C90BF8013197108243
:1024D0000091C90B1091CA0B480194E0890E911C20
:1024E00080914010882311F40C94A12183E192E1A2
:1024F0000E94E15D10923F1010923E10DE01119695
:102500007D01CD010E94A27284E790E19093941026
:1025100080939310F80184818F3209F08BC06FE2B1
:1025200070E0C4010E947FC98C010F5F1F4F6AE0F9
:10253000662E0115110509F483C06FE270E0C80131
:102540000E947FC96C01009709F47BC00817190726
:1025500008F077C05C01A01AB10AA501B801CE014C
:1025600080960E94A8C9E0E2F0E0EC0FFD1FEA0DA2
:10257000FB1D10828E01005E1F4FF80181918823A0
:1025800039F09091C00095FFFCCF8093C600F6CF44
:102590008091C00085FFFCCF6092C60060919310CF
:1025A000709194106115710511F06C5F7F4F21E0FF
:1025B000AE01405E5F4FCE0105960E9468638111B7
:1025C00031C0EBE0F3E08491882371F09091C0007A
:1025D00095FFFCCF8093C6003196F5CF9091C00057
:1025E00095FFFCCF8093C600D8018D918D0181119C
:1025F000F5CFE9E0F3E08491882341F09091C000A9
:1026000095FFFCCF8093C6003196F5CF8091C00036
:1026100085FFFCCF8AE08093C600C7010E949A72B2
:102620000C94A121F0929410E092931086010F5F18
:102630001F4F7FCF85E990E1909394108093931082
:10264000840160919310709194106115710511F0DF
:102650006C5F7F4F18A21BA222E0A801CE018096DA
:102660000E9468638823F1F0CE0180960E942C2896
:102670008823C1F06CA57DA58EA59FA541E00E9491
:10268000EC72882379F0E8A9B0E2EB9FF001112405
:10269000E259F24F309731F085EE80831BA20E9401
:1026A000AC72782ECE0180960E94EF5E772009F101
:1026B000EBEFF2E08491882341F09091C00095FF08
:1026C000FCCF8093C6003196F5CFF8018191882325
:1026D00039F09091C00095FFFCCF8093C600F6CFF3
:1026E00010926C1010926D1010926E1010926F106C
:1026F0002CC0E3EEF2E08491882341F09091C00079
:1027000095FFFCCF8093C6003196F5CFF8018191FB
:10271000882339F09091C00095FFFCCF8093C600CC
:10272000F6CFE1EEF2E08491882341F09091C00071
:1027300095FFFCCF8093C6003196F5CF8091C00005
:1027400085FFFCCF8AE08093C600C7010E949A7281
:102750000C94A12180913E1090913F10019721F49B
:102760000E9428A90E94E256E090C90BF090CA0B83
:10277000E4E0EE0EF11C6AE270E0C7010E947FC93E
:10278000009719F0FC013197108200E010E09801E9
:1027900041E0B701C7010E94EE56809140108823A6
:1027A00031F081E090E090933F1080933E100E94C2
:1027B0000D356093390B70933A0B80933B0B9093DC
:1027C0003C0B0C94A1218091C90B9091CA0B6AE239
:1027D00070E005960E947FC98C01892BE1F0209161
:1027E000E00B3091E10B40E6429FC001439F900D0A
:1027F00011246EE470E08651944F0E947FC960E21C
:1028000070E00E947FC901969093CA0B8093C90B18
:10281000F801319710828091C90B9091CA0B0596EF
:1028200021E020933D1000E010E0980140E0BC0161
:102830000E94EE560C94A1210E940D3560933D0B31
:1028400070933E0B80933F0B9093400B0091390B9C
:1028500010913A0B20913B0B30913C0B601B710B9C
:10286000820B930B28EE33E040E050E00E943DC421
:10287000CA01B9012CE330E040E050E00E943DC4C1
:102880007F936F933F932F9384E395E09F938F9370
:102890008E010F5F1F4F1F930F930E9472BEE6E7DA
:1028A000F8E084912DB73EB7285F3F4F0FB6F894FC
:1028B0003EBF0FBE2DBF882349F09091C00095FF09
:1028C000FCCF8093C60031968491F5CFF8018191B9
:1028D000882339F09091C00095FFFCCF8093C6000B
:1028E000F6CF8091C00085FFFCCF8AE08093C600C0
:1028F0000C94A12183E50E94E4AD882311F40C948B
:10290000A1210E940AAE0E94D8C58B0180E50E94D9
:10291000E4AD882311F40C94A1210F3F110509F0B7
:1029200010F40C9466220C94A1216FEF7FEF8FEFCF
:102930009FEF0E9471A30C94A12183E50E94E4AD56
:10294000882311F40C94A1210E940AAE0E94D8C5DC
:102950007093DF0B6093DE0B0C94A12189E690E06D
:102960000E94BE9C81110C94A121EEE2F5E08491BD
:10297000882341F09091C00095FFFCCF8093C60062
:102980003196F5CFE091A01834E0E39FF0011124D7
:10299000E95AFD4E608171818281938141E00E94FC
:1029A0007D27EBE2F5E08491882341F09091C0000F
:1029B00095FFFCCF8093C6003196F5CFE091A0182B
:1029C000F0E0EE0FFF1FE750FD4E60817181072E92
:1029D000000C880B990B0E94A7BE41E00E947D2746
:1029E000E7E2F5E08491882341F09091C00095FFE3
:1029F000FCCF8093C6003196F5CF6091471270915D
:102A000048128091491290914A1241E00E947D271C
:102A1000E4E2F5E08491882341F09091C00095FFB5
:102A2000FCCF8093C6003196F5CF6091DE0B70919C
:102A3000DF0B072E000C880B990B0E94A7BE41E00C
:102A40000E947D27E0E2F5E08491882341F0909197
:102A5000C00095FFFCCF8093C6003196F5CFE09182
:102A6000A018F0E0E959FD4E608170E080E090E050
:102A70000E946B27EBE1F5E08491882341F090916F
:102A8000C00095FFFCCF8093C6003196F5CF6091D2
:102A9000661270E080E090E00E946B278091C00099
:102AA00085FFFCCF8AE08093C6000C94732583E5F4
:102AB0000E94E4AD882319F10E940AAE20E030E0C4
:102AC000A9010E94A1BE87FD0FC00E940AAE20E0AE
:102AD00030E04FE753E40E94C4C6181644F00E9449
:102AE0000AAE0E94D8C505C060E070E002C06FEF7A
:102AF00070E07093A9186093A8180C94A1218FEF2F
:102B000090E09093A9188093A8180C94A12110929A
:102B1000A9181092A8180C94A121999AA19A0C9422
:102B2000A12161E080E00E94BBAD0C94A121109234
:102B300087180C94A12181E0809387180C94A1211F
:102B400083E50E94E4AD8823A1F00E940AAE20E054
:102B500030E04AE754E40E94FEB80E94DEC560936C
:102B600031027093320280933302909334020C94BA
:102B7000A12188E50E94E4AD81110C94692289E5C8
:102B80000E94E4AD81110C9469228AE50E94E4ADB3
:102B900081110C94692285E40E94E4AD81110C94AA
:102BA00069220E9428A98D9A129A81E00E94E7A8C2
:102BB0000C94A12183E50E94E4AD0E940AAE20E0BE
:102BC00030E04AE754E40E94FEB80E94DEC56093FC
:102BD00098187093991880939A1890939B180C9456
:102BE000A12182E50E94E4AD882329F00E940AAE6B
:102BF0004B015C0106C0812C912C40E8A42E4FE3D0
:102C0000B42E47EC52E026965FAF4EAF269708E30E
:102C100013E185EB92E124969FAF8EAF24973CE4BD
:102C2000232E33E1332E22961FAE22972696AEAD89
:102C3000BFAD26978D912696BFAFAEAF26970E9467
:102C4000E4AD882309F46DC02296BFAD2297B3305E
:102C500009F05CC00E940AAEA50194010E9467C5FC
:102C60002B013C0120E030E040EA51E40E94A1BE8B
:102C700087FF45C0A3019201F801608171818281C3
:102C800093810E9467C56B017C019B01AC0160913F
:102C9000A1127091A2128091A3129091A4120E948D
:102CA000FEB86093A1127093A2128093A312909326
:102CB000A412A70196012496AEADBFAD24976D91E5
:102CC0007D918D919C910E94FEB82496EEADFFAD52
:102CD00024976083718382839383D1016D917D9169
:102CE0008D919C910E94A5BEA70196010E94FEB8FD
:102CF0000E94DEC5F1016083718382839383D801D2
:102D00004D925D926D927C9213970BC00E940AAE19
:102D1000A50194010E9467C5F801608371838283D5
:102D200093832296FFAD2297FF5F2296FFAF2297F3
:102D30000C5F1F4F24962EAD3FAD24972C5F3F4F65
:102D400024963FAF2EAF249734E0230E311CF4308D
:102D500009F06CCF0E94753E0C94A121EAE7F4E0E3
:102D60008491882311F40C94A1219091C00095FFC7
:102D7000FCCF8093C6003196F3CF8091C90B909120
:102D8000CA0B6AE270E005960E947FC9009711F4B1
:102D90000C94A121FC01319710820C94A121E7E74A
:102DA000F4E08491882341F09091C00095FFFCCF1E
:102DB0008093C6003196F5CF609118137091191366
:102DC00080911A1390911B1342E00E947D27E4E743
:102DD000F4E08491882341F09091C00095FFFCCFEE
:102DE0008093C6003196F5CF60911C1370911D132E
:102DF00080911E1390911F1342E00E947D27E1E70E
:102E0000F4E08491882341F09091C00095FFFCCFBD
:102E10008093C6003196F5CF6091201370912113F5
:102E2000809122139091231342E00E947D27EEE6C9
:102E3000F4E08491882341F09091C00095FFFCCF8D
:102E40008093C6003196F5CF6091241370912513BD
:102E5000809126139091271342E00E947D27E3E69C
:102E6000F4E08491882341F09091C00095FFFCCF5D
:102E70008093C6003196F5CF2FB7F8946091081370
:102E80007091091380910A1390910B132FBF0E9428
:102E9000A7BE209138133091391340913A135091C5
:102EA0003B130E9467C542E00E947D27E0E6F4E004
:102EB0008491882341F09091C00095FFFCCF8093CE
:102EC000C6003196F5CF2FB7F89460910C1370912E
:102ED0000D1380910E1390910F132FBF0E94A7BE68
:102EE00020913C1330913D1340913E1350913F137C
:102EF0000E9467C542E00E947D27EDE5F4E08491E1
:102F0000882341F09091C00095FFFCCF8093C600CC
:102F10003196F5CF2FB7F89460911013709111137B
:102F200080911213909113132FBF0E94A7BE20917E
:102F300040133091411340914213509143130E942A
:102F400067C542E00E947D278091C00085FFFCCFCD
:102F50008AE08093C6000C94A12180E00E94BCA866
:102F60000C94A12181E00E94BCA80C94A121909115
:102F7000C00095FFFCCF8093C60081918111F7CFEF
:102F80008091C00085FFFCCF8AE08093C600E5E514
:102F9000F4E08491882341F09091C00095FFFCCF2C
:102FA0008093C6003196F5CF659B03C0E1EDF2E05A
:102FB00009C0E6EDF2E006C09091C00095FFFCCF9D
:102FC0008093C60081918111F7CF8091C00085FF69
:102FD000FCCF8AE08093C600EDE4F4E0849188237E
:102FE00041F09091C00095FFFCCF8093C6003196D0
:102FF000F5CF649B03C0E1EDF2E009C0E6EDF2E03D
:1030000006C09091C00095FFFCCF8093C6008191CF
:103010008111F7CF8091C00085FFFCCF8AE08093BB
:10302000C600E5E4F4E08491882341F09091C0006B
:1030300095FFFCCF8093C6003196F5CF80910301B8
:1030400081FF03C0E1EDF2E009C0E6EDF2E006C069
:103050009091C00095FFFCCF8093C60081918111B3
:10306000F7CF8091C00085FFFCCF8AE08093C60037
:10307000EDE3F4E08491882341F09091C00095FF46
:10308000FCCF8093C6003196F5CF4B9B03C0E1ED9A
:10309000F2E009C0E6EDF2E006C09091C00095FFB5
:1030A000FCCF8093C60081918111F7CF8091C00041
:1030B00085FFFCCF8AE08093C6000C94A1219CE59B
:1030C000E92E93E1F92E07EC12E024E0D22ED00E87
:1030D000D8018D918D010E94E4AD882349F00E94B2
:1030E0000AAE0E94DEC5F7016083718382839383F9
:1030F000F4E0EF0EF11CD012EBCF0E94016E0C94A5
:10310000A121F4E0EF0EF11CD01611F40C94A121D2
:10311000D8018D918D010E94E4AD882391F30E9426
:103120000AAEF7016083718382839383EACF83E5DC
:103130000E94E4AD882351F00E940AAE6093AD1264
:103140007093AE128093AF129093B01284E50E94F8
:10315000E4AD882311F40C94A1210E940AAE60937F
:10316000B1127093B2128093B3129093B4120C9474
:10317000A12183E50E94E4AD882351F00E940AAEAC
:103180006093C9127093CA128093CB129093CC12A1
:1031900084E50E94E4AD882351F00E940AAE60935A
:1031A000CD127093CE128093CF129093D01282E4FE
:1031B0000E94E4AD882361F00E940AAE0E94DEC541
:1031C0006093C5127093C6128093C7129093C81271
:1031D00088E50E94E4AD882351F00E940AAE609316
:1031E000A9127093AA128093AB129093AC128AE545
:1031F0000E94E4AD882351F00E940AAE6093A512AC
:103200007093A6128093A7129093A81285E40E944F
:10321000E4AD882311F40C94A1210E940AAE6093BE
:10322000A1127093A2128093A3129093A4120C94F3
:10323000A121ADE0EA2EA9E1FA2E07EC12E0B3E0FD
:10324000DB2ED00ED8018D918D010E94E4AD882334
:1032500039F00E940AAEF701608371838283938301
:10326000F4E0EF0EF11CD012EDCF0C94A1218AED09
:1032700090E00E94BE9C81110C94A12188E50E94DF
:10328000E4AD882381F00091A01810E00E940AAEFE
:10329000000F111F000F111FF801E15EFF4E608348
:1032A00071838283938389E50E94E4AD882381F052
:1032B0000091A01810E00E940AAE000F111F000F2D
:1032C000111FF801E95DFF4E608371838283938350
:1032D0008AE50E94E4AD882381F00091A01810E0F7
:1032E0000E940AAE000F111F000F111FF801E15DCF
:1032F000FF4E6083718382839383E6E7F8E08491D5
:10330000882341F09091C00095FFFCCF8093C600C8
:103310003196F5CFEDE2F4E08491882341F090916D
:10332000C00095FFFCCF8093C6003196F5CF109278
:10333000A0188091A018823008F058C0EFE1F4E0A6
:103340008191882339F09091C00095FFFCCF809344
:10335000C600F6CFE091A01824E0E29FF00111240E
:10336000E15EFF4E608171818281938142E00E9423
:103370007D2704E913E0F8018191882339F09091C9
:10338000C00095FFFCCF8093C600F6CFE091A01857
:1033900034E0E39FF0011124E95DFF4E608171810B
:1033A0008281938142E00E947D27D8018D918D0119
:1033B000882339F09091C00095FFFCCF8093C60020
:1033C000F4CFE091A018B4E0EB9FF0011124E15D8F
:1033D000FF4E608171818281938142E00E947D274E
:1033E0008091A0188F5F8093A018A3CF8091C00018
:1033F00085FFFCCF8AE08093C600A3C783E50E94C7
:10340000E4AD882309F49DC70E940AAE0E94D8C586
:10341000709362026093610294C783E50E94E4ADF9
:10342000882309F48EC70E940AAE0E94D8C5709303
:10343000100260930F0285C780E50E94E4AD8823E7
:1034400051F00E940AAE609342027093430280934F
:1034500044029093450289E40E94E4AD882381F000
:103460000E940AAE2DEB37E346E05EE30E94FEB811
:1034700060933E0270933F0280934002909341021A
:1034800084E40E94E4AD882381F00E940AAE2DEB13
:1034900037E346E05EE30E9467C560933A027093AB
:1034A0003B0280933C0290933D0283E40E94E4AD92
:1034B000882351F00E940AAE6093000270930102CB
:1034C00080930202909303020E94A3A8E6E9F3E02E
:1034D0008191882339F09091C00095FFFCCF8093B3
:1034E000C600F6CFE9E9F3E08191882339F09091A5
:1034F000C00095FFFCCF8093C600F6CF60914202DA
:1035000070914302809144029091450242E00E94F2
:103510007D27EDE9F3E08191882339F09091C00097
:1035200095FFFCCF8093C600F6CF2DEB37E346E046
:103530005EE360913E0270913F0280914002909163
:1035400041020E9467C542E00E947D27E1EAF3E064
:103550008191882339F09091C00095FFFCCF809332
:10356000C600F6CF2DEB37E346E05EE360913A020A
:1035700070913B0280913C0290913D020E94FEB806
:1035800042E00E947D27E5EAF3E08191882339F04B
:103590009091C00095FFFCCF8093C600F6CF60915C
:1035A000000270910102809102029091030242E0B8
:1035B0000E947D278091C00085FFFCCF8AE0809328
:1035C000C6000E94753EBDC683E50E94E4AD882317
:1035D00019F00E940AAE03C060E070E0CB01609376
:1035E000D1127093D2128093D3129093D412A9C6A1
:1035F00085E40E94E4AD882341F00E940AAE0E9457
:10360000D8C58B0177FD12C002C000E010E02D96F6
:103610001FAE2D972E961FAE2E97E6E12F96EFAF99
:103620002F97F3E46096FFAF60970EC02D961FAE04
:103630002D972E961FAE2E972CE82F962FAF2F97F3
:1036400032E460963FAF609783E50E94E4AD882343
:1036500071F00E940AAE2D966FAF2D972E967FAF18
:103660002E972F968FAF2F9760969FAF609783E42A
:103670000E94E4AD882349F00E940AAE0E94D8C59A
:10368000AC967FAF6EAFAC9706C045E050E0AC960D
:103690005FAF4EAFAC970E940D352C966CAF7DAFEF
:1036A0008EAF9FAF2C97033011051CF4E9EAF3E0CD
:1036B0001AC0ECEBF3E08191882339F09091C000BF
:1036C00095FFFCCF8093C600F6CF8091C00085FFA8
:1036D000FCCF8AE08093C60034C69091C00095FF6D
:1036E000FCCF8093C60081918111F7CF8091C000FB
:1036F00085FFFCCF8AE08093C6000E9463358FE788
:1037000017FF68C0809366122C968CAD9DADAEAD50
:10371000BFAD2C976A968CAF9DAFAEAFBFAF6A9727
:10372000E0968CAF9DAFAEAFBFAFE09761961FAE96
:10373000619790E46F969FAF6F97ACE1A096AFAFA3
:10374000A097B6E4A196BFAFA1976B961FAE6B97FB
:103750006C961FAE6C976D961FAE6D976E961FAEF2
:103760006E972FE730E040E050E028962CAF3DAF59
:103770004EAF5FAF28973FE7432E512C612C712C41
:10378000A8961CAE1DAE1EAE1FAEA89731E0A29645
:103790003FAFA29766961FAE1EAE669722961FAEEB
:1037A0002297212C312C23961FAE2397A80149592B
:1037B0005D4EAA965FAF4EAFAA97C801880F991FBA
:1037C000880F991FDC01A95ABD4EA496BFAFAEAFBA
:1037D000A49707C0F801E959FD4E808395CF0E9458
:1037E000813280916512882309F478C10E946C3A75
:1037F00017FF0FC0B09147122296BFAF22972090BB
:10380000481230904912E0914A122396EFAF239765
:1038100012C0A496AEADBFADA497BC912296BFAF27
:103820002297A496EEADFFADA49721803280F3815C
:103830002396FFAF239722962FAD2297322D432D4B
:1038400023965FAD23976B966FAD6B976C967FADAC
:103850006C976D968FAD6D976E969FAD6E970E942B
:10386000C4C6181694F022962FAD22976B962FAFF0
:103870006B976C962FAE6C976D963FAE6D972396B7
:103880003FAD23976E963FAF6E9722962FAD22974E
:10389000322D432D23965FAD239761966FAD6197CF
:1038A0006F967FAD6F97A0968FADA097A1969FADB5
:1038B000A1970E94A1BE87FD12C022964FAD22970C
:1038C00061964FAF61976F962FAE6F97A0963FAE00
:1038D000A09723965FAD2397A1965FAFA197A2967D
:1038E0008FADA297882309F479C02D962FAD2D971F
:1038F0002E963FAD2E972F964FAD2F9760965FADCA
:10390000609722966FAD2297722D832D23969FADDF
:1039100023970E94C4C618160CF0E0C00E940D3513
:10392000DC01CB012C962CAD3DAD4EAD5FAD2C979F
:10393000821B930BA40BB50B89389341A105B105EC
:1039400008F4CCC0D301C20128962CAD3DAD4EADDC
:103950005FAD2897821B930BA40BB50BB595A7956C
:103960009795879517FF03C08093661205C0AA96A6
:10397000EEADFFADAA9780830E940D356A966CAFBD
:103980007DAF8EAF9FAF6A979B01AC012C968CAD3B
:103990009DADAEADBFAD2C97281B390B4A0B5B0B11
:1039A000A8962CAF3DAF4EAF5FAFA8972D969FADB9
:1039B0002D976B969FAF6B972E96AFAD2E976C960B
:1039C000AFAF6C972F96BFAD2F976D96BFAF6D972A
:1039D0006096EFAD60976E96EFAF6E972D962FAD18
:1039E0002D972E963FAD2E972F964FAD2F97609621
:1039F0005FAD609722966FAD2297722D832D23962F
:103A00009FAD23970E94A1BE87FF5CC70E940D3522
:103A1000DC01CB016A962CAD3DAD4EAD5FAD6A9732
:103A2000821B930BA40BB50B89389341A105B105FB
:103A300008F448C70E940D352C966CAF7DAF8EAF51
:103A40009FAF2C97DC01CB016A962CAD3DAD4EADFE
:103A50005FAD6A97821B930BA40BB50B66964EADB8
:103A60005FAD6697141615060CF45FC528968CADED
:103A70009DADAEADBFAD2897840D951DA61DB71D9C
:103A8000B595A7959795879517FF16C780936612EA
:103A900066962EAD3FAD66972F5F3F4F66963FAF60
:103AA0002EAF66972D963FAD2D9761963FAF6197EC
:103AB0002E964FAD2E976F964FAF6F972F965FADA7
:103AC0002F97A0965FAFA09760968FAD6097A19655
:103AD0008FAFA19791E0A2969FAFA29720E030E030
:103AE00040EA51E42D966FAD2D972E967FAD2E971F
:103AF0002F968FAD2F9760969FAD60970E9479C4E7
:103B00009B01AC0122966FAD2297722D832D2396D7
:103B10009FAD23970E94C4C61816ACF4E8E9F3E001
:103B20008491882341F09091C00095FFFCCF809351
:103B3000C6003196F5CF8091C00085FFFCCF8AE0AA
:103B40008093C600FEC30E940D35DC01CB01E096D8
:103B50002CAD3DAD4EAD5FADE097821B930BA40B3A
:103B6000B50B813D9740A105B10508F452C017FF80
:103B700010C0E0906612F12CE2E9F3E08491882312
:103B8000D9F09091C00095FFFCCF8093C60031968C
:103B9000F5CFAA96AEADBFADAA97EC90F12CECE8AC
:103BA000F3E08491882341F09091C00095FFFCCF11
:103BB0008093C6003196F5CF42E022966FAD2297F2
:103BC000722D832D23969FAD23970E947D27E8E8D1
:103BD000F3E08491882341F09091C00095FFFCCFE1
:103BE0008093C6003196F5CFB701FF0C880B990B77
:103BF0000E946B278091C00085FFFCCF8AE08093F4
:103C0000C6000E940D35E0966CAF7DAF8EAF9FAFC2
:103C1000E0970E940D356B017C010E940D356A967C
:103C20008CAC9DACAEACBFAC6A972C962CAD3DADC8
:103C30004EAD5FAD2C97820E931EA41EB51EC81804
:103C4000D908EA08FB08DC01CB018C0D9D1DAE1DD7
:103C5000BF1D81389F44A241B105A8F0EBE6F3E017
:103C60008491882341F09091C00095FFFCCF809310
:103C7000C6003196F5CF8091C00085FFFCCF8AE069
:103C80008093C6005EC366964EAD5FAD6697AC96F8
:103C90008EAD9FADAC97841795070CF0A0CDEFE1EA
:103CA000F3E08491882341F09091C00095FFFCCF10
:103CB0008093C6003196F5CF8091C00085FFFCCF80
:103CC0008AE08093C6003DC30E9428A93AC30E949F
:103CD000484137C30E94A23F0E944D6E32C30E94EA
:103CE0009F3A2FC380E090E00E944F810E9428A954
:103CF00083E50E94E4AD882341F00E940AAE0E9451
:103D0000D8C57093140260931302809113029091AE
:103D100014028230910509F0BFC088E50E94E4AD2D
:103D2000882349F10E940AAE6B017C010E9438543D
:103D30009B01AC0160E070E0CB010E9478C49B0164
:103D4000AC01C701B6010E94C4C618161CF40E943B
:103D50000AAE09C00E9438549B01AC0160E070E0DB
:103D6000CB010E9478C46093040270930502809393
:103D700006029093070282E50E94E4AD882351F089
:103D80000E940AAE60931A0B70931B0B80931C0B5E
:103D900090931D0BE6E7F8E08491882341F0909121
:103DA000C00095FFFCCF8093C6003196F5CFE8E0C8
:103DB000F4E08491882341F09091C00095FFFCCFFE
:103DC0008093C6003196F5CF6FE1E62E64E0F62EC3
:103DD000F7018191882339F09091C00095FFFCCFC5
:103DE0008093C600F6CF60911F10709120108091D3
:103DF00021109091221042E00E947D2704E913E0F7
:103E0000F8018191882339F09091C00095FFFCCF93
:103E10008093C600F6CF6091271070912810809192
:103E2000291090912A1042E00E947D27D7018D91A0
:103E30007D01882339F09091C00095FFFCCF8093DD
:103E4000C600F4CF609104027091050280910602D1
:103E50009091070242E00E947D27F80181918F0135
:103E6000882339F09091C00095FFFCCF8093C60065
:103E7000F4CF60912B1070912C1080912D109091A7
:103E80002E1042E00E947D278091C00085FFFCCF6C
:103E90008AE08093C60008C0049730F081E090E08B
:103EA00090931402809313021092191980911302B7
:103EB00090911402909312028093110210921A1999
:103EC00010921B1910921C1910921D193AC283E509
:103ED0000E94E4AD882309F434C20E940AAE0E9415
:103EE000D8C57093FF126093FE126531710534F0EE
:103EF00084E190E09093FF128093FE128091FE1275
:103F00009091FF1297FD02C00C94AA161092FF1216
:103F10001092FE120C94AA1686EE93E00E94116590
:103F200010C20E94CF840DC282E50E94E4AD8823B6
:103F300029F00E940AAE9B01AC0104C020E030E0F1
:103F400040E85FE383E5E3962FAFE397E4963FAF66
:103F5000E497E5964FAFE597E6965FAFE6970E9448
:103F6000E4AD882309F4EDC10E940AAEE3962FADBB
:103F7000E397E4963FADE497E5964FADE597E69677
:103F80005FADE6970E9467C560931B1070931C108D
:103F900080931D1090931E100E94753ED2C182E541
:103FA0000E94E4AD882329F00E940AAE9B01AC0177
:103FB00004C020E030E040E85FE383E5E3962FAF04
:103FC000E397E4963FAFE497E5964FAFE597E69623
:103FD0005FAFE6970E94E4AD882309F4B2C10E9466
:103FE0000AAEE3962FADE397E4963FADE497E596EE
:103FF0004FADE597E6965FADE6970E9467C5609383
:104000003710709338108093391090933A100E94B3
:10401000753E97C182E50E94E4AD882329F00E9495
:104020000AAE9B01AC0104C020E030E040E85FE351
:1040300083E5E3962FAFE397E4963FAFE497E596E9
:104040004FAFE597E6965FAFE6970E94E4AD882311
:1040500009F477C10E940AAEE3962FADE397E49688
:104060003FADE497E5964FADE597E6965FADE697F1
:104070000E9467C56093300B7093310B8093320BB5
:104080009093330B0E94753E5CC183E50E94E4ADC2
:10409000882309F456C10E940AAE0E94D8C565362D
:1040A00071052CF477FF05C060E070E002C064E6A3
:1040B00070E070939718609396180E94753E41C106
:1040C00083E50E94E4AD882309F43BC10E940AAE57
:1040D0000E94D8C5693C71052CF477FF05C060E0EB
:1040E00070E002C068EC70E07093951860939418CB
:1040F0000E94753E26C183E50E94E4AD882309F441
:1041000020C10E940AAE0E94D8C521E030E0613093
:10411000710511F020E030E03093370B2093360B1F
:104120000E94753E0EC183E50E94E4AD882309F428
:1041300008C10E940AAE0E94D8C56D3371052CF4E7
:1041400077FF05C060E070E002C06CE370E0709340
:104150002F0B60932E0B0E94753EF3C082E40E94E9
:10416000E4AD882351F00E940AAE0E94D8C5709336
:10417000B0186093AF180E94753E85E40E94E4ADCC
:10418000882309F4DEC00E940AAE0E94D8C570934D
:104190002D0B60932C0B70932B0B60932A0B0E94BA
:1041A000753ECFC083E50E94E4AD81118FC3C9C0C5
:1041B00083E50E94E4AD882309F4C3C00E940AAEDF
:1041C0000E94D8C58B0184E50E94E4AD882329F0C4
:1041D0000E940AAE0E94D8C502C06FEF7FEF023086
:1041E000110508F0AEC08091061390E068177907BA
:1041F00009F4DCC36F3FFFEF7F0709F4D7C3CB019E
:104200000E944F81D3C3109201131092001399C0E2
:104210000E94785496C00E94475493C080E090E07A
:104220000E942B9B8EC083E50E94E4AD882309F495
:1042300088C00E940AAE6B017C0120E030E0A90139
:104240000E94A1BE811104C081E080935F0279C009
:1042500020E030E040E251E4C701B6010E9467C5AA
:104260006093A4187093A5188093A6189093A7182C
:1042700010925F0266C01092071380919C18909173
:104280009D18A0919E18B0919F188093C50B909394
:10429000C60BA093C70BB093C80B0E949C9AE0E09A
:1042A000F0E019954EC084E50E94E4AD882329F022
:1042B0008FEF9FEF0E944F8144C0E6E7F8E08491C2
:1042C000882341F09091C00095FFFCCF8093C600F9
:1042D0003196F5CFEAE1F4E08491882341F09091A2
:1042E000C00095FFFCCF8093C6003196F5CF80913A
:1042F000E00B9091E10B20E6289FF001299FF00D43
:104300001124E651F44F8191882339F09091C00037
:1043100095FFFCCF8093C600F6CFE8E1F4E08491EE
:10432000882341F09091C00095FFFCCF8093C60098
:104330003196F5CF8091C00085FFFCCF8AE0809355
:10434000C6000E94749ACFC3819187FD02C00C946D
:10435000BB10D12C0C94C5106EE470E1CE01019617
:104360000E940F90BE016F5F7F4FCE01CB960E94DF
:10437000438FCE0101960E947C8FCE01CB960E9486
:10438000378DBE01655C7F4FCE0180960E940790FD
:104390000F5F1F4FC090340BD090350BB6E0BC9D23
:1043A000C001BD9D900D1124801791070CF077C0BE
:1043B0000696801791070CF472C061E470E1CE019B
:1043C00001960E940F90BE016F5F7F4FCE01CB968A
:1043D0000E94438FCE0101960E947C8FCE01CB9626
:1043E0000E94378D68E374E0CE0180960E94928E21
:1043F000882339F0BE01655C7F4FCE0180960E9414
:104400002E8F4AEF96014203C001439F900D112465
:104410006801C80ED91E87E293E00E940F654AE04A
:10442000B601CE0101960E94DC8F89819A810E949B
:104430000F65CE0101960E947C8F85ED99E00E9468
:104440000F65CE0180960E94378D88A199A10E94A8
:104450000F6588EB94E00E940F650E94036586E378
:1044600093E00E940F654AE0B601CE0101960E94DA
:10447000DC8F89819A810E940F65CE0101960E948E
:104480007C8F85ED99E00E940F658BAD9CAD0E94FD
:104490000F6588EB94E00E940F650E940365CE01D2
:1044A00080960E947C8F0C94D1100E94FFADAB01CE
:1044B000BC0140936C1050936D1060936E1070931C
:1044C0006F1083E192E10E94F85C3BCF0E940AAE3C
:1044D00038CF0E9428A988E50E94E4AD882311F016
:1044E0005F9A479A89E50E94E4AD81118A9A8AE52C
:1044F0000E94E4AD882381F09FB7F8948091080171
:104500008160809308019FBF9FB7F8948091080154
:104510008460809308019FBF85E40E94E4AD8823F6
:1045200009F40FCF8D9A129A0CCFA8968CAC9DAC43
:10453000AEACBFACA897880E991EAA1EBB1EA8964B
:104540002CAD3DAD4EAD5FADA897281B390B4A0B86
:104550005B0BCA01B90128962CAD3DAD4EAD5FADE8
:1045600028970E942EC4A50194010E942FC8D30150
:10457000C201820F931FA41FB51F84319105A105AD
:10458000B1050CF12C013D018C3E9105A105B10551
:104590002CF0FBEE4F2E512C612C712C40E8441670
:1045A000510461047104FCF08EEF90E0A0E0B0E0F3
:1045B00084199509A609B70928968CAF9DAFAEAFAF
:1045C000BFAF289716C0E4E14E2E512C612C712C00
:1045D00024E130E040E050E028962CAF3DAF4EAFF4
:1045E0005FAF289706C028964CAE5DAE6EAE7FAE2C
:1045F0002897E0E0F4E08491882341F09091C00096
:1046000095FFFCCF8093C6003196F5CFC301B20170
:1046100062D4EBEFF3E08491882341F09091C000E5
:1046200095FFFCCF8093C6003196F5CF28966CADF0
:104630007DAD8EAD9FAD28974ED4E4EFF3E084912D
:10464000882341F09091C00095FFFCCF8093C60075
:104650003196F5CF42E061966FAD61976F967FAD71
:104660006F97A0968FADA097A1969FADA19745D4C7
:10467000EDEEF3E08491882341F09091C00095FF26
:10468000FCCF8093C6003196F5CF42E06B966FADBC
:104690006B976C967FAD6C976D968FAD6D976E96A0
:1046A0009FAD6E972AD48091C00085FFFCCF8AE031
:1046B0008093C60066962EAD3FAD669723303105D8
:1046C0000CF4D4C928966CAD7DAD8EAD9FAD289706
:1046D0000E94A7BE20E030E040E850E40E94FEB80F
:1046E0006B017C0161962FAD61976F963FAD6F971F
:1046F000A0964FADA097A1965FADA1976B966FADB9
:104700006B976C967FAD6C976D968FAD6D976E962F
:104710009FAD6E970E9478C420ED3FE049E450E4DD
:104720000E94FEB820E030E040E05FE30E94FEB867
:104730009B01AC01C701B6010E9467C56B017C01FA
:10474000C501B4010E94A7BE20E030E04AE754E46E
:104750000E9467C54B015C01E7EEF3E0849188237A
:1047600041F09091C00095FFFCCF8093C600319638
:10477000F5CF42E0C701B601C0D3E1EEF3E084918A
:10478000882341F09091C00095FFFCCF8093C60034
:104790003196F5CF42E0C501B401AFD38091C0009E
:1047A00085FFFCCF8AE08093C6002AE939E949E118
:1047B0005FE3C701B6010E94FEB86B017C019B015B
:1047C000AC010E9479C4A50194010E9467C564965A
:1047D0006CAF7DAF8EAF9FAF6497A5019401C70109
:1047E000B6010E94FEB820E030E040E05EE30E94A7
:1047F000FEB84B015C01E4EDF3E08491882341F0C5
:104800009091C00095FFFCCF8093C6003196F5CF04
:104810008091C00085FFFCCF8AE08093C600EEEC5B
:10482000F3E08491882341F09091C00095FFFCCF84
:104830008093C6003196F5CF42E0C701B6015DD343
:104840008091C00085FFFCCF8AE08093C600E8EC31
:10485000F3E08491882341F09091C00095FFFCCF54
:104860008093C6003196F5CF42E064966CAD7DAD85
:104870008EAD9FAD649741D38091C00085FFFCCF82
:104880008AE08093C600E2ECF3E08491882341F053
:104890009091C00095FFFCCF8093C6003196F5CF74
:1048A00042E0C501B40129D38091C00085FFFCCF4F
:1048B0008AE08093C600DAC8AA96EEADFFADAA974B
:1048C0008083E6C8A2961FAEA29708C90E940AAECE
:1048D0000E94D8C561157105F9F48091280B90915B
:1048E000290B9093FA128093F9129093FC12809303
:1048F000FB128091260B9091270B9093DF0B8093F6
:10490000DE0B8091240B9091250B9093A918809336
:10491000A8180E94603915CD61307105F9F48091B5
:10492000220B9091230B9093FA128093F91290939B
:10493000FC128093FB128091200B9091210B90939D
:10494000DF0B8093DE0B80911E0B90911F0B9093D9
:10495000A9188093A8180E946039F3CC62307105C1
:1049600069F41092FA121092F9121092FC1210923D
:10497000FB121092DF0B1092DE0BE3CC633071055B
:1049800009F0DFCC1092FA121092F9121092FC1278
:104990001092FB121092DF0B1092DE0B0E9428A9DE
:1049A0008D9A129A80E00E94E7A8CBCC012B09F0E7
:1049B0004DC020E030E044EB52E46091241370914C
:1049C000251380912613909127130E9479C4609338
:1049D000241370932513809326139093271336E0A6
:1049E000C32E33E1D32EE12CF12C00E211E424E2BA
:1049F00033E140E253E16CE173E188E193E10E942D
:104A0000834520E030E040EA51E460912413709146
:104A1000251380912613909127130E9479C46093E7
:104A20002413709325138093261390932713E12C5E
:104A3000F12C00E010E424E233E140E253E16CE1C8
:104A400073E188E193E10E9483457BCC20E030E074
:104A500040EF51E460912413709125138091261347
:104A6000909127130E9479C46093241370932513A7
:104A7000809326139093271386E0C82E83E1D82EC7
:104A8000E12CF12C00E010E424E233E140E253E1B8
:104A90006CE173E188E193E10E94834520E030E01E
:104AA00040EF52E4609124137091251380912613F6
:104AB000909127130E9478C4609324137093251358
:104AC0008093261390932713E12CF12C08E412E431
:104AD00024E233E140E253E16CE173E188E193E1E8
:104AE0000E9483452ECCE296AEADBFADE2970FB6E5
:104AF000F894BEBF0FBEADBFCB58DF4F0FB6F894D2
:104B0000DEBF0FBECDBFDF91CF911F910F91FF9000
:104B1000EF90DF90CF90BF90AF909F908F907F905D
:104B20006F905F904F903F902F9008954F925F92BB
:104B30006F927F928F929F92AF92BF92FF920F934C
:104B40001F93CF93DF93182F8CEE91E19093780F02
:104B50008093770F1092081282E090E0A0E0B0E01E
:104B60008093F1119093F211A093F311B093F4118B
:104B70001092760F1092720F1092730F1092740FA2
:104B80001092750F8FEF9FEFDC0180936E0F909363
:104B90006F0FA093700FB093710F112379F115303F
:104BA00008F0F9C040E060E070E0CB010E94EC72D8
:104BB000882309F4F0C020E1129FC0011124825A19
:104BC000924FFC01E254FE4F20812F7709F0E3C0A1
:104BD0003C96408151816281738144365105610563
:104BE000710508F4D8C0349780809180A280B3808A
:104BF00081149104A104B10421F4CDC0812C912C25
:104C0000540140E0C501B4010E94EC72F82E8823E3
:104C100009F4C1C08091790D90917A0D811592406F
:104C200009F0B9C0A0917E0DAA2309F4B4C0609127
:104C30007C0D70917D0D6115710509F4ACC020915A
:104C40007B0D222309F4A7C0A09303122093F51132
:104C500080E030E0E1E0F0E0C82FAF01082E02C0B4
:104C6000440F551F0A94E2F72417350741F0982F97
:104C70008F5F983089F789E08093FE118CC0809314
:104C8000FE112091840D3091850D2115310519F00B
:104C900040E050E008C02091920D3091930D40917A
:104CA000940D5091950D2093F6113093F711409388
:104CB000F8115093F91124013501460E571E611C5D
:104CC000711C40920412509205126092061270926A
:104CD0000712E0917F0DF091800DF0930A12E0939E
:104CE0000912B0E00E945FC4460E571E681E791E6E
:104CF00040920B1250920C1260920D1270920E1292
:104D000085E0EE0FFF1F8A95E1F7E150FE4FEF2F90
:104D1000FF27E6954E0E5F1E611C711C4092FF112D
:104D20005092001260920112709202122091810D35
:104D30003091820D2115310521F0890120E030E00C
:104D400008C000918E0D10918F0D2091900D309123
:104D5000910DB501A4014419550966097709400F61
:104D6000511F621F731F04C076956795579547952D
:104D7000CA95D2F74093FA115093FB116093FC113E
:104D80007093FD11453F2FE052076105710528F42E
:104D90008CE080930812F12C1AC0453F5F4F6105EB
:104DA000710510F480E111C080919A0D90919B0DD6
:104DB000A0919C0DB0919D0D80930B1290930C12BD
:104DC000A0930D12B0930E1280E2809308128F2DE3
:104DD000DF91CF911F910F91FF90BF90AF909F9067
:104DE0008F907F906F905F904F9008954F925F9259
:104DF0006F927F928F929F92AF92BF92EF92FF92AB
:104E00000F931F93CF93DF93CDB7DEB7A0970FB665
:104E1000F894DEBF0FBECDBF611571058105910508
:104E200041F48091C00085FFFCCF80E38093C600F1
:104E30003DC09E012F5F3F4F7901812C912C540181
:104E40008901442E512C612C712C3FEF831A930A57
:104E5000A30AB30AA30192010E943DC4F701619322
:104E60007F01B901CA01611571058105910569F7D5
:104E7000A40120E030E0F1E08F1A9108A108B10808
:104E8000F401E21BF30BE00FF11F80818A3010F474
:104E9000805D01C0895C9091C00095FFFCCF80933C
:104EA000C6002F5F3F4F2417350751F7A0960FB666
:104EB000F894DEBF0FBECDBFDF91CF911F910F9150
:104EC000FF90EF90BF90AF909F908F907F906F90EA
:104ED0005F904F90089597FF0EC02091C00025FF6E
:104EE000FCCF2DE22093C60090958095709561953A
:104EF0007F4F8F4F9F4F4AE079CF8F929F92AF9213
:104F0000BF92CF92DF92EF92FF92CF93DF936B012C
:104F10007C01C42F20E030E0A9010E94A1BE87FFE0
:104F20000BC08091C00085FFFCCF8DE28093C6004E
:104F3000F7FAF094F7F8F094D0E060E070E080E0E9
:104F40009FE3DC1741F020E030E040E251E40E94B2
:104F500067C5DF5FF6CF9B01AC01C701B6010E94B8
:104F600079C46B017C010E94DEC54B015C010E948B
:104F7000A5BE9B01AC01C701B6010E9478C46B01BC
:104F80007C014AE0C501B40131DFCC2361F0E2E2EB
:104F9000F5E08191882339F09091C00095FFFCCF16
:104FA0008093C600F6CFCC2309F120E030E040E248
:104FB00051E4C701B6010E94FEB84B015C010E949A
:104FC000D8C56B01770FEE08FF08C701B60183DF74
:104FD000C701B6010E94A7BE9B01AC01C501B40187
:104FE0000E9478C46B017C01C150DDCFDF91CF916D
:104FF000FF90EF90DF90CF90BF90AF909F908F90F9
:105000000895682F8AE79FE00C94C38C009769F09D
:10501000FC0101900020E9F73197AF01481B590BC3
:10502000BC018AE79FE00C94F88B80E090E0089543
:10503000BC0180E090E04AE0D9DE8091C00085FFAD
:10504000FCCF8DE08093C6008091C00085FFFCCF2F
:105050008AE08093C60008958F929F92AF92BF928C
:10506000CF92DF92EF92FF920F931F93CF93DF9334
:1050700000D01F92CDB7DEB7FC018381813011F0E3
:1050800080E06BC0818181FFFBCF81899289A389F8
:10509000B489892B8A2B8B2B09F45EC07F0140E0F9
:1050A00050E0BA01CF010E94F85C882349F3F70170
:1050B00085889688A788B08CC18CD28C82E090E0DD
:1050C000A0E0B0E0F60180839183A283B3839E01C8
:1050D0002F5F3F4FB501A401C6010E94B57388231D
:1050E00079F200E010E09801B501A401C6010E9428
:1050F0002473882329F289809A80AB80BC80F601D2
:105100008789803141F4F8EF8F16FFEF9F06A104E5
:10511000B10448F4DCCF88EF88168FEF9806A80614
:105120008FE0B806A0F2F701158A168A178A108E4A
:10513000118A128A138A148A818180688183C70147
:105140000E940775882309F49BCF40E050E0BA0124
:10515000C7010E94F85C01C081E00F900F900F9092
:105160000F90DF91CF911F910F91FF90EF90DF9003
:10517000CF90BF90AF909F908F90089568E374E0B8
:105180000E94928E91E0811190E0892F08952F92D4
:105190003F924F925F926F927F928F929F92AF92C7
:1051A000BF92CF92DF92EF92FF920F931F93CF9314
:1051B000DF93CDB7DEB7CE55D1090FB6F894DEBF79
:1051C0000FBECDBF80916B108F9380916A108F932B
:1051D00087E898E09F938F938E01015C1F4F1F9388
:1051E0000F930E9472BE0F900F900F900F900F9030
:1051F0000F90F12CF80101900020E9F73197E01BA6
:10520000F10BFE1684F46801CF0CD11CF7FCDA9484
:10521000F6018081082E000C990B0E9445C9F60109
:105220008083F394E7CF40E050E0BA0188E790E153
:105230000E94F85C6E961FAE6E97CE0101967C01BF
:1052400080E8A82E88E0B82E6E0191E2C90ED11C2C
:1052500096E7292E98E0392E2BE6422E28E0522E92
:1052600034E0832E912C80917B10823040F46E9636
:105270002FAD6E97211114C08FEF9FEF16C0809154
:10528000801090918110A0918210B09183108F7145
:105290009927AA27BB27892B8A2B8B2B41F723C061
:1052A00080916A1090916B10019690936B1080938F
:1052B0006A10C25ADF4F0FB6F894DEBF0FBECDBFE3
:1052C000DF91CF911F910F91FF90EF90DF90CF90E2
:1052D000BF90AF909F908F907F906F905F904F9016
:1052E0003F902F90089540E050E0B70188E790E1AB
:1052F0000E949C7418160CF0BACF20E0F7010190C0
:105300000020E9F73197EE19FF092E17A4F43701B1
:10531000620E711C27FD7A94F301808190E06F96F4
:105320002FAF6F970E9445C9F30180836F962FAD11
:105330006F972F5FE3CF8A858E3709F494CF45E0CE
:1053400050E0B801C7010E949AC9892B09F08BCFA0
:105350001F930F93BF92AF92DF92CF920E9472BEC3
:105360000F900F900F900F900F900F9080916C0DF9
:1053700090916D0D04970CF06CC020916A0D3091E6
:105380006B0DF0E6F29FC001F39F900D1124B60162
:105390008651944F0E9493C9F1018491E6E7F8E0A9
:1053A000882349F09091C00095FFFCCF8093C60000
:1053B00031968491F5CFF2018491EBE6F8E08823F1
:1053C00049F09091C00095FFFCCF8093C6003196C4
:1053D0008491F5CF80916A0D90916B0D20E6289F06
:1053E000F001299FF00D1124E651F44F819188239B
:1053F00039F09091C00095FFFCCF8093C600F6CFA6
:10540000E9E6F8E08491882341F09091C00095FF8F
:10541000FCCF8093C6003196F5CF8091C00085FF08
:10542000FCCFFAE0F093C60080916A0D90916B0D6D
:105430000196B4010E941CC890936B0D80936A0D75
:1054400080916C0D90916D0D019690936D0D8093F0
:105450006C0D80916C0D90916D0D049724F48CE788
:1054600098E00E94CD5321E06E962FAF6E97FBCE51
:10547000CF92DF92EF92FF921F93CF93DF93109220
:10548000401080917B10882321F088E790E10E94F2
:10549000E15D1092F0111092ED1185E38093EC1113
:1054A0000E940D35EB0161E08091EC110E94D23336
:1054B0008CEE91E10E94F45E60E082E30E94D233C0
:1054C00061E083E30E94D23361E084E30E94D2333F
:1054D00061E085E30E94D23361E085E30E94A3335B
:1054E00085E08093EE1182E58CBD1DBC1AE08FEF44
:1054F0000E94F95E1150D9F720E030E0A90160E088
:105500008CEE91E10E941F5F182F8093EF11813084
:1055100049F00E940D356C1B7D0B613D774060F3B7
:1055200081E054C02AEA31E040E050E068E08CEECF
:1055300091E10E941F5F82FF03C01093F0110EC023
:1055400014E00E94FE5E8093EF111150D1F78A3A69
:1055500011F082E03BC082E08093F0118091F01165
:10556000823021F0C12CD12C760105C0C12CD12C68
:10557000E12C80E4F82E20E030E0A90167E38CEE16
:1055800091E10E941F5FA701960169E28CEE91E113
:105590000E941F5F8093EF11882349F00E940D3510
:1055A0006C1B7D0B613D774030F38AE00FC080912A
:1055B000F011823011F520E030E0A9016AE38CEEB1
:1055C00091E10E941F5F882351F088E08093ED11E4
:1055D0008CEE91E10E94F45EE3E6F8E020C00E94C8
:1055E000FE5E807C803C19F483E08093F0110E9481
:1055F000FE5E0E94FE5E0E94FE5E8CEE91E10E94C5
:10560000F45E1092EE1181E091DA811145C021C063
:105610009091C00095FFFCCF8093C6003196849195
:105620008111F6CFE6E5F8E08491882341F090916E
:10563000C00095FFFCCF8093C6003196F5CF8091D6
:10564000C00085FFFCCF8AE08093C60086EC94E022
:1056500073C080E06BDA81111FC0EFE4F8E0849141
:10566000882341F09091C00095FFFCCF8093C60045
:105670003196F5CFECE3F8E08491882341F09091E6
:10568000C00095FFFCCF8093C6003196F5CF809186
:10569000C00085FFFCCF26C061EF71E188E790E193
:1056A0000E948E5D811122C0EFE4F8E0849188238E
:1056B00041F09091C00095FFFCCF8093C6003196D9
:1056C000F5CFECE2F8E08491882341F09091C0009E
:1056D00095FFFCCF8093C6003196F5CF8091C00036
:1056E00085FFFCCF8AE08093C60028C081E08093CC
:1056F0004010E3E6F8E08491882341F09091C000E7
:1057000095FFFCCF8093C6003196F5CFE1E2F8E03B
:105710008491882341F09091C00095FFFCCF809345
:10572000C6003196F5CF8091C00085FFFCCF8AE09E
:105730008093C60085EE94E00E9411658BE1E8E756
:10574000F0E1A9E9B0E101900D928A95E1F780912D
:10575000761090917710909398108093971084E72B
:1057600090E19093941080939310DF91CF911F91CB
:10577000FF90EF90DF90CF9008958F929F92AF921D
:10578000BF92CF92DF92EF92FF920F931F93CF932E
:10579000DF93CDB7DEB7CC52D1400FB6F894DEBF61
:1057A0000FBECDBF60E080E2FDD7999AA19A2FEF9E
:1057B00037EA81E6215030408040E1F700C0000028
:1057C000E0918A0FF0918B0F12E01083E091860F29
:1057D000F091870F1082E091880FF091890F8FEC84
:1057E00080831092920FE0918E0FF0918F0F86E0E0
:1057F0008083E0918C0FF0918D0F80818061808398
:10580000E0918C0FF0918D0F808188608083E09112
:105810008C0FF0918D0F808180688083E0918C0FD8
:10582000F0918D0F80818F7D80839FEFA1EEB4E09A
:105830009150A040B040E1F700C0000088E694E03D
:105840000E941165EFEFF9EF20E0E150F0402040B9
:10585000E1F700C000008EEF94E00E9411653FEF79
:1058600089EF90E0315080409040E1F700C00000A7
:105870008EE095E00E941165AFEFB9EFE0E0A15036
:10588000B040E040E1F700C000001093C00010926B
:10589000C50080E18093C4008091C1008061809345
:1058A000C1008091C10088608093C1008091C100D7
:1058B00080688093C100EDE5F9E08491882341F090
:1058C0009091C00095FFFCCF8093C6003196F5CF34
:1058D0008091C00085FFFCCF8AE08093C60086E7F8
:1058E00098E0FC012491222341F03091C00035FF63
:1058F000FCCF2093C6003196F5CF24B720FF14C00B
:10590000E5E5F9E03491332341F04091C00045FFD3
:10591000FCCF3093C6003196F5CF3091C00035FFF3
:10592000FCCF3AE03093C60021FF14C0E5E4F9E073
:105930003491332341F04091C00045FFFCCF3093B8
:10594000C6003196F5CF3091C00035FFFCCF3AE06C
:105950003093C60022FF14C0E4E3F9E0349133230E
:1059600041F04091C00045FFFCCF3093C600319616
:10597000F5CF3091C00035FFFCCF3AE03093C60040
:1059800023FF14C0E4E2F9E03491332341F0409165
:10599000C00045FFFCCF3093C6003196F5CF309163
:1059A000C00035FFFCCF3AE03093C60025FF14C09D
:1059B000E4E1F9E02491222341F03091C00035FF69
:1059C000FCCF2093C6003196F5CF2091C00025FF73
:1059D000FCCF2AE02093C60014BEECE0F9E024914D
:1059E000222341F03091C00035FFFCCF2093C60048
:1059F0003196F5CFE5E0F9E02491222341F0309192
:105A0000C00035FFFCCF2093C6003196F5CF209122
:105A1000C00025FFFCCF2AE02093C600FC012491A2
:105A2000E6E7F8E0222349F03091C00035FFFCCFD3
:105A30002093C60031962491F5CFE5EFF8E024914C
:105A4000222341F03091C00035FFFCCF2093C600E7
:105A50003196F5CFE0EEF8E02491222341F0309129
:105A6000C00035FFFCCF2093C6003196F5CFE4EDA2
:105A7000F8E02491222341F03091C00035FFFCCFA3
:105A80002093C6003196F5CFEDECF8E02491222367
:105A900041F03091C00035FFFCCF2093C600319615
:105AA000F5CF2091C00025FFFCCF2AE02093C6004F
:105AB000E2ECF8E02491222341F03091C00035FF60
:105AC000FCCF2093C6003196F5CFE6EBF8E02491A9
:105AD000222341F03091C00035FFFCCF2093C60057
:105AE0003196F5CF2091C00025FFFCCF2AE020930E
:105AF000C600FC018491E6E7F8E0882349F0909124
:105B0000C00095FFFCCF8093C60031968491F5CFFD
:105B1000E7EAF8E08491882341F09091C00095FF76
:105B2000FCCF8093C6003196F5CF80914A199091B1
:105B30004B198E010F5F1F4F009721F4C80180554C
:105B4000994104C09801281B390BC9019A838983A4
:105B500069817A81072E000C880B990BBCD9E0E98A
:105B6000F8E08491882341F09091C00095FFFCCF2C
:105B70008093C6003196F5CF60ED74E080E090E050
:105B8000AAD98091C00085FFFCCF8AE08093C6002F
:105B90001092CB0B1092CC0B1092CD0B1092CE0B1F
:105BA0000E94484120E030E048E452E460911B103C
:105BB00070911C1080911D1090911E100E9478C44D
:105BC00020E030E040E05FE30E94FEB86093040212
:105BD000709305028093060290930702E5E1F5E0D9
:105BE0008191882339F09091C00095FFFCCF80937C
:105BF000C600F6CF8091C00085FFFCCF8AE080937D
:105C0000C6000BD7609343127093441280934512E1
:105C1000909346120E94F36484E295E00E9411651D
:105C2000CE01815E9E4F0E94DA76CE01815E9E4F4C
:105C3000A5DA882309F46BC068E374E0C8010E9408
:105C40000F906CE275E0CE0193950E940F90A80131
:105C5000BE017395CE01815E9E4F0E944B8DCE0199
:105C600093950E947C8FC8010E947C8F68E374E04A
:105C7000C8010E940F9067E374E0CE0193950E94E3
:105C80000F90A801BE017395CE01815E9E4F0E94C8
:105C90004B8DCE0193950E947C8FC8010E947C8F12
:105CA000BE01615E7E4FC8010E94079025E030E092
:105CB0004CE2B801CE0193950E94FA71C8010E948E
:105CC0007C8F8EE295E00E940F65C050DF4F888187
:105CD0009981C050D1400E940F6588EB94E00E94EA
:105CE0000F650E9403653FEF89EF90E031508040DF
:105CF0009040E1F700C0000080E495E00E9411654B
:105D0000CE0193950E947C8FFF24F39407C0AFE3EC
:105D1000BCE91197F1F700C00000F12C7ED680900D
:105D2000431290904412A0904512B0904612DC01AC
:105D3000CB0188199909AA09BB09893E9340A1059D
:105D4000B10578F00E94F36484E295E00E94116549
:105D500064D66093431270934412809345129093DB
:105D60004612CE01815E9E4F0E947C8FFF2009F477
:105D700057CF0E944D6EE0903602F090370210929D
:105D8000BD181092BE181092BF181092C018209122
:105D90003E0230913F02409140025091410260E04A
:105DA00070E08FE793E40E9467C56093B518709325
:105DB000B6188093B7189093B818F0923902E09211
:105DC00038021092C1181092C2181092C318109283
:105DD000C4186093B9187093BA188093BB18909345
:105DE000BC18259A249A8091010180628093010158
:105DF0008091010180648093010187ED80937A0096
:105E000010927E0010927D0080917D0080688093CA
:105E10007D0080917D00806280937D0080917D0077
:105E2000806480937D0080E888BD80916E008460EE
:105E300080936E006AEF70E080E090E0B6D581E07C
:105E400090E09093B2188093B11860E080910A02BC
:105E500090910B020E94E2A320E030E040E85FE373
:105E60000E94A1BE87FF0AC080910A0290910B0296
:105E7000409790930B0280930A02E7CF80912C0BFE
:105E800090912D0B909337028093360260E08091C1
:105E90006112909162120E94E2A36B017C018091D9
:105EA0002C0B90912D0BBC01990F880B990B0E9424
:105EB000A7BE9B01AC01C701B6010E94C4C618165B
:105EC00054F4809161129091621240969093621204
:105ED00080936112DBCF81E090E09093B4188093BF
:105EE000B31861E080910C0290910D020E94E2A330
:105EF00020E030E040E85FE30E94A1BE87FF0AC0D7
:105F000080910C0290910D02409790930D02809326
:105F10000C02E7CF80912A0B90912B0B90933902C2
:105F20008093380261E080916312909164120E9424
:105F3000E2A36B017C0180912A0B90912B0BBC0199
:105F4000990F880B990B0E94A7BE9B01AC01C7015A
:105F5000B6010E94C4C6181654F480916312909141
:105F6000641240969093641280936312DBCF809109
:105F70000802909109020E94CD3920E030E040E80B
:105F80005FE30E94A1BE87FF0AC080910802909142
:105F9000090240979093090280930802E8CF80910C
:105FA0005F12909160120E94CD396B017C0180914B
:105FB000AF189091B018BC01990F880B990B0E94F3
:105FC000A7BE9B01AC01C701B6010E94C4C618164A
:105FD00054F480915F1290916012409690936012F9
:105FE00080935F12DCCF1092AD181092AC1880E154
:105FF000E8E2F3E1DF011D928A95E9F71092D512EC
:106000001092D6121092D7121092D8121092D91262
:106010001092DA121092DB121092DC121092DD1242
:106020001092DE121092DF121092E0121092E11222
:106030001092E2121092E3121092E4121092E51202
:106040001092E6121092E7121092E812819A3B9A8F
:10605000879A80910A01826080930A0180910701EA
:10606000806180930701849A0E9A579A5F9A3F9AAB
:10607000479A829A8A9A80910701816080930701EA
:106080009FB7F894809108018160809308019FBFB9
:10609000809107018460809307019FB7F8948091F5
:1060A00008018460809308019FBF859A8D9A0A9A9F
:1060B000129A6D98759A809104018D7F80930401E6
:1060C0009FB7F894809105018260809305019FBF7E
:1060D00053985B9A6C98749A809A88985F9A479ABA
:1060E000399A41985F9A479A869A8E988A9A8091AF
:1060F0000A01886080930A019FB7F89480910B0190
:10610000877F80930B019FBF8091070188608093F8
:1061100007019FB7F89480910801877F8093080159
:106120009FBF9FB7F8948091080181608093080118
:106130009FBF9FB7F8948091080184608093080105
:106140009FBF839A8B988D9A0C9A1498129A80917B
:1061500081008F7E80938100809181008860809390
:106160008100809180008D7F8093800080918000ED
:106170008E7F80938000809180008F738093800059
:10618000809180008F7C8093800080918100887F47
:1061900082608093810080E090E4909389008093F6
:1061A0008800109285001092840080916F008260B8
:1061B00080936F0080E00E94BCA878948CE495E006
:1061C0000E94116560E081E3EDD29FB7F894809161
:1061D0000B01816080930B019FBF4AD9BFEFE3EDB4
:1061E000F0E3B150E040F040E1F700C0000088E685
:1061F00094E00E9411658CE695E00E941165809103
:10620000401068E374E0811106C0CE01815E9E4FAC
:106210000E940F90C6C0CE018B5D9E4F0E940F90D2
:10622000CE0193950E94A272C12CDD24D394CC0E92
:10623000DD1E24E0C20ED11C21E046E755E068E7F0
:1062400070E1C6010E946863882309F446C0CB5EF2
:10625000DE4FE880F980C551D1403FEFE31AF30AE1
:106260008AE090E0C55DDE4F99838883CB52D140B0
:106270009E01255D3E4FA701B801C6010E945664EC
:1062800068E374E0CE01815E9E4F0E940F9068012A
:10629000C601801B910B8E159F055CF4D6016D9194
:1062A0006D016623A9F3CE01815E9E4F0E94068F89
:1062B000EFCFCE01815E9E4F0E94BE28882341F021
:1062C000BE01615E7E4FCE018B5D9E4F0E942E8F80
:1062D000CE01815E9E4F0E947C8F80E091E08C0F0A
:1062E0009D1F04960E94E15DCE018B5D9E4F0E9432
:1062F000BE28811103C0EEE7F5E026C08CE291E0F4
:10630000C15EDE4F99838883CF51D14044E0B8010C
:10631000CE01815E9E4F0E94393E89819A81AB8178
:10632000BC8181159840A105B105C0F468E374E013
:10633000CE018B5D9E4F0E94198F10C09091C000BE
:1063400095FFFCCF8093C60081918111F7CF80919A
:10635000C00085FFFCCF8AE08093C600C15EDE4F9F
:1063600019821882CF51D140CF5DDE4F1982188239
:10637000C152D140CD5DDE4F19821882C352D14047
:10638000BE016B5D7E4FCE01815E9E4F0E94438FAA
:10639000CE0193950E949A72CE018B5D9E4F0E9412
:1063A0007C8FBE01615E7E4FC8010E94079021E094
:1063B00030E04CE7B801CE0193950E94FA71BE011E
:1063C0007395CE01815E9E4F0E94438FCE019395BF
:1063D0000E947C8FC8010E947C8FCE01815E9E4FFF
:1063E0000E94BE28882309F467C068E374E0C801EE
:1063F0000E940F908091FE129091FF12892B81F4E0
:1064000062E975E0CE0193950E940F90BE01615E36
:106410007E4FCE0193950E94F58E65EB75E00FC01F
:1064200067EB75E0CE0193950E940F90BE01615E0F
:106430007E4FCE0193950E94F58E6CEC75E00E9424
:10644000DE8EBC01C8010E942E8FCE0193950E9462
:106450007C8F62E574E0CE0193950E940F90B801A5
:10646000CE0193950E94F58E68EB74E00E94DE8E5B
:10647000BC01C8010E942E8FCE0193950E947C8F93
:10648000E980FA8080E794E00E9411658FEC95E046
:106490000E94116587EE95E00E94116584E096E008
:1064A0000E941165C7010E9411658AEB94E00E9469
:1064B0001165C8010E947C8F81E080935F02109279
:1064C000A4181092A5181092A6181092A718A19AB5
:1064D000CE01815E9E4F0E947C8FC45DDE4F0FB661
:1064E000F894DEBF0FBECDBFDF91CF911F910F910A
:1064F000FF90EF90DF90CF90BF90AF909F908F90E4
:1065000008958091411290914212009731F00197C5
:10651000909342128093411206C081E090E09093E4
:10652000401280933F1280913F1290914012892B2C
:1065300061F01092401210923F120E94FA768CE4A1
:106540009DE19093421280934112089580E090E083
:10655000892B41F080E090E0892B21F00E9400001F
:10656000811121C080E090E0892B41F080E090E033
:10657000892B21F00E940000811118C080E090E07A
:10658000892B21F00E94608C811113C080E090E083
:10659000892BA1F080E090E0892B81F00E9400001F
:1065A00081110AC008950E940000DCCF0E94000003
:1065B000E5CF0E940000EACF0C940000089590E01F
:1065C000FC013197E231F10508F04EC08827EE5802
:1065D000FF4F8F4F0C944BC8809180008F7703C082
:1065E000809180008F7D809380000895809180004D
:1065F000877FF9CF84B58F7702C084B58F7D84BD46
:1066000008958091B0008F7703C08091B0008F7D96
:106610008093B0000895809190008F7707C080919B
:1066200090008F7D03C080919000877F80939000C1
:1066300008958091A0008F7707C08091A0008F7D82
:1066400003C08091A000877F8093A000089580916F
:1066500020018F7707C0809120018F7D03C080913A
:106660002001877F8093200108953FB7F89480919F
:10667000951290919612A0919712B091981226B50A
:10668000A89B05C02F3F19F00196A11DB11D3FBF6A
:10669000BA2FA92F982F8827820F911DA11DB11DF8
:1066A000BC01CD0142E0660F771F881F991F4A95F4
:1066B000D1F70895FC01848DDF01A80FB11DA35A05
:1066C000BF4F2C91848D90E001968F739927848F12
:1066D000A689B7892C93A089B1898C9180648C9309
:1066E000938D848D981306C00288F389E02D8081F4
:1066F0008F7D80830895CF93DF93282F30E0F901B9
:10670000EA5FF34F8491F901E054F44FD491F90119
:10671000E658F44FC491CC2389F0811150DFEC2F5F
:10672000F0E0EE0FFF1FE05AF44FA591B491EC9109
:10673000ED2381E090E021F480E002C080E090E071
:10674000DF91CF9108951F93CF93DF93282F30E0EF
:10675000F901EA5FF34F8491F901E054F44FD491C9
:10676000F901E658F44FC491CC23C1F0162F8111E2
:1067700026DFEC2FF0E0EE0FFF1FEA5BF44FA59150
:10678000B4918FB7F894111105C09C91ED2FE0954D
:10679000E92302C0EC91ED2BEC938FBFDF91CF91F9
:1067A0001F910895CF93DF9390E0FC01E054F44FE4
:1067B0002491FC01E658F44F8491882361F190E024
:1067C000880F991FFC01E45DF44FC591D491FC0141
:1067D000EA5BF44FA591B491611109C09FB7F89499
:1067E0008881209582238883EC912E230BC0623010
:1067F00061F49FB7F8943881822F80958323888332
:10680000EC912E2B2C939FBF06C08FB7F894E88194
:106810002E2B28838FBFDF91CF9108951F93CF93A5
:10682000DF93182FEB0161E0BDDF209711F460E0EA
:1068300004C0CF3FD10531F461E0812FDF91CF91CA
:106840001F9181CFE12FF0E0EA5FF34FE4914E2FEB
:1068500050E0FA013197E231F10508F09DC0882738
:10686000EC57FF4F8F4F0C944BC884B5806884BDA4
:10687000C7BD97C084B5806284BDC8BD92C08091F9
:106880008000806880938000D0938900C093880046
:1068900088C080918000806280938000D0938B00BC
:1068A000C0938A007EC080918000886080938000C1
:1068B000D0938D00C0938C0074C08091B00080682C
:1068C0008093B000C093B3006CC08091B000806230
:1068D0008093B000C093B40064C080919000806841
:1068E00080939000D0939900C09398005AC08091F3
:1068F0009000806280939000D0939B00C0939A0098
:1069000050C080919000886080939000D0939D004B
:10691000C0939C0046C08091A00080688093A00036
:106920008091A0008F7B8093A000D093A900C0939A
:10693000A80037C08091A00080628093A000D0930F
:10694000AB00C093AA002DC08091A0008860809306
:10695000A000D093AD00C093AC0023C08091200173
:10696000806880932001D0932901C093280119C029
:1069700080912001806280932001D0932B01C093ED
:106980002A010FC080912001886080932001D0935C
:106990002D01C0932C0105C0C038D1050CF04CCF9F
:1069A00046CFDF91CF911F9108958F929F92AF9222
:1069B000BF92CF92DF92EF92FF926B017C0155DE86
:1069C0004B015C01C114D104E104F104E9F04DDE96
:1069D000DC01CB0188199909AA09BB09883E9340BB
:1069E000A105B10578F321E0C21AD108E108F10848
:1069F00088EE880E83E0981EA11CB11CC114D1043E
:106A0000E104F10421F7DECFFF90EF90DF90CF900B
:106A1000BF90AF909F908F9008952FB7F89460919A
:106A200091127091921280919312909194122FBFB3
:106A300008951F920F920FB60F9211242F933F9338
:106A40008F939F93AF93BF938091911290919212E5
:106A5000A0919312B09194123091901223E0230FE1
:106A60002D3720F40196A11DB11D05C026E8230F86
:106A70000296A11DB11D20939012809391129093C4
:106A80009212A0939312B0939412809195129091C8
:106A90009612A0919712B09198120196A11DB11D66
:106AA0008093951290939612A0939712B093981298
:106AB000BF91AF919F918F913F912F910F900FBEFA
:106AC0000F901F901895E9EFF2E111821082138266
:106AD00012821092DF0B1092DE0BA7E6B2E11C923D
:106AE0002D9811961C922C981092DF0B1092DE0BB1
:106AF000109266129FB7F894E2E0F1E080818F7DFA
:106B000080839FBF08950F931F93CF93DF93CDB7DB
:106B1000DEB72D970FB6F894DEBF0FBECDBF8D87C1
:106B2000D2DF909107138D85911176C0E5E2FBE0ED
:106B30009491992341F02091C00025FFFCCF9093C0
:106B4000C6003196F5CF082F10E0682F70E080E086
:106B500090E00E946B278091C00085FFFCCF8AE007
:106B60008093C600E4E8FAE08491882341F0909194
:106B7000C00095FFFCCF8093C6003196F5CF809181
:106B8000C00085FFFCCF8AE08093C6008091FE1292
:106B90009091FF12B8016F5F7F4F4AE0892BA1F4FB
:106BA000CE0107960E94DC8F65E276E0CE01019669
:106BB0000E940F90BE01695F7F4FCE0101960E9437
:106BC000F58E61E876E013C0CE0107960E94DC8F57
:106BD0006DE276E0CE0101960E940F90BE01695FE2
:106BE0007F4FCE0101960E94F58E69E976E00E9402
:106BF000DE8EBC0189E392E10E942E8FCE010196C8
:106C00000E947C8FCE0107960E947C8F8AE090E0E4
:106C10009093DC0B8093DB0B0E94379D2D960FB673
:106C2000F894DEBF0FBECDBFDF91CF911F910F91C2
:106C300008950F931F93CF93DF93CDB7DEB72D97B2
:106C40000FB6F894DEBF0FBECDBF8D873CDF9091AD
:106C500007138D85911176C0E5E2FBE094919923AD
:106C600041F02091C00025FFFCCF9093C6003196E3
:106C7000F5CF082F10E0682F70E080E090E00E94D0
:106C80006B278091C00085FFFCCF8AE08093C6000F
:106C9000E7E5FAE08491882341F09091C00095FFE8
:106CA000FCCF8093C6003196F5CF8091C00085FF60
:106CB000FCCF8AE08093C6008091FE129091FF1273
:106CC000B8016F5F7F4F4AE0892BA1F4CE01079690
:106CD0000E94DC8F65E276E0CE0101960E940F9063
:106CE000BE01695F7F4FCE0101960E94F58E65E37C
:106CF00076E013C0CE0107960E94DC8F6DE276E04D
:106D0000CE0101960E940F90BE01695F7F4FCE01B8
:106D100001960E94F58E68E676E00E94DE8EBC0148
:106D200089E392E10E942E8FCE0101960E947C8F12
:106D3000CE0107960E947C8F89E090E09093DC0B57
:106D40008093DB0B0E94379D2D960FB6F894DEBF23
:106D50000FBECDBFDF91CF911F910F9108951F926C
:106D60000F920FB60F9211240BB60F922F933F93F1
:106D70004F935F936F937F938F939F93AF93BF9343
:106D8000EF93FF930E94EC9E811187C280910E02C7
:106D900081111AC08091671280938F1281112D9AF0
:106DA0008091681280938E1281112C9A80916612C4
:106DB00080938D12882341F09FB7F894809102014F
:106DC0008062809302019FBF90918F1280910E028A
:106DD000891708F02D9890918E1280910E028917D4
:106DE00008F02C9890918D1280910E02891740F036
:106DF0009FB7F894809102018F7D809302019FBF1D
:106E000080910E028F5F8F7780930E0280918C129B
:106E100090E08830910508F087C0FC018827EA5689
:106E2000FF4F8F4F0C944BC888E080937B0087E422
:106E300080937C0080917A00806480937A0081E066
:106E400019C020917800309179008091881290913A
:106E50008912A0918A12B0918B12820F931FA11DEB
:106E6000B11D8093881290938912A0938A12B093D7
:106E70008B1282E080938C1257C088E080937B0055
:106E800086E480937C0080917A00806480937A000D
:106E900083E0F0CF209178003091790080918412C6
:106EA00090918512A0918612B0918712820F931F44
:106EB000A11DB11D8093841290938512A093861218
:106EC000B093871284E0D6CF88E080937B0085E47E
:106ED00080937C0080917A00806480937A0085E0C2
:106EE000C9CF2091780030917900809180129091E3
:106EF0008112A0918212B0918312820F931FA11D63
:106F0000B11D8093801290938112A0938212B0934E
:106F1000831286E0AFCF87E0ADCF10928C128091C4
:106F20007F128F5F80937F1280917F12803108F4EF
:106F3000B4C180916512811118C08091881290911E
:106F4000891290937C1280937B1280918012909191
:106F5000811290937E1280937D1280918412909181
:106F6000851290937A128093791281E08093651252
:106F700010927F12109288121092891210928A1227
:106F800010928B1210928012109281121092821223
:106F9000109283121092751210927612109277123C
:106FA000109278121092841210928512109286120A
:106FB0001092871220917B1230917C128091611285
:106FC000909162128217930754F0809173129091FE
:106FD00074120196909374128093731209C0809179
:106FE00071129091721201969093721280937112A5
:106FF0008091711290917212049744F01092741261
:107000001092731210927212109271128091731278
:1070100090917412049734F01092741210927312BB
:1070200080E007DE20917B1230917C1280910A0271
:1070300090910B02281739074CF08091F91290912A
:10704000FA121816190614F480E05DDD20917D1205
:1070500030917E128091631290916412821793078F
:1070600054F080916F12909170120196909370126B
:1070700080936F1209C080916D1290916E120196EB
:1070800090936E1280936D1280916D1290916E129A
:10709000049744F01092701210926F1210926E12B8
:1070A00010926D1280916F1290917012049734F0CB
:1070B0001092701210926F1281E0BBDD20917D1250
:1070C00030917E1280910C0290910D0228173907A1
:1070D0004CF08091FB129091FC121816190614F4D2
:1070E00081E011DD2091791230917A1280915F1246
:1070F000909160128217930754F080916B129091D7
:107100006C12019690936C1280936B1209C080915F
:10711000691290916A12019690936A128093691293
:107120008091691290916A12049744F010926C1247
:1071300010926B1210926A121092691280916B1267
:1071400090916C1204970CF44CC010926C12109237
:107150006B121092DF0B1092DE0B9FB7F8948091A8
:1071600002018F7D809302019FBF809107138111DF
:1071700036C0E5E2FBE08491882341F09091C000A5
:1071800095FFFCCF8093C6003196F5CFE1EBFAE096
:107190008491882341F09091C00095FFFCCF8093AB
:1071A000C6003196F5CF8091C00085FFFCCF8AE004
:1071B0008093C6008091FE129091FF12892B19F4E2
:1071C00062E376E002C064E676E089E392E10E9441
:1071D000198F8BE090E09093DC0B8093DB0B0E9487
:1071E000379D2091791230917A1280910802909106
:1071F0000902281739070CF450C08091DE0B9091DA
:10720000DF0B181619060CF048C01092DF0B109215
:10721000DE0B9FB7F894809102018F7D809302016D
:107220009FBF80910713811136C0E5E2FBE0849196
:10723000882341F09091C00095FFFCCF8093C60059
:107240003196F5CFEBEEFAE08491882341F09091EE
:10725000C00095FFFCCF8093C6003196F5CF80919A
:10726000C00085FFFCCF8AE08093C6008091FE12AB
:107270009091FF12892B19F46EE776E002C065E960
:1072800076E089E392E10E94198F8CE090E0909380
:10729000DC0B8093DB0B0E94379DFF91EF91BF9138
:1072A000AF919F918F917F916F915F914F913F919E
:1072B0002F910F900BBE0F900FBE0F901F9018953F
:1072C000CF92DF92EF92FF921092DD0BC090571297
:1072D000D0905812E0905912F0905A128091F91201
:1072E0009091FA12BC01990F880B990B0E94A7BECE
:1072F00020E030E040EA51E40E9478C49B01AC01F8
:10730000C701B6010E94A1BE87FF11C0C701B60127
:107310000E94D8C570935412609353127EDB609321
:107320004B1270934C1280934D1290934E12C0905A
:107330005B12D0905C12E0905D12F0905E12809132
:10734000FB129091FC12BC01990F880B990B0E94C3
:10735000A7BE20E030E040EA51E40E9478C49B01DF
:10736000AC01C701B6010E94A1BE87FF11C0C701D1
:10737000B6010E94D8C570935612609355124DDB2A
:1073800060934F1270935012809351129093521247
:10739000FF90EF90DF90CF9008952F923F924F9201
:1073A0005F926F927F928F929F92AF92BF92CF9295
:1073B000DF92EF92FF920F931F93CF93DF93EC0135
:1073C00047E659E081E090E0FA0125913491C21737
:1073D000D3070CF05DC09C0121503109220F331FEF
:1073E000220F331FD901AB59B64FFD01659174913E
:1073F0002D59364FF901A590B490FC01EE0FFF1FF7
:10740000EE0FFF1FEB59F64FE590F490FD01C5908C
:10741000D490FA0105911491F90125903490072E2A
:10742000000C880B990B0E94A7BE2B013C01CA19C6
:10743000DB09BE01DD0F880B990B0E94A7BE4B0133
:107440005C01B7016C197D09072E000C880B990BA4
:107450000E94A7BE9B01AC01C501B4010E94FEB809
:107460006B017C01B80162197309072E000C880BAF
:10747000990B0E94A7BE9B01AC01C701B6010E94F7
:1074800067C59B01AC01C301B2010E9479C411C060
:1074900001964C5F5F4F8D33910509F095CFE5E57F
:1074A000FAE065917491072E000C880B990B0E94ED
:1074B000A7BEDF91CF911F910F91FF90EF90DF90CA
:1074C000CF90BF90AF909F908F907F906F905F9084
:1074D0004F903F902F9008950F931F93CF93DF937A
:1074E0000BE712E160E0F801808191810E94E2A344
:1074F000C7E5D2E1688379838A839B8361E0F801E1
:10750000828193810E94E2A36C837D838E839F831B
:107510008091791290917A1240DF609347127093B4
:1075200048128093491290934A128FB7F8941092A0
:1075300065128FBFDF91CF911F910F910895CF9367
:10754000DF93C1EADEE0FE018491882341F090914F
:10755000C00095FFFCCF8093C6003196F5CFE5E5DE
:10756000FEE08491882341F09091C00095FFFCCF0C
:107570008093C6003196F5CF8091C00085FFFCCF87
:107580008AE08093C600FE018491E1EAFEE0882350
:1075900049F09091C00095FFFCCF8093C6003196D2
:1075A0008491F5CF409138135091391360913A137B
:1075B00070913B138DE49EE00E94737240913C13E6
:1075C00050913D1360913E1370913F138AE49EE009
:1075D0000E94737240914013509141136091421385
:1075E0007091431387E49EE00E94737240914413AC
:1075F00050914513609146137091471384E49EE0C7
:107600000E9473728091C00085FFFCCF8AE0809356
:10761000C600FE018491E1EAFEE0882349F09091E2
:10762000C00095FFFCCF8093C60031968491F5CFC2
:10763000EAE2FEE08491882341F09091C00095FF3A
:10764000FCCF8093C6003196F5CF8091C00085FFB6
:10765000FCCF8AE08093C600FE018491E1EAFEE05F
:10766000882349F09091C00095FFFCCF8093C6001D
:1076700031968491F5CF4091B5125091B612609138
:10768000B7127091B81281E29EE00E94737240912D
:10769000B9125091BA126091BB127091BC128EE176
:1076A0009EE00E9473724091BD125091BE12609193
:1076B000BF127091C0128BE19EE00E9473724091E4
:1076C000C1125091C2126091C3127091C41288E12C
:1076D0009EE00E9473728091C00085FFFCCF8AE01B
:1076E0008093C600FE018491E1EAFEE0882349F020
:1076F0009091C00095FFFCCF8093C6003196849195
:10770000F5CFEAEFFDE08491882341F09091C0002D
:1077100095FFFCCF8093C6003196F5CF8091C000D5
:1077200085FFFCCF8AE08093C600FE018491E1EAE8
:10773000FEE0882349F09091C00095FFFCCF809334
:10774000C60031968491F5CF40915C1350915D1342
:1077500060915E1370915F1381EF9DE00E946272F1
:1077600040916013509161136091621370916313A3
:107770008EEE9DE00E9462724091641350916513F9
:1077800060916613709167138BEE9DE00E946272A8
:10779000409168135091691360916A1370916B1353
:1077A00088EE9DE00E9462728091C00085FFFCCF50
:1077B0008AE08093C600FE018491E1EAFEE088231E
:1077C00049F09091C00095FFFCCF8093C6003196A0
:1077D0008491F5CFE3EBFDE08491882341F0909113
:1077E000C00095FFFCCF8093C6003196F5CF809105
:1077F000C00085FFFCCF8AE08093C600FE01849123
:10780000E1EAFEE0882349F09091C00095FFFCCFAB
:107810008093C60031968491F5CF4091AD1250917E
:10782000AE126091AF127091B0128AEA9DE00E9490
:1078300073724091B1125091B2126091B312709173
:10784000B41287EA9DE00E9473728091C00085FFA8
:10785000FCCF8AE08093C600FE018491E1EAFEE05D
:10786000882349F09091C00095FFFCCF8093C6001B
:1078700031968491F5CFE4EFFCE08491882341F0C8
:107880009091C00095FFFCCF8093C6003196F5CF54
:107890008091C00085FFFCCF8AE08093C600FE0186
:1078A0008491E1EAFEE0882349F09091C00095FFC1
:1078B000FCCF8093C60031968491F5CF4091C912D8
:1078C0005091CA126091CB127091CC128BEE9CE059
:1078D0000E9473724091CD125091CE126091CF12DE
:1078E0007091D01288EE9CE00E9473724091C51294
:1078F0005091C6126091C7127091C81285EE9CE03B
:107900000E9462724091A9125091AA126091AB122A
:107910007091AC1282EE9CE00E9473724091A512AD
:107920005091A6126091A7127091A8128FED9CE061
:107930000E9473724091A1125091A2126091A31201
:107940007091A4128CED9CE00E9473728091C00033
:1079500085FFFCCF8AE08093C600FE018491E1EAB6
:10796000FEE0882349F09091C00095FFFCCF809302
:10797000C60031968491F5CFEAECFCE0849188232F
:1079800041F09091C00095FFFCCF8093C6003196E6
:10799000F5CF8091C00085FFFCCF8AE08093C600C0
:1079A000FE018491E1EAFEE0882349F09091C00055
:1079B00095FFFCCF8093C60031968491F5CF40911E
:1079C0000D1950910E1960910F197091101981ECD9
:1079D0009CE00E94737240911119509112196091AC
:1079E0001319709114198EEB9CE00E9473724091F0
:1079F00015195091161960911719709118198BEB80
:107A00009CE00E9473728091C00085FFFCCF8AE0E9
:107A10008093C600FE018491E1EAFEE0882349F0EC
:107A20009091C00095FFFCCF8093C6003196849161
:107A3000F5CFEDEAFCE08491882341F09091C000FD
:107A400095FFFCCF8093C6003196F5CF8091C000A2
:107A500085FFFCCF8AE08093C600FE018491E1EAB5
:107A6000FEE0882349F09091C00095FFFCCF809301
:107A7000C60031968491F5CF409142025091430265
:107A8000609144027091450283EA9CE00E94737207
:107A90002DEB37E346E05EE360913E0270913F02DA
:107AA00080914002909141020E9467C5AB01BC01E8
:107AB00080EA9CE00E9473722DEB37E346E05EE3C0
:107AC00060913A0270913B0280913C0290913D029C
:107AD0000E94FEB8AB01BC018DE99CE00E9473726C
:107AE0008091C00085FFFCCF8AE08093C600FE0134
:107AF0008491E1EAFEE0882349F09091C00095FF6F
:107B0000FCCF8093C60031968491F5CFEAE8FCE083
:107B10008491882341F09091C00095FFFCCF809321
:107B2000C6003196F5CF8091C00085FFFCCF8AE07A
:107B30008093C60040911B1050911C1060911D1045
:107B400070911E1086E89CE00E9473728091C000C4
:107B500085FFFCCF8AE08093C600FE018491E1EAB4
:107B6000FEE0882349F09091C00095FFFCCF809300
:107B7000C60031968491F5CFE5E7FCE08491882337
:107B800041F09091C00095FFFCCF8093C6003196E4
:107B9000F5CF8091C00085FFFCCF8AE08093C600BE
:107BA00040913710509138106091391070913A100F
:107BB00081E79CE00E9473728091C00085FFFCCF3A
:107BC0008AE08093C600FE01C491E1EAFEE0CC2386
:107BD00049F08091C00085FFFCCFC093C60031966C
:107BE000C491F5CFE0E6FCE08491882341F09091C8
:107BF000C00095FFFCCF8093C6003196F5CF8091F1
:107C0000C00085FFFCCF8AE08093C6004091300B16
:107C10005091310B6091320B7091330B8CE59CE0ED
:107C20000E9473728091C00085FFFCCF8AE0809330
:107C3000C600E4EAF6E08191882339F09091C00013
:107C400095FFFCCF8093C600F6CF6091360B709104
:107C5000370B072E000C880B990B0E946B27809125
:107C6000C00085FFFCCF8AE08093C600DF91CF91F2
:107C70000895EF92FF921F93CF93DF937C01C62F5D
:107C8000D72F142F160FF701808191810E9418C4FD
:107C90008993F701808191810196918380831C13E0
:107CA000F2CFDF91CF911F91FF90EF900895EF9267
:107CB000FF921F93CF93DF937C01C62FD72F142FF2
:107CC000160F6991F701808191810E9420C4F7010C
:107CD000808191810196918380831C13F2CFDF9183
:107CE000CF911F91FF90EF9008950F931F93CF9323
:107CF000DF93CDB7DEB72C970FB6F894DEBF0FBE7B
:107D0000CDBF80E390E3A0E3B0E08D839E83AF839B
:107D1000B88704E610E01C870B8744E0BE016B5F68
:107D20007F4FCE010B96C3DF40E168E373E1CE01E4
:107D30000B96BDDF40E165EB72E1CE010B96B7DF3C
:107D400040E16CE573E1CE010B96B1DF44E06DEAF2
:107D500072E1CE010B96ABDF44E061EB72E1CE0144
:107D60000B96A5DF44E069EC72E1CE010B969FDF34
:107D700044E06DEC72E1CE010B9699DF44E065ECD6
:107D800072E1CE010B9693DF44E069EA72E1CE0125
:107D90000B968DDF44E065EA72E1CE010B9687DF3A
:107DA00044E061EA72E1CE010B9681DF4CE06DE0C8
:107DB00079E1CE010B967BDF42E062E27BE0CE010F
:107DC0000B9675DF42E060E27BE0CE010B966FDF41
:107DD00042E06EE17BE0CE010B9669DF42E068E2B3
:107DE0007BE0CE010B9663DF42E066E27BE0CE01F2
:107DF0000B965DDF42E064E27BE0CE010B9657DF3D
:107E000044E062E472E0CE010B9651DF44E06EE3A1
:107E100072E0CE010B964BDF44E06AE372E0CE01E4
:107E20000B9645DF44E06BE170E1CE010B963FDF3E
:107E300044E067E370E1CE010B9639DF44E060E394
:107E40007BE0CE010B9633DF42E066E978E1CE01BC
:107E50000B962DDF42E064E978E1CE010B9627DF37
:107E600042E06EEF72E1CE010B9621DF42E066E365
:107E70007BE0CE010B961BDF42E06EE27BE0CE01A1
:107E80000B9615DF42E06CE27BE0CE010B960FDF34
:107E900042E06AE27BE0CE010B9609DF42E06FEA46
:107EA00078E1CE010B9603DF42E064E073E1CE019E
:107EB0000B96FDDE80E290E09A87898742E0BE0162
:107EC000675F7F4FCE010B96F2DE86E590E3A8E375
:107ED000B0E089839A83AB83BC831C870B8744E023
:107EE000BE016F5F7F4FCE010B96E1DEE1EAFEE05F
:107EF0008491882341F09091C00095FFFCCF80933E
:107F0000C6003196F5CFECE4FCE08491882341F083
:107F10009091C00095FFFCCF8093C6003196F5CFBD
:107F20008091C00085FFFCCF8AE08093C6002C962C
:107F30000FB6F894DEBF0FBECDBFDF91CF911F917A
:107F40000F910895AF92BF92CF92DF92EF92FF927E
:107F50000F931F93CF93DF93CDB7DEB7E0970FB6A4
:107F6000F894DEBF0FBECDBF80E1EBE8F2E0DE01AA
:107F7000919601900D928A95E1F780E1EBE9F2E0AC
:107F8000DE01519601900D928A95E1F780E1EBEACE
:107F9000F2E0DE01119601900D928A95E1F7DE0183
:107FA000919668E373E1AE014F5E5F4F25EB32E1DE
:107FB000CE0101965C018CE593E18E010F5C1F4FB1
:107FC000CD90DD90ED90FD90FB01C192D192E192B8
:107FD000F192BF01FA01C190D190E190F190AF010F
:107FE000F901C192D192E192F1929F01F501C19004
:107FF000D190E190F1905F01FC01C192D192E192A8
:10800000F192CF01A017B107D9F60E94016E80E06E
:1080100090E0AAEFB3E48093AD129093AE12A093D8
:10802000AF12B093B0128093B1129093B212A0939A
:10803000B312B093B4121092C9121092CA121092D5
:10804000CB121092CC1280E29EE4A0E0B0E08093CC
:10805000C5129093C612A093C712B093C812109283
:10806000CD121092CE121092CF121092D01280E048
:1080700090E0A0EAB1E48093A9129093AA12A09391
:10808000AB12B093AC128DEC9CECACECBEE38093E5
:10809000A5129093A612A093A712B093A81280E005
:1080A00090E0A0EAB0E48093A1129093A212A09372
:1080B000A312B093A41210921519109216191092CF
:1080C0001719109218191092111910921219109272
:1080D00013191092141910920D1910920E19109272
:1080E0000F191092101988EC90E09093230B809355
:1080F000220B1092210B1092200B10921F0B10924A
:108100001E0B8CED90E09093290B8093280B83E25B
:1081100090E09093270B8093260B1092250B1092E2
:10812000240B8AE097EDA1EBB1E480934202909397
:108130004302A0934402B09345028EE297E1A8E582
:10814000BEE380933E0290933F02A0934002B0931F
:1081500041028EE395ECA2E1B4E480933A0290935D
:108160003B02A0933C02B0933D020E94A3A880E092
:1081700090E0A0E8BFE38093000290930102A093F7
:108180000202B093030280E090E0A1EBB3E480939D
:108190001B1090931C10A0931D10B0931E1081E033
:1081A0008093460280E991E090932D0B80932C0BF5
:1081B00090932B0B80932A0B88E790E09093B01854
:1081C0008093AF1880E090E0A0E9B0E4809337108E
:1081D00090933810A0933910B0933A1080E090E05B
:1081E000A0E0B0E48093300B9093310BA093320B5E
:1081F000B093330B80E590E0909397188093961896
:1082000090939518809394181092FF121092FE127A
:1082100081E090E0909305138093041310922F0B4C
:1082200010922E0B1092370B1092360BE1EAFEE003
:108230008491882341F09091C00095FFFCCF8093FA
:10824000C6003196F5CFEFE7FEE08491882341F038
:108250009091C00095FFFCCF8093C6003196F5CF7A
:108260008091C00085FFFCCF8AE08093C600E09635
:108270000FB6F894DEBF0FBECDBFDF91CF911F9137
:108280000F91FF90EF90DF90CF90BF90AF902DCDEA
:10829000CF93DF93CDB7DEB72C970FB6F894DEBF40
:1082A0000FBECDBF84E690E09C878B8786E590E388
:1082B000A8E3B0E089839A83AB83BC8344E0BE012A
:1082C0006B5F7F4FCE010B96D4DC43E050E0BE01E4
:1082D0006B5F7F4FCE0101960E949AC9892B09F0EE
:1082E0001DC140E168E373E1CE010B96C2DC40E1C1
:1082F00065EB72E1CE010B96BCDC40E16CE573E10D
:10830000CE010B96B6DC0E94016E44E06DEA72E18C
:10831000CE010B96AEDC44E061EB72E1CE010B9630
:10832000A8DC44E069EC72E1CE010B96A2DC44E0EB
:108330006DEC72E1CE010B969CDC44E065EC72E1E1
:10834000CE010B9696DC44E069EA72E1CE010B9611
:1083500090DC44E065EA72E1CE010B968ADC44E0F1
:1083600061EA72E1CE010B9684DC4CE06DE079E1CC
:10837000CE010B967EDC42E062E27BE0CE010B9602
:1083800078DC42E060E27BE0CE010B9672DC42E0FA
:108390006EE17BE0CE010B966CDC42E068E27BE0B4
:1083A000CE010B9666DC42E066E27BE0CE010B96E6
:1083B00060DC42E064E27BE0CE010B965ADC44E0F4
:1083C00062E472E0CE010B9654DC44E06EE372E0AE
:1083D000CE010B964EDC44E06AE372E0CE010B96D0
:1083E00048DC44E06BE170E1CE010B9642DC44E0F6
:1083F00067E370E1CE010B963CDC44E060E37BE098
:10840000CE010B9636DC42E066E978E1CE010B96B0
:1084100030DC42E064E978E1CE010B962ADC42E0F0
:108420006EEF72E1CE010B9624DC42E066E37BE066
:10843000CE010B961EDC42E06EE27BE0CE010B9695
:1084400018DC81E08093460242E06CE27BE0CE01E2
:108450000B960FDC42E06AE27BE0CE010B9609DC72
:1084600042E06FEA78E1CE010B9603DC80912C0BA1
:1084700090912D0B8A3F910534F48AEF90E0909310
:108480002D0B80932C0B80912A0B90912B0B8A3F04
:10849000910534F48AEF90E090932B0B80932A0B94
:1084A0008091AF189091B0188035910534F480E533
:1084B00090E09093B0188093AF1842E064E073E1CD
:1084C000CE010B96D6DB42E0BE01675F7F4FCE0147
:1084D0000B96CFDB0E94A3A8E1EAFEE084918823FB
:1084E00041F09091C00095FFFCCF8093C60031967B
:1084F000F5CFE5E6FEE08491882341F09091C0003D
:1085000095FFFCCF8093C6003196F5CF8091C000D7
:1085100085FFFCCF8AE08093C60001C013DD0FD831
:108520002C960FB6F894DEBF0FBECDBFDF91CF9172
:1085300008958F929F92AF92BF92CF92DF92EF9267
:10854000FF920F931F93CF93DF93CDB7DEB764975E
:108550000FB6F894DEBF0FBECDBF6B837C838D83D7
:108560009E8358874F833A8729871C870B87CD8640
:10857000DE86EF86F88A898A9A8AAB8ABC8A8CE280
:1085800091E09A83898344E0BE016D5F7F4FCE0105
:1085900001968DDB8B819C81AD81BE8181309840BD
:1085A000A105B10518F142E0BE01695F7F4FCE0120
:1085B00001967DDB42E0BE01675F7F4FCE010196F1
:1085C00076DB42E0BE01655F7F4FCE0101966FDB37
:1085D00044E0BE01635F7F4FCE01019668DB44E05B
:1085E000BE016F5E7F4FCE01019661DB64960FB6D0
:1085F000F894DEBF0FBECDBFDF91CF911F910F91D9
:10860000FF90EF90DF90CF90BF90AF909F908F90B2
:1086100008952F923F924F925F926F927F928F9226
:108620009F92AF92BF92CF92DF92EF92FF920F9301
:108630001F93CF93DF93CDB7DEB768970FB6F8944B
:10864000DEBF0FBECDBF1C012A013B01480159010D
:10865000DC01D8966D917D918D919C91DB970E9464
:10866000A5BE6B017C01A30192010E94FEB80E948D
:1086700050C50E94DEC56D877E878F87988BA501C8
:108680009401C701B6010E94FEB80E9450C50E9425
:10869000DEC5698B7A8B8B8B9C8B2D853E854F85B8
:1086A0005889283731054105510540F488E790E0A5
:1086B000A0E0B0E08D879E87AF87B88B29893A8983
:1086C0004B895C89283731054105510540F488E71D
:1086D00090E0A0E0B0E0898B9A8BAB8BBC8B9101D2
:1086E0002C5B3F4FD9018D919D910D90BC91A02D98
:1086F0008D839E83AF83B887BC01CD010E94A7BE46
:1087000069837A838B839C83F10164AD75AD86ADFB
:1087100097AD0E94A5BE69877A878B879C8720E0EA
:1087200030E0A90169817A818B819C810E94A1BE80
:10873000882339F1A7019601C701B6010E94FEB84E
:108740004B015C0129853A854B855C85CA01B901DD
:108750000E94FEB89B01AC01C501B4010E9478C41F
:108760004B015C0129813A814B815C81CA01B901CD
:108770000E9479C49B01AC01C501B4010E9467C588
:1087800003C060E070E0CB010E9450C50E94D8C5D4
:108790002B013C016D817E818F819885909580951C
:1087A000709561957F4F8F4F9F4F0E94A7BE4B01E1
:1087B0005C01F101E05CFF4F6081718182819381F6
:1087C0000E94A5BE6D837E838F83988720E030E072
:1087D000A901C501B4010E94A1BE882349F12D81E0
:1087E0003E814F815885CA01B9010E94FEB86D8B48
:1087F0007E8B8F8B988FA7019601C701B6010E94CF
:10880000FEB89B01AC016D897E898F89988D0E948D
:1088100078C46B017C01A5019401C501B4010E94DB
:1088200079C49B01AC01C701B6010E9467C503C0B2
:1088300060E070E0CB010E940DC6D10150968D9092
:108840009D90AD90BC90539775016401C418D508F4
:10885000E608F7080E94D8C5C61AD70AE80AF90A36
:10886000F7FE6BC020E030E0A90169817A818B813D
:108870009C810E94A1BE882309F447C029813A81C6
:108880004B815C81CA01B9010E9479C46B017C01F2
:10889000C501B4010E94A5BE9B01AC01C701B60190
:1088A0000E94FEB86B017C0129853A854B855C8569
:1088B000CA01B9010E94FEB89B01AC01C701B60113
:1088C0000E9478C46B017C012D813E814F815885C7
:1088D000CA01B9010E94FEB89B01AC01C701B601F3
:1088E0000E9479C46B017C0120E030E040E850E454
:1088F00069817A818B819C810E94FEB89B01AC01C9
:10890000C701B6010E9467C503C060E070E0CB01FB
:108910000E9450C50E94D8C52B013C0197FF03C09F
:10892000412C512C3201481459046A047B0410F084
:1089300024013501C12CD12C76018FB7F894F101B7
:10894000E45BFF4F9081911121C0F101448A558A67
:10895000668A778AC40CD51CE61CF71CD101C08E30
:10896000D18EE28EF38E2D853E854F85588924AFBA
:1089700035AF46AF57AFA05CBF4F29893A894B89C5
:108980005C892D933D934D935C9313978FBF6896AD
:108990000FB6F894DEBF0FBECDBFDF91CF911F9110
:1089A0000F91FF90EF90DF90CF90BF90AF909F908E
:1089B0008F907F906F905F904F903F902F90089591
:1089C000AF92BF92CF92DF92EF92FF920F931F93DD
:1089D000CF93DF935B016A01790108E313E1F801AA
:1089E0002081318142815381FC01608171818281CA
:1089F00093810E94FEB80E9471C7C8E2D3E16883E8
:108A000079838A839B83F80124813581468157814C
:108A1000F50160817181828193810E94FEB80E947C
:108A200071C76C837D838E839F83F8012085318598
:108A300042855385F60160817181828193810E9414
:108A4000FEB80E9471C7688779878A879B87F8017B
:108A50002485358546855785F7016081718182813E
:108A600093810E94FEB80E9471C76C877D878E87B4
:108A70009F878FB7F894488159816A817B81E8E0AC
:108A8000F3E140835183628373834C815D816E8106
:108A90007F814483558366837783488559856A85BA
:108AA0007B8540875187628773874C855D856E859E
:108AB0007F8544875587668777878FBF1092E51239
:108AC0001092E6121092E7121092E812E5EDF2E130
:108AD00010821182128213821482158216821782EA
:108AE00010861186128613861486158616861786BA
:108AF000DF91CF911F910F91FF90EF90DF90CF907A
:108B0000BF90AF9008952F923F924F925F926F92D5
:108B10007F928F929F92AF92BF92CF92DF92EF920D
:108B2000FF920F931F93CF93DF93CDB7DEB7C1575B
:108B3000D1090FB6F894DEBF0FBECDBF2C013B01AB
:108B40005A0149013E2C2F2CDEAACDAA80915F024A
:108B50008111F8C080913E1090913F10019709F06B
:108B6000F1C0DA01CD90DD90ED90FC904090A4181A
:108B70005090A5186090A6187090A718A3019201B4
:108B8000C701B6010E94A1BE4091F5125091F612A4
:108B90006091F7127091F8128823A9F08091F11278
:108BA0009091F212A091F312B091F4128A019B01FC
:108BB000081B190B2A0B3B0BD901C80181309440CB
:108BC000A105B10530F4411551056105710509F0A4
:108BD0009EC0452B462B472B49F4809170109091F5
:108BE0007110A0917210B091731029C02091ED12F4
:108BF0003091EE124091EF125091F012C701B60180
:108C00000E94A1BE882309F473C020E030E0A901CE
:108C1000C701B6010E94A1BE882309F469C0A3015F
:108C20009201C701B6010E94C4C61816A4F480912F
:108C3000E9129091EA12A091EB12B091EC12019717
:108C4000A109B1098093F5129093F612A093F7123F
:108C5000B093F8121BC0A3019201C701B6010E9494
:108C6000A1BE87FF13C08091E9129091EA12A091F2
:108C7000EB12B091EC120196A11DB11D8093F1127F
:108C80009093F212A093F312B093F4128091F11228
:108C90009091F212A091F312B091F4124091F5125A
:108CA0005091F6126091F7127091F812481B590B0F
:108CB0006A0B7B0B7695679557954795480F591F1B
:108CC0006A1F7B1F4093E9125093EA126093EB12E4
:108CD0007093EC1210925F0240936C1050936D10E1
:108CE00060936E1070936F1083E192E10E94F85CC4
:108CF000F50180819181A281B3818093ED129093DF
:108D0000EE12A093EF12B093F0120C94435281E054
:108D100080935F02198A1A8A1B8A1C8A19821A8216
:108D20001B821C829401A501BE016F5E7F4FCE01A4
:108D3000019646DE8FEF90E09093A9188093A818D3
:108D40000C9443521092F1121092F2121092F312FC
:108D50001092F4121092E9121092EA121092EB1291
:108D60001092EC121092F5121092F6121092F71265
:108D70001092F8121092ED121092EE121092EF1261
:108D80001092F0128091AD188F5F68968FAF689740
:108D9000803119F468961FAE68976896FFAD6897A2
:108DA000EF2EFF0FFF088091AC1890E08E159F0505
:108DB00039F40E9403A50E94AC9D0E948132F3CF3A
:108DC000209138133091391340913A1350913B134D
:108DD000D2016D917D918D919C910E94FEB80E946F
:108DE00071C76C966CAF7DAF8EAF9FAF6C972091C3
:108DF0003C1330913D1340913E1350913F13F301CA
:108E000060817181828193810E94FEB80E9471C746
:108E1000A0966CAF7DAF8EAF9FAFA097209140130F
:108E2000309141134091421350914313D5016D91FC
:108E30007D918D919C910E94FEB80E9471C7A4966D
:108E40006CAF7DAF8EAF9FAFA4972091441330914C
:108E500045134091461350914713F401608171818D
:108E6000828193810E94FEB80E9471C72F966CAFD9
:108E70007DAF8EAF9FAF2F978091341390913513B4
:108E8000A0913613B09137132F962CAD3DAD4EAD5A
:108E90005FAD2F97281739074A075B0709F4ADC064
:108EA000E091061334E0E39FF0011124E95AFD4EEE
:108EB0002091D1123091D2124091D3125091D412FC
:108EC00060817181828193810E94A1BE87FF2FC042
:108ED0002F964CAD5DAD6EAD7FAD2F9740933413A3
:108EE000509335136093361370933713EBE0FFE024
:108EF0008491882341F09091C00095FFFCCF80932E
:108F0000C6003196F5CFE1EFFEE08491882341F071
:108F10009091C00095FFFCCF8093C6003196F5CFAD
:108F20008091C00085FFFCCF8AE08093C6008091CD
:108F3000341390913513A0913613B09137132F96B7
:108F40002CAD3DAD4EAD5FAD2F97281B390B4A0BB5
:108F50005B0BCA01B90157FF07C0909580957095CA
:108F600061957F4F8F4F9F4F0E94A7BE6B017C0181
:108F700020E030EC48E254E46091441370914513D2
:108F800080914613909147130E94FEB89B01AC015B
:108F9000C701B6010E94C4C618167CF52F964CADC9
:108FA0005DAD6EAD7FAD2F97409334135093351365
:108FB0006093361370933713EBE0FFE084918823BE
:108FC00041F09091C00095FFFCCF8093C600319690
:108FD000F5CFE3EDFEE08491882341F09091C0004D
:108FE00095FFFCCF8093C6003196F5CF8091C000ED
:108FF00085FFFCCF8AE08093C600E091AD186E2F0C
:1090000070E07CA36BA37DE4E79FF0011124E8549A
:10901000FC4E10828091281390912913A0912A135D
:10902000B0912B138DA39EA3AFA3B8A76C96CCAC25
:10903000DDACEEACFFAC6C97C81AD90AEA0AFB0AA1
:10904000F7FE08C0F094E094D094C094C11CD11CE9
:10905000E11CF11C8DE4ABA1BCA18A9FF0018B9FA8
:10906000F00D1124E459FC4EC082D182E282F382D9
:1090700020912C1330912D1340912E1350912F13CA
:1090800029A73AA74BA75CA7A0968CAC9DACAEAC29
:10909000BFACA097821A930AA40AB50AB7FE08C00B
:1090A000B094A09490948094811C911CA11CB11C3C
:1090B0008DE44BA15CA1849FF001859FF00D1124EC
:1090C000E459FC4E84829582A682B7826091301367
:1090D0007091311380913213909133136DA77EA755
:1090E0008FA798ABA4964CAC5DAC6EAC7FACA4974C
:1090F000461A570A680A790A77FE08C07094609485
:1091000050944094411C511C611C711C8DE4ABA116
:10911000BCA18A9FF0018B9FF00D1124E459FC4EF5
:1091200040865186628673862091341330913513C0
:10913000409136135091371329AB3AAB4BAB5CAB34
:109140002F962CAD3DAD4EAD5FAD2F9769A97AA995
:109150008BA99CA9261B370B480B590B57FF07C03F
:1091600050954095309521953F4F4F4F5F4FA091BF
:109170000F02B09110020E9453C824E630E040E094
:1091800050E00E942FC88DE4ABA1BCA18A9FF001E2
:109190008B9FF00D1124E459FC4E248735874687B8
:1091A0005787C901DA0184159505A605B70514F49A
:1091B000D301C201B701A60188159905AA05BB050F
:1091C00044F0C816D906EA06FB0654F4AC01BD010A
:1091D00007C0C814D904EA04FB0414F4B501A401BF
:1091E0008DE42BA13CA1829FF001839FF00D1124FF
:1091F000E459FC4E408B518B628B738B463051058A
:109200006105710514F40C944352DF01A85BBF4F54
:109210004091A8185091A918052E000C660B770BE9
:109220004D935D936D937C9313976C964CAD5DADB0
:109230006EAD7FAD6C978DA19EA1AFA1B8A548176B
:1092400059076A077B0714F010A202C081E080A3CF
:10925000A0962CAD3DAD4EAD5FADA09769A57AA5AA
:109260008BA59CA526173707480759076CF48DE492
:10927000ABA1BCA18A9FF0018B9FF00D1124E45992
:10928000FC4E80A1826080A3A4962CAD3DAD4EAD76
:109290005FADA4976DA57EA58FA598A92617370762
:1092A000480759076CF48DE4ABA1BCA18A9FF0017B
:1092B0008B9FF00D1124E459FC4E80A1846080A3A3
:1092C0002F962CAD3DAD4EAD5FAD2F9769A97AA914
:1092D0008BA99CA926173707480759076CF48DE41A
:1092E000ABA1BCA18A9FF0018B9FF00D1124E45922
:1092F000FC4E80A1886080A3EDA9FEA980819DE439
:109300002BA13CA1929FF001939FF00D1124E459F1
:10931000FC4E81A3CD28CE28CF2811F05F98479826
:109320008DE44BA15CA1849FF001859FF00D112479
:10933000E459FC4E84819581A681B781892B8A2BC3
:109340008B2B09F08A988DE46BA17CA1869FF0019C
:10935000879FF00D1124E459FC4E80859185A285EC
:10936000B385892B8A2B8B2B81F09FB7F894809142
:1093700008018E7F809308019FBF9FB7F89480916A
:1093800008018B7F809308019FBF8DE4ABA1BCA136
:109390008A9FF0018B9FF00D1124E459FC4E8485C7
:1093A0009585A685B785892B8A2B8B2B11F08D98F7
:1093B00012988DE42BA13CA1829FF001839FF00DB8
:1093C0001124E459FC4E448555856685778523969E
:1093D0004CAF5DAF6EAF7FAF2397452B462B472B2E
:1093E00049F4C090CD12D090CE12E090CF12F09000
:1093F000D01208C0C090C912D090CA12E090CB120F
:10940000F090CC129601A701632D722DC8010E9425
:10941000A1BE87FF03C03C2C2D2C8701809128130F
:1094200090912913A0912A13B0912B136C962CAD17
:109430003DAD4EAD5FAD6C97281B390B4A0B5B0BF6
:10944000CA01B9010E94A7BE209138133091391387
:1094500040913A1350913B130E9467C56DA37EA3C0
:109460008FA398A7698B7A8B8B8B9C8B80912C1305
:1094700090912D13A0912E13B0912F13A0962CAD87
:109480003DAD4EAD5FADA097281B390B4A0B5B0B72
:10949000CA01B9010E94A7BE20913C1330913D132F
:1094A00040913E1350913F130E9467C54B015C01F0
:1094B0006D8B7E8B8F8B988F8091301390913113B1
:1094C000A0913213B0913313A4962CAD3DAD4EADA7
:1094D0005FADA497281B390B4A0B5B0BCA01B9017E
:1094E0000E94A7BE20914013309141134091421336
:1094F000509143130E9467C56B017C01698F7A8F7D
:109500008B8F9C8F8091341390913513A0913613DB
:10951000B09137132F962CAD3DAD4EAD5FAD2F976B
:10952000281B390B4A0B5B0BCA01B9010E94A7BE6D
:1095300020914413309145134091461350914713A5
:109540000E9467C52B013C0160910F0270911002CF
:10955000072E000C880B990B0E94A7BE9B01AC0143
:10956000C301B2010E94FEB820E030E048EC52E4B2
:109570000E9467C56D8F7E8F8F8F98A32DE44BA1BE
:109580005CA1249FF001259FF00D1124E459FC4EAD
:1095900020813181428153812FAB38AF49AF5AAF1F
:1095A0002630310541055105E4F44480558066803C
:1095B000778036E0431651046104710494F44084CA
:1095C00051846284738446E044165104610471043A
:1095D00044F4DC01CB01BF7786A797A7A0ABB1AB62
:1095E0002EC06DA17EA18FA198A50E94FBB82B0172
:1095F0003C01C501B4010E94FBB89B01AC01C30151
:10960000B2010E9479C44B015C01C701B6010E94FE
:10961000FBB89B01AC01C501B4010E9479C40E9452
:10962000AFC72DE4ABA1BCA12A9FF0012B9FF00D89
:109630001124E459FC4E66A777A780AB91AB8DE46B
:109640002BA13CA1829FF001839FF00D1124E459CE
:10965000FC4E46A557A560A971A94BAF5CAF6DAF95
:109660007EAF9A01AB0160E070E080E89FE30E946A
:1096700067C59B01AC01632D722DC8010E94FEB825
:109680006B017C018091AD182091AC1890E0821B99
:1096900091098C010F701127A6961FAF0EAFA697E8
:1096A000A701960160E074E284E799E40E9467C52F
:1096B0000E9471C74B015C01023011050CF441C0DE
:1096C0002801110F66087708C301B2010E94A7BEE6
:1096D00020E030E040E051E40E94A1BE87FF31C0AD
:1096E0008091C5129091C612A091C712B091C81274
:1096F00088169906AA06BB0620F588199909AA09B1
:10970000BB09BC01CD01660F771F881F991FA301FC
:1097100092010E943DC4CA01B9010E94A5BE0E94E7
:1097200071C7680D791D8A1D9B1D0E94A5BE9B01F6
:10973000AC0160E074E284E799E40E9467C56B01C4
:109740007C01A70196016BAD7CAD8DAD9EAD0E94F5
:10975000FEB827966CAF7DAF8EAF9FAF27978DE495
:109760002BA13CA1829F8001839F100D11240459DD
:109770001C4E27964CAD5DAD6EAD7FAD2797D801E1
:1097800092964D935D936D937C93959750966D91C2
:109790007D918D919C9153970E94A5BE6DA37EA350
:1097A0008FA398A7A70196010E94FEB80E9450C5FA
:1097B0000E94DEC52B966CAF7DAF8EAF9FAF2B970F
:1097C000F80160AF71AF82AF93AF8E010F5E1F4F94
:1097D0001EAB0DAB005111091AAB09AB05EB12E141
:1097E00065961FAF0EAF65978E010F5D1F4F1AA3D1
:1097F00009A309A91AA961961FAF0EAF6197212C81
:10980000312C10E819A70FE30DA7ADA9BEA96D91E2
:109810007D918D919D91BEABADABA70196010E944C
:10982000FEB86196EEADFFAD619761937193819340
:1098300091936196FFAFEEAF61974B015C01E894A5
:10984000B7F86596AEADBFAD65974D905D906D90E4
:109850007D906596BFAFAEAF6597A3019201C5013C
:10986000B4010E94C4C61816A4F4A5019401C30152
:10987000B2010E9467C55B018C019B01AC01B10183
:1098800089A59DA50E94A1BE87FD03C0150109A75A
:109890001DA70DA91EA929A13AA10217130709F0B6
:1098A000B4CF20E030E040E85FE3B10189A59DA599
:1098B0000E94A1BE87FF49C08E010F5E1F4F91011C
:1098C00049A55DA5A9A9BAA96D917D918D919C919C
:1098D0000E94FEB8E9A9FAA96193719381939193CB
:1098E000FAABE9ABE017F10751F78DE42BA13CA1EE
:1098F000829F8001839F100D112404591C4E9101F9
:1099000049A55DA527966CAD7DAD8EAD9FAD279722
:109910000E94FEB8D80192966D937D938D939C938F
:1099200095972B966CAD7DAD8EAD9FAD2B970E941C
:10993000A5BE910149A55DA50E94FEB80E94DEC5A5
:10994000F80160AF71AF82AF93AF2BAD3CAD4DADC1
:109950005EAD6DA17EA18FA198A50E9467C56B0128
:109960007C010FA918AD29AD3AAD012B022B032BB9
:10997000A1F58DE42BA13CA1829F8001839F100D56
:10998000112404591C4EF80184819581A681B78168
:10999000892B8A2B8B2B09F580859185A285B38530
:1099A000892B8A2B8B2BC9F42091B1123091B212E2
:1099B0004091B3125091B412C701B6010E94FEB893
:1099C0000E9450C50C5B1F4F0E94DEC5D8016D93ED
:1099D0007D938D939C93139721C12091AD1230916B
:1099E000AE124091AF125091B012C701B6010E9461
:1099F000FEB80E9450C50E94DEC52DE4EBA1FCA17B
:109A00002E9F80012F9F100D112400551C4ED80150
:109A10006D937D938D939C93139780904C139090AE
:109A20004D13A0904E13B0904F130E94A5BE2B0172
:109A30003C016FA978AD89AD9AAD0E94A7BE9B018C
:109A4000AC01C301B2010E94FEB82DA13EA14FA1FD
:109A500058A50E9467C52B013C01C501B4010E94B5
:109A6000A5BE9B01AC01C301B2010E94C4C6181679
:109A70002CF4F80180829182A282B38280905013EC
:109A800090905113A0905213B09053132DE40BA15A
:109A90001CA1209FC001219F900D11249C012459DD
:109AA0003C4E190189010C5B1F4FD8016D917D91CE
:109AB0008D919C910E94A5BE2B013C01F101648116
:109AC0007581868197810E94A7BE9B01AC01C3016D
:109AD000B2010E94FEB82DA13EA14FA158A50E943F
:109AE00067C52B013C01C501B4010E94A5BE9B01C5
:109AF000AC01C301B2010E94C4C6181634F4D801E7
:109B00008D929D92AD92BC92139780905813909035
:109B10005913A0905A13B0905B138DE4EBA1FCA1F4
:109B20008E9F80018F9F100D112400551C4ED8016F
:109B30006D917D918D919C910E94A5BE2B013C0160
:109B400023966CAD7DAD8EAD9FAD23970E94A7BED1
:109B50009B01AC01C301B2010E94FEB82DA13EA140
:109B60004FA158A50E9467C52B013C01C501B40156
:109B70000E94A5BE9B01AC01C301B2010E94C4C6F4
:109B800018162CF4F80180829182A282B382809010
:109B9000541390905513A0905613B09057132DE482
:109BA0000BA11CA1209FC001219F900D11249C019D
:109BB00024593C4E190189010C5B1F4FD8016D914E
:109BC0007D918D919C910E94A5BE2B013C01F101DC
:109BD00060857185828593850E94A7BE9B01AC013B
:109BE000C301B2010E94FEB82DA13EA14FA158A50C
:109BF0000E9467C52B013C01C501B4010E94A5BEAE
:109C00009B01AC01C301B2010E94C4C6181634F412
:109C1000D8018D929D92AD92BC9213978DE4EBA1E9
:109C2000FCA18E9F80018F9F100D112404591C4EA2
:109C3000F801EC5BFF4F60817181828193810E940A
:109C4000A5BE4B015C01A70196010E9467C5AA96BB
:109C50006CAF7DAF8EAF9FAFAA97D801D2966D93B0
:109C60007D938D939C93D5972DEB37E346E051E49C
:109C7000C501B4010E94FEB80E94D8C5F801648FE6
:109C8000758F868F978FC090A912D090AA12E090FE
:109C9000AB12F090AC1220E030E040E05FE3C7018F
:109CA000B6010E94FEB86DA379A78DA799AB09856F
:109CB0001A852B853C85AE960CAF1DAF2EAF3FAFFE
:109CC000AE972091A5123091A6124091A712509103
:109CD000A81263962CAF3DAF4EAF5FAF639720E005
:109CE00030E040E05FE363966CAD7DAD8EAD9FAD3F
:109CF00063970E94FEB85B018C01AE966CAD7DADA2
:109D00008EAD9FADAE979F779501A8010E94C4C606
:109D1000181674F49501A8016DA179A58DA599A9CE
:109D20000E94A1BE87FD04C0ADA2B9A60DA719ABC4
:109D30004D855E856F857889E2964CAF5DAF6EAFDD
:109D40007FAFE2976091A1127091A2128091A3124D
:109D50009091A41267966CAF7DAF8EAF9FAF67975F
:109D600020E030E040E05FE30E94FEB85B018C0140
:109D7000E2966CAD7DAD8EAD9FADE2979F7795017C
:109D8000A8010E94C4C6181674F49501A8016DA11B
:109D900079A58DA599A90E94A1BE87FD04C0ADA299
:109DA000B9A60DA719AB8DE40BA11CA1809FF001F2
:109DB000819FF00D1124E459FC4E12A11BAF03A1A9
:109DC0000FAF14A124961FAF249705A128960FAFBB
:109DD00028972BAD3FAD412F502F6DA179A58DA5B3
:109DE00099A90E94A1BE87FD0CC01BAD1DA30FAD9C
:109DF00009A724961FAD24971DA728960FAD289775
:109E000009ABA6960EAD1FADA697023011050CF456
:109E1000EBC01091E5121DAB2090E6120091E71205
:109E20000FAB3090E81227E137EB41ED58E3612F9B
:109E3000722D802F932D0E94C4C618160CF0D4C02A
:109E40002091D5123091D6124091D7125091D8124C
:109E500069817A818B819C810E9478C42B013C01AD
:109E60002091D9123091DA124091DB125091DC121C
:109E70006D817E818F8198850E9478C44B015C0141
:109E8000A3019201C301B2010E94FEB82B013C0163
:109E9000A5019401C501B4010E94FEB89B01AC016B
:109EA000C301B2010E9479C40E94AFC74B015C019B
:109EB000A70196010E94C4C618164CF4A50194018E
:109EC000C701B6010E9467C57B018C0104C0E12C6B
:109ED000F12C00E81FE32091DD123091DE12409159
:109EE000DF125091E012AE966CAD7DAD8EAD9FADA0
:109EF000AE970E9478C44B015C01E894B7F8639672
:109F00002CAD3DAD4EAD5FAD6397C501B4010E9470
:109F1000C4C61816B4F4A501940163966CAD7DAD6A
:109F20008EAD9FAD63970E9467C55B016C019B017D
:109F3000AC01B701C8010E94A1BE87FD02C0750136
:109F400086012091E1123091E2124091E31250918A
:109F5000E412E2966CAD7DAD8EAD9FADE2970E94AE
:109F600078C44B015C01E894B7F867962CAD3DAD21
:109F70004EAD5FAD6797C501B4010E94C4C6181607
:109F8000B4F4A501940167966CAD7DAD8EAD9FAD27
:109F900067970E9467C55B016C019B01AC01B7012B
:109FA000C8010E94A1BE87FD02C07501860197010C
:109FB000A8016BAD7FAD24968FAD249728969FADF9
:109FC00028970E94FEB87B018C019B01AC016DA912
:109FD000722D8FA9932D0E94A1BE87FD0BC0EDAA03
:109FE0002F2C0FAB312E06C01DA11DAB29A40DA532
:109FF0000FAB39A88DE42BA13CA1829F8001839FE8
:10A00000100D112404591C4E8DA9922DAFA9B32D0A
:10A01000F80182A793A7A4A7B5A7AA966CAD7DADBA
:10A020008EAD9FADAA9790589B01AC010E9479C458
:10A03000D8019E962D913D914D915C91D1970E94B2
:10A04000FEB89B01AC016BE077ED83E29BE30E94DD
:10A0500078C40E94AFC7B62EC72E7C01262F372F9B
:10A06000AC016DA9722D8FA9932D0E94A1BE87FD11
:10A0700005C0DB2C2C2CAE2C3F2C02C0DDA8AFA8D9
:10A080008DE4EBA1FCA18E9F80018F9F100D112408
:10A0900004591C4E8D2D922DAA2DB32DF80186A3A7
:10A0A00097A3A0A7B1A72B2D3C2DA7016BAD7FAD2A
:10A0B00024968FAD249728969FAD28970E94A1BE25
:10A0C00018162CF081E0D801D7968C9302C0F801C5
:10A0D00017AA2DE40BA11CA1209FC001219F900D68
:10A0E00011249C0124593C4E790181E0D901D69676
:10A0F0008C9380E1FE013196A5EDB2E101900D92C5
:10A100008A95E1F78BAD9FAD2496AFAD2497289645
:10A11000BFAD28978093E5129093E612A093E712C3
:10A12000B093E8129C01AD016DA179A58DA599A907
:10A130000E9467C52B013C012BAD3FAD24964FAD6E
:10A14000249728965FAD28976D2D722D8A2D932D1B
:10A150000E9467C5AB01BC0193018201C7010E9447
:10A1600009436896BFAD6897B093AD186C960CAD77
:10A170001DAD2EAD3FAD6C9700932813109329139E
:10A1800020932A1330932B13A0962CAD3DAD4EADEA
:10A190005FADA09720932C1330932D1340932E1373
:10A1A00050932F13A4964CAD5DAD6EAD7FADA497CB
:10A1B00040933013509331136093321370933313E1
:10A1C0002F966CAD7DAD8EAD9FAD2F976093341300
:10A1D0007093351380933613909337138091AD1895
:10A1E0008FB7F8946090AC188FBF8091AD1890E055
:10A1F000861991098F70992704974CF41091AC1827
:10A20000F12C00E080E090E05DE4E52EA0C08091BC
:10A21000AD1883508F70F82EA12CB12C00E010E007
:10A220004DE4442E55245394F61441F38F2DF11030
:10A2300001C080E1FF24FA94F80E4F9CC001112464
:10A24000DC01A459BC4EBCA3ABA30115110509F454
:10A2500069C0A114B10409F465C0F80172A4C3A4D3
:10A26000D4A4E5A4272D3C2D4D2D5E2D66A177A10C
:10A2700080A591A50E94A1BE882309F453C0D801EE
:10A28000D7968C91811144C0F50186A097A0A0A417
:10A29000B1A4A5019401672D7C2D8D2D9E2D0E94CA
:10A2A000C4C61816ACF5A5019401C501B4010E94FD
:10A2B000FEB84B015C01F80182A993A9A4A9B5A934
:10A2C000BC01CD0190589B01AC010E9479C4D8011A
:10A2D0009E962D913D914D915C91D1970E94FEB833
:10A2E0009B01AC01C501B4010E9478C40E94AFC7B4
:10A2F0001B015C019B01AC01672D7C2D8D2D9E2DDA
:10A300000E94A1BE87FD04C0722CC32CDA2CEB2C5A
:10A31000872D9C2DAD2DBE2DF80186A397A3A0A758
:10A32000B1A756AA58010BA11CA17ECFE19E9001B6
:10A330001124F901E459FC4E6F01009769F41F5F85
:10A34000103109F410E08F2D902FFC2C0D2D209151
:10A35000AD181213EBCF0AC0DC01D7962C91211156
:10A36000EECF6F2D702F0E94926DE9CF009741F0D4
:10A37000FC0127A9211104C06F2D702F0E94926D3E
:10A38000D090AC18E12CF12C3DE4C32E4D2D0D2CBA
:10A39000000C550B8091AD1890E04817590709F44F
:10A3A00047C0C49EC001C59E900D11248C01045964
:10A3B0001C4E1801E114F104A1F1D701D6968C913D
:10A3C000811104C0F80186A9882359F1D70192961A
:10A3D0004D905D906D907C909597C49EF001C59EC8
:10A3E000F00D1124E459FC4EA301920166A177A15E
:10A3F00080A591A50E9467C54B015C01A301920154
:10A40000F70166A177A180A591A50E9467C5AB0160
:10A41000BC0195018401C7010E940943D701D6966A
:10A420001C92D394B0E1DB1201C0D12C7101AECFEC
:10A43000E114F10419F1F70182A093A0A4A0B5A042
:10A44000A50194016DEC7CEC8CE49DE30E9467C552
:10A450002B013C01A5019401D70196966D917D9148
:10A460008D919C9199970E9467C5AB01BC019301A6
:10A470008201C7010E940943F70116AA80916F006B
:10A48000826080936F00CF58DF4F0FB6F894DEBF25
:10A490000FBECDBFDF91CF911F910F91FF90EF9035
:10A4A000DF90CF90BF90AF909F908F907F906F90F4
:10A4B0005F904F903F902F9008952F923F924F9230
:10A4C0005F926F927F928F929F92AF92BF92CF9244
:10A4D000DF92EF92FF920F931F93CF93DF9300D001
:10A4E0001F92CDB7DEB74C01FC01E356F74E049145
:10A4F000892B21F0002E000C110B09C0809106134E
:10A50000882319F001E010E002C00FEF1FEFC40133
:10A51000880F991F880F991F9C838B83885E9C4EA0
:10A520001C01FC01108211821282138224E233E1A9
:10A5300040E253E16CE173E188E193E10E94E04481
:10A540008B819C818056974E0E94B5AD6B017C013A
:10A55000B801110F880B990B0E94A7BE2B013C017B
:10A560008B819C81805D964E5C0120E030E040EC68
:10A570005FE3C701B6010E94FEB8A30192010E94E9
:10A58000FEB8F50160837183828393838B819C8104
:10A59000815B9D4F9A838983FC0180819181A28197
:10A5A000B3818093630290936402A0936502B09399
:10A5B00066026AE077ED83EA9BE30E9413AE20E037
:10A5C00030E040EF51E46091630270916402809149
:10A5D0006502909166020E9467C536E0C32E33E1A2
:10A5E000D32E7B018C012CE339E148E359E164E38C
:10A5F00079E180E399E10E9483456AE077ED83EA9F
:10A600009BE30E9413AE0E9428A9F10110821182DF
:10A610001282138224E233E140E253E16CE173E100
:10A6200088E193E10E94E0448B819C818953914FA2
:10A630009C838B830E94B5AD9058A30192010E9428
:10A64000FEB8F50160837183828393836AE077EDBE
:10A6500083EA9BE30E9413AE20E030E040EF52E437
:10A66000609163027091640280916502909166022C
:10A670000E9467C57B018C012CE339E148E359E175
:10A6800064E379E180E399E10E9483456AE077ED34
:10A6900083EA9BE30E9413AE0E9428A98B819C81D0
:10A6A0000E94B5AD9B01AC010E9479C4A301920147
:10A6B0000E94FEB8F501608371838283938320E05A
:10A6C00030E040E05FE3E981FA816081718182815D
:10A6D00093810E94FEB8609363027093640280933A
:10A6E0006502909366026AE077ED83EA9BE30E943D
:10A6F00013AE20E030E044E353E4609163027091D4
:10A70000640280916502909166020E9467C57B0198
:10A710008C012CE339E148E359E164E379E180E31A
:10A7200099E10E9483456AE077ED83EA9BE30E940A
:10A7300013AE0E9428A9C4010E94FD7FF10180810F
:10A740009181A281B381F50180839183A283B38338
:10A7500010926302109264021092650210926602D7
:10A760001092091910920819109207190F900F9062
:10A770000F900F90DF91CF911F910F91FF90EF906D
:10A78000DF90CF90BF90AF909F908F907F906F9011
:10A790005F904F903F902F90089540916A0D509197
:10A7A0006B0D60E6649F9001659F300D1124BC0124
:10A7B000C9018651944F0E94BEBDE6E7F8E084913E
:10A7C000882341F09091C00095FFFCCF8093C60094
:10A7D0003196F5CFECEBFEE08491882341F0909127
:10A7E000C00095FFFCCF8093C6003196F5CF8091D5
:10A7F0006A0D90916B0D20E6289FF001299FF00DC6
:10A800001124E651F44F8191882339F09091C000D2
:10A8100095FFFCCF8093C600F6CFEAEBFEE0849173
:10A82000882341F09091C00095FFFCCF8093C60033
:10A830003196F5CF8091C00085FFFCCF8AE08093F0
:10A84000C60080916A0D90916B0D019664E070E0F6
:10A850000E941CC890936B0D80936A0D80916C0DC3
:10A8600090916D0D019690936D0D80936C0D0895F0
:10A870008EEA9EE00E94B5AD20910D1930910E191F
:10A8800040910F19509110190C9479C40895CF93E9
:10A89000DF93CAE0D0E06DEC7CEC8CEC9DE30E9491
:10A8A00013AE2197C1F78ED21092FA121092F912BC
:10A8B0001092FC121092FB121092DF0B1092DE0B22
:10A8C00080916C0D90916D0D04971CF487EA9EE0C9
:10A8D00064DF0E94C5A810923F1010923E101092A3
:10A8E000A9181092A81880E0DF91CF910C94E7A8E6
:10A8F000AF92BF92CF92DF92EF92FF920F931F938E
:10A90000CF93DF9380915F02882309F4A6C082E091
:10A9100090E090933F1080933E1084E50E94E4AD58
:10A92000882309F447C00E940AAE0E94D8C5EB01F3
:10A93000CB010E944F8111E0CD2B09F010E0C12E18
:10A94000D12C88E40E94E4AD882331F00E940AAE45
:10A950000E94D8C5EB0102C0C0E0D0E089E40E94AB
:10A96000E4AD8823B1F00E940AAE0E94D8C57B01F5
:10A97000112359F0161617061CF4C6010E9471A384
:10A980001C161D06BCF4CE0113C01C161D0644F097
:10A990000BC01111F5CF1C161D0664F4E12CF12C2F
:10A9A000BE01C6010E9471A31E141F041CF4C7013E
:10A9B0000E94379F60E070E081EF9FEF0E94C99A8C
:10A9C000C0909D12D0909E12E0909F12F090A01225
:10A9D00020E030E04AE754E4C701B6010E94C4C653
:10A9E00018164CF4C0926302D0926402E0926502A1
:10A9F000F09266020CC080E090E0AAE7B5E4809394
:10AA0000630290936402A0936502B0936602A090E3
:10AA10009912B0909A12C0909B12D0909C1210E89C
:10AA2000E12E1FE4F12E03EC17ECA8019701C801F9
:10AA3000B7010E94C07E109203131092021310926D
:10AA40003F1010923E1080914010882331F081E039
:10AA500090E090933F1080933E10DF91CF911F9133
:10AA60000F91FF90EF90DF90CF90BF90AF9008953F
:10AA70000F931F93CF93DF93FC0124813581211520
:10AA8000310519F4FB01108211C0EA0121972C173E
:10AA90003D0708F4E9018B01FC0160817181AE0181
:10AAA000C8010E94A8C9C00FD11F1882DF91CF91A1
:10AAB0001F910F9108953F924F925F926F927F92F4
:10AAC0008F929F92AF92BF92CF92DF92EF92FF92BE
:10AAD0000F931F93CF93DF93CDB7DEB7C558D1093E
:10AAE0000FB6F894DEBF0FBECDBF8C017B01312CB9
:10AAF0006B0184E0C80ED11C8EE4A82E80E1B82E34
:10AB000090E4892E912C8C0E9D1EE4E08E0E911CFB
:10AB10002FEB622E22E0722E33E6432E38E0532EC6
:10AB2000F7018781823008F434C184859585A68534
:10AB3000B7858F719927AA27BB27892B8A2B8B2B47
:10AB400009F027C1A114B10411F010924E104EE487
:10AB500050E1BE016F5F7F4FC6010E949C741816C2
:10AB60000CF017C12C85322F3871303109F0A1C09B
:10AB700080913312909134120197029708F499C092
:10AB8000BE016F5F7F4FCE0187589F4F0E94847236
:10AB9000A0961FAEA097F8018081811107C064EBD9
:10ABA00076E0CE01815A9F4F0E9474C9B801CE0150
:10ABB000815A9F4F0E9474C9BE0167587F4FCE01D2
:10ABC000815A9F4F0E9474C964EB76E0CE01815A8E
:10ABD0009F4F0E9474C9CE01805C9F4F0E94A27259
:10ABE00021E0AE0147585F4FB601C4010E9468637F
:10ABF00081113CC08091331290913412892BB1F5B0
:10AC0000F2018491E3E6F8E0882349F09091C000D6
:10AC100095FFFCCF8093C60031968491F5CFE6EB8B
:10AC2000F6E08191882339F09091C00095FFFCCF28
:10AC30008093C600F6CF8091C00085FFFCCF8AE0EC
:10AC40008093C600FE01E758FF4F8191882339F0B9
:10AC50009091C00095FFFCCF8093C600F6CF809105
:10AC6000C00085FFFCCF8AE08093C6008BE1FE0127
:10AC7000EC5BFF4FDE01959601900D928A95E1F70E
:10AC800024968EAD9FAD24979CA38BA37AA269A234
:10AC9000BE016F5D7F4FCE01815A9F4F0CDFCE0109
:10ACA00081960E949A72CE01805C9F4F0E949A7298
:10ACB00037CF8981882309F46CC0853E09F430CFF1
:10ACC0008E3209F42DCF8F3509F42ACF80914E10A2
:10ACD000882331F08E3209F423CF8F3509F420CF49
:10ACE00023FD1ECF81E0303109F080E080936910B0
:10ACF000811108C08985873409F012CF8A858E3783
:10AD000009F40ECFBE016F5F7F4F81E490E10E9496
:10AD1000847280913312909134120097F9F4F80103
:10AD20008191882339F09091C00095FFFCCF8093EA
:10AD3000C600F6CFE1E4F0E18191882339F09091EB
:10AD4000C00095FFFCCF8093C600F6CF8091C00075
:10AD500085FFFCCF8AE08093C600E2CE813091056A
:10AD600051F48091351290913612019690933612DB
:10AD700080933512D5CE029709F0D2CE832D90E084
:10AD800020913512309136128217930711F03394C7
:10AD9000C7CECB57DF4F0FB6F894DEBF0FBECDBF87
:10ADA000DF91CF911F910F91FF90EF90DF90CF90A7
:10ADB000BF90AF909F908F907F906F905F904F90DB
:10ADC0003F90089583E192E10E94077583E192E14B
:10ADD000F8D6EBE3F0E11182128208952F923F92B0
:10ADE0004F925F926F927F928F929F92AF92BF929B
:10ADF000CF92DF92EF92FF920F931F93CF93DF9347
:10AE0000CDB7DEB7C752D1400FB6F894DEBF0FBE44
:10AE1000CDBF50914010552309F4C7C21801290134
:10AE2000C95DDE4F4883C752D1406B01CB5DDE4F19
:10AE300099838883C552D14083E192E1C2D61092B2
:10AE40003F1010923E103E0128EE620E711CC301AD
:10AE50000E94A27284E790E19093941080939310E3
:10AE6000F60180818F3209F085C06FE270E0C60183
:10AE70000E947FC901967C0183010C5F1F4FE11482
:10AE8000F10409F47DC06FE270E0C7010E947FC940
:10AE90005C01009709F475C0E816F90608F071C066
:10AEA0004C018E189F08A401B701CE0101960E94A3
:10AEB000A8C9E1E0F0E0EC0FFD1FE80DF91D1082DC
:10AEC000CE0101967C01FC018191882339F090919B
:10AED000C00095FFFCCF8093C600F6CF8091C000E4
:10AEE00085FFFCCF9AE09093C6006091931070911B
:10AEF00094106115710511F06C5F7F4F21E0AE0178
:10AF00004F5F5F4FC8010E94686381112AC0E7E864
:10AF1000FFE08491882371F09091C00095FFFCCFF1
:10AF20008093C6003196F5CF9091C00095FFFCCF7D
:10AF30008093C600F70181917F018111F5CFE5E88B
:10AF4000FFE08491882341F09091C00095FFFCCFF1
:10AF50008093C6003196F5CF8091C00085FFFCCF6D
:10AF6000C0C170929410609293107501FFEFEF1AB8
:10AF7000FF0A85CF85E990E1909394108093931018
:10AF800076019091931080919410C95DDE4F2881D5
:10AF9000C752D140692F782F222309F4AAC1611525
:10AFA000710511F06C5F7F4F21E0A70183E192E111
:10AFB0000E946863882309F46BC1809124129091E8
:10AFC0002512A0912612B0912712809370109093B1
:10AFD0007110A0937210B0937310E7E7FFE08491B3
:10AFE000882341F09091C00095FFFCCF8093C6006C
:10AFF0003196F5CFF7018191882339F09091C00007
:10B0000095FFFCCF8093C600F6CFEFE6FFE084917A
:10B01000882341F09091C00095FFFCCF8093C6003B
:10B020003196F5CF6091701070917110809172100F
:10B03000909173104AE00E94F6268091C00085FF2F
:10B04000FCCF8AE08093C6002114310441045104EE
:10B0500071F020926C1030926D1040926E105092F0
:10B060006F10B201A10183E192E1C2D408C0109235
:10B070006C1010926D1010926E1010926F10E1E62D
:10B08000FFE08491882341F09091C00095FFFCCFB0
:10B090008093C6003196F5CF8091C00085FFFCCF2C
:10B0A0008AE08093C600B701CE01815E9E4F0E9468
:10B0B0000F90CB5DDE4F68817981C552D140CE01C2
:10B0C000875E9E4F0E940F90BE01615E7E4FCE0153
:10B0D000835F9E4F0E940790BE01675E7E4FCE0148
:10B0E0008D5E9E4F0E94079080914010882309F446
:10B0F000A8C0CE0187539F4F0E94A27209EC10E0B6
:10B100000C0F1D1F0C5F1F4F21E046E755E068E75D
:10B1100070E1C8010E946863882329F0C80151D5F5
:10B12000DD24D39401C0D12C68E374E0CE01895FA3
:10B130009E4F0E940F90BE016D5E7E4F8E010F5F8D
:10B140001F4FC8010E94079061E479E0C8010E9486
:10B15000DE8EBC01CE01895F9E4F0E942E8FC801FA
:10B160000E947C8FCF5EDE4F48815981C151D14012
:10B17000C35FDE4F68817981CD50D140CE01895FB8
:10B180009E4F0E94B18E7E0187E9E80EF11C42E3DA
:10B1900050E0B701CE01895F9E4F6ADCFF92EF92CB
:10B1A00080E29FE09F938F931F930F930E9472BE44
:10B1B0000F900F900F900F900F900F90DD2011F0D7
:10B1C00022E101C022EC89ECE82EF12CEC0EFD1EF0
:10B1D00094E0E90EF11C46E755E068E770E1C7012D
:10B1E0000E946863882379F0F80101900020E9F754
:10B1F0003197AF01401B510BB801C7010E94487540
:10B20000C701DFD414C0E1E1FFE08491882341F05D
:10B210009091C00095FFFCCF8093C6003196F5CF8A
:10B220008091C00085FFFCCF8AE08093C600CE01EC
:10B23000895F9E4F0E947C8FCE0187539F4F0E9453
:10B240009A72CE018D5E9E4F0E947C8FCE01835FED
:10B250009E4F0E947C8F812C912C540175016401BA
:10B2600000E010E020E030E040E050E060E070E01E
:10B27000CB010E94994210924813CE01875E9E4FE7
:10B280000E947C8FCE01815E9E4F0E947C8F8AC07F
:10B29000EDE4FFE08491882341F09091C00095FF98
:10B2A000FCCF8093C6003196F5CFF70181918823BA
:10B2B00039F09091C00095FFFCCF8093C600F6CF87
:10B2C000EBE4FFE08491882341F09091C00095FF6A
:10B2D000FCCF8093C6003196F5CF8091C00085FFEA
:10B2E000FCCF8AE08093C60010923F1010923E106F
:10B2F00059C06115710511F06C5F7F4F26E5A701FC
:10B3000083E192E10E94686381112AC0E7E3FFE0D4
:10B310008491882341F09091C00095FFFCCF8093E9
:10B32000C6003196F5CFF7018191882339F09091CD
:10B33000C00095FFFCCF8093C600F6CFE5E3FFE0A9
:10B340008491882341F09091C00095FFFCCF8093B9
:10B35000C6003196F5CF8091C00085FFFCCF1FC09D
:10B3600081E080933C10E3E2FFE08491882341F088
:10B370009091C00095FFFCCF8093C6003196F5CF29
:10B38000F6018191882339F09091C00095FFFCCFA0
:10B390008093C600F6CF8091C00085FFFCCF8AE085
:10B3A0008093C600C3010E949A72C95DDE4F0FB63A
:10B3B000F894DEBF0FBECDBFDF91CF911F910F91EB
:10B3C000FF90EF90DF90CF90BF90AF909F908F90C5
:10B3D0007F906F905F904F903F902F9008952091B5
:10B3E0004413309145134091461350914713609197
:10B3F00024137091251380912613909127130E9496
:10B40000FEB80E9471C7E8E2F3E16487758786871A
:10B4100097878FB7F89444855585668577854093DF
:10B4200014135093151360931613709317138FBF53
:10B4300008954F925F926F927F928F929F92AF92F8
:10B44000BF92CF92DF92EF92FF920F931F93CF9311
:10B45000DF93CDB7DEB7A0970FB6F894DEBF0FBE6F
:10B46000CDBFE0910713E11195C1ED8EFE8E0F8FD8
:10B4700018A3298F3A8F4B8F5C8F6D8B7E8B8F8BB0
:10B48000988F8091130290911402019709F0C6C021
:10B4900080911B1090911C10A0911D10B0911E1056
:10B4A000898B9A8BAB8BBC8B8091061381110FC05B
:10B4B00020E030E048E452E469897A898B899C89EC
:10B4C0000E9478C4698B7A8B8B8B9C8B06C08130F1
:10B4D00021F4412C512C320106C0412C512C88E41E
:10B4E000682E82EC782E88E50E94E4AD882309F46A
:10B4F00095C00E940AAE6D877E878F87988B82E504
:10B500000E94E4AD882329F00E940AAE9B01AC01A1
:10B5100004C020E030E040E85FE36D857E858F85E4
:10B5200098890E9467C56D877E878F87988B8DE489
:10B530000E94E4AD882309F45AC00E940AAE0E941A
:10B54000D8C54B0129893A894B895C896D857E85EF
:10B550008F8598890E94C4C6181654F0A3019201E1
:10B560006D857E858F8598890E94A1BE87FF58C012
:10B570008114910409F054C089EC96E00E940F6593
:10B5800020E030E040E251E460911813709119130B
:10B5900080911A1390911B130E94FEB80E94D8C587
:10B5A000AB01BC012AE0CE0101960E94B08F8981D7
:10B5B0009A810E940F6581E499E00E940F6588EBF3
:10B5C00094E00E940F650E9403659FEFA0E7B2E040
:10B5D0009150A040B040E1F700C000008CED96E033
:10B5E0000E941165CE0101960E947C8FD3C02989EB
:10B5F0003A894B895C896D857E858F8598890E9403
:10B60000C4C618160CF4B8CFA30192016D857E85CF
:10B610008F8598890E94A1BE87FDAECF812C912C89
:10B6200085E40E94E4AD81110AC020E83FE443ECC8
:10B6300057ECC601B5010E94C4C61816DCF480910F
:10B6400004139091051318161906A4F48FE00E94B4
:10B650007B33892B09F088C08091021390910313EA
:10B660008B3091050CF476C080913E1090913F1084
:10B67000019789F0ED8CFE8C0F8D18A1298D3A8DE4
:10B680004B8D5C8D6D897E898F89988D0E944C973A
:10B690000E94C3947FC010920313109202138AE099
:10B6A00090E0909301138093001368E374E0CE015F
:10B6B00007960E940F908091FE129091FF12892BA5
:10B6C00019F46EEE76E002C06FEF76E0CE010796D9
:10B6D0000E94198F62E574E0CE0101960E940F90DE
:10B6E000BE01695F7F4FCE0101960E94F58E68EB27
:10B6F00074E00E94DE8EBC01CE0107960E942E8F60
:10B70000CE0101960E947C8FEF80F88488E694E059
:10B710000E9411658AE097E00E94116585E297E03A
:10B720000E9411658EE397E00E9411658BE597E01A
:10B730000E9411658CE797E00E941165C7010E9485
:10B7400011658AEB94E00E941165CE0107960E9474
:10B750007C8F90CF10924B1310924A1301969093C6
:10B7600003138093021386CF80914A1390914B1359
:10B77000823091054CF010924B1310924A131092A4
:10B7800003131092021376CF019690934B1380937C
:10B790004A1370CFA0960FB6F894DEBF0FBECDBF90
:10B7A000DF91CF911F910F91FF90EF90DF90CF909D
:10B7B000BF90AF909F908F907F906F905F904F90D1
:10B7C00008953F924F925F926F927F928F929F92D5
:10B7D000AF92BF92CF92DF92EF92FF920F931F939F
:10B7E000CF93DF9300D01F92CDB7DEB7382E809174
:10B7F0003E1090913F10019719F03110D8C0E2C06F
:10B800008091FD128111F9CFF89460E088E00E94E8
:10B81000A33360E08BE00E94A33360E08AE00E94E3
:10B82000A33360E085E00E94A33360E089E00E94DA
:10B83000A3335F9A479A8A9A9FB7F8948091080138
:10B840008160809308019FBF9FB7F89480910801A1
:10B850008460809308019FBF8D9A129A8091FD1297
:10B86000811152C08090241390902513A09026132C
:10B87000B0902713C0902013D0902113E090221392
:10B88000F090231301E010E080910613811102C0B3
:10B8900000E010E06091FB127091FC12072E000C8A
:10B8A000880B990B0E94A7BE20E030E040E05FE3E8
:10B8B0000E9479C40E94D8C52B013C016091F91205
:10B8C0007091FA12072E000C880B990B0E94A7BEEC
:10B8D00020E030E040E05FE30E9479C40E94D8C5D8
:10B8E00069837A838B839C8360916C1070916D1057
:10B8F00080916E1090916F10920149815A810E943F
:10B90000994281E08093FD125F98479800E010E033
:10B910008BEDE82EFF24F394B801012E000C880B68
:10B92000990B0E94A7BE4B015C0120E030E040EA89
:10B9300051E4609138137091391380913A139091CA
:10B940003B130E94FEB89B01AC01C501B4010E94EB
:10B95000A1BE87FF52CFC8018170992721E08227BD
:10B96000817020911102309112022250310922304F
:10B97000310530F4882311F0889A08C0889808C0EF
:10B9800090910613913031F4882311F0419A09C047
:10B99000419807C0911105C0882311F0889A01C011
:10B9A0008898C7010197F1F70F5F1F4FB5CF8091BE
:10B9B0004913811107C0F89461E00E94BBAD81E09A
:10B9C000809349130F900F900F900F90DF91CF91BC
:10B9D0001F910F91FF90EF90DF90CF90BF90AF90AD
:10B9E0009F908F907F906F905F904F903F900895C1
:10B9F0008F929F92AF92BF92CF92DF92EF92FF927F
:10BA00000F931F93CF93DF93EC018B81811102C0C1
:10BA100080E077C009891A892B893C8904171507AA
:10BA200026073707A8F36A017B01823029F4C8860C
:10BA3000D986EA86FB860DC0C114D104E104F10465
:10BA400051F41C821D821E821F82188619861A8656
:10BA50001B8681E056C088849984AA84BB84E98DC2
:10BA6000FA8D258530E0275F3F4FB501A401415095
:10BA7000510961097109022E04C0769567955795A1
:10BA800047950A94D2F7D701C6010197A109B109D8
:10BA900004C0B695A795979587952A95D2F78417F0
:10BAA0009507A607B70720F089288A288B2849F42C
:10BAB0004D895E896F89788D4C835D836E837F832A
:10BAC00004C0841B950BA60BB70B4C015D018E01C6
:10BAD0000C5F1F4F81149104A104B10409F4A7CF96
:10BAE0004C815D816E817F819801898D9A8D0E9444
:10BAF000B57391E0891A9108A108B1088111EACFC4
:10BB000087CFDF91CF911F910F91FF90EF90DF9042
:10BB1000CF90BF90AF909F908F9008950F931F93F9
:10BB2000CF93DF93FC012381222311F080E044C0F6
:10BB30008B01EC01FB018789803139F18032B1F74B
:10BB400083E08B83F801428D538D648D758D4D8B11
:10BB50005E8B6F8B788F9E012F5E3F4FC8010E94D6
:10BB60003674882319F31A8F098F81E089831C8228
:10BB70001D821E821F82188619861A861B861C86C5
:10BB80001D861E861F86188A17C082E08B831D8A39
:10BB90001E8A1F8A188EFB01808D918DA0E0B0E077
:10BBA00025E0880F991FAA1FBB1F2A95D1F7898B03
:10BBB0009A8BAB8BBC8BD7CFDF91CF911F910F911D
:10BBC0000895CF93DF93EC010E9407751B82DF91EC
:10BBD000CF9108953F924F925F926F927F928F9292
:10BBE0009F92AF92BF92CF92DF92EF92FF920F930C
:10BBF0001F93CF93DF93CDB7DEB72C970FB6F89492
:10BC0000DEBF0FBECDBF5C01DC0159968D909C90CC
:10BC10005A97F40181859285A385B4859C01AD0175
:10BC20002F5F3F4F4F4F5F4F29873A874B875C8786
:10BC3000D5011496CD90DD90ED90FC901797C1142E
:10BC4000D104E104F10439F0BFEFCB1ADB0AEB0AAF
:10BC5000FB0A312C07C0F401C080D180E280F38060
:10BC600033243394260137011D821E821F821886D9
:10BC7000F40181859285A385B4852D813E814F8114
:10BC80005885281739074A075B0708F064C089857B
:10BC90009A85AB85BC858C159D05AE05BF0550F416
:10BCA00082E0C82ED12CE12CF12C92E0492E512CAF
:10BCB000612C712C9E012F5F3F4FB701A601C4017B
:10BCC0000E94B573882309F446C089819A81AB81AB
:10BCD000BC81892B8A2B8B2B41F0260137019FEFEA
:10BCE000491A590A690A790A05C0C414D504E60438
:10BCF000F70491F02D813E814F8158852F5F3F4F92
:10BD00004F4F5F4F2D833E834F8358873FEFC31ABA
:10BD1000D30AE30AF30AACCF0FEF1FEF2FEF3FE098
:10BD2000B301A201C4010E942473F82E882399F064
:10BD3000D50114964D915D916D917C9117974115A8
:10BD400051056105710549F093018201C4010E940A
:10BD50002473811102C0F12C29C0D50114964D9293
:10BD60005D926D927C921797332051F0D301C201FE
:10BD70000196A11DB11DF40180839183A283B38339
:10BD8000F50185899689A789B08D892B8A2B8B2B04
:10BD900069F4D50155964D925D926D927C925897BB
:10BDA00011968C911197806811968C938F2D2C96FB
:10BDB0000FB6F894DEBF0FBECDBFDF91CF911F91BC
:10BDC0000F91FF90EF90DF90CF90BF90AF909F903A
:10BDD0008F907F906F905F904F903F900895FC01FF
:10BDE00023812111EECE089561E0FC0180810C9445
:10BDF000A3338EBD0DB407FEFDCF08958FEF8EBD2A
:10BE00000DB407FEFDCF8EB508950F931F93CF930A
:10BE1000DF938B010E940D35EB01F0DF8F3F49F07E
:10BE20000E940D356C1B7D0B60177107B0F380E02D
:10BE300001C081E0DF91CF911F910F910895CF92C2
:10BE4000DF92EF92FF921F93CF93DF9300D01F9268
:10BE5000CDB7DEB76C01162FFC019281892F806A65
:10BE600086958CBD90FD03C081E0963009F480E09A
:10BE70008DBD60E0F601808129833A834B835C832A
:10BE80000E94A3336CE271E0C601BFDF812F8064A2
:10BE9000B0DF88E1E82EF12C5C814B813A81298169
:10BEA000DA01C9010E2C04C0B695A7959795879520
:10BEB0000A94D2F729833A834B835C839ADFF8E0B4
:10BEC000EF1AF10829813A814B815C8188EFE816ED
:10BED0008FEFF80629F7112321F0183021F08FEFAA
:10BEE00003C085E901C087E884DF1C3009F486DFE0
:10BEF00010E084DFF601838387FF04C01F3F11F049
:10BF00001F5FF7CF0F900F900F900F90DF91CF91A1
:10BF10001F91FF90EF90DF90CF9008950F931F93A4
:10BF2000CF93DF93EC0189018C81833039F089E074
:10BF3000440F551F661F771F8A95D1F79A01AB01F1
:10BF400068E1CE017CDF882311F086E02FC08EEF00
:10BF50008EBD80E090E00DB407FEFDCFF801E80F44
:10BF6000F91F20812EBD0DB407FEFDCF21812EBD0E
:10BF70000296811522E0920771F70DB407FEFDCFFE
:10BF80008FEF37DF8FEF35DF39DF8B838F718530B0
:10BF900029F083E18983CE0127DF09C068E572E0DB
:10BFA000CE0133DF182F811106C087E18983CE01CE
:10BFB0001BDF10E00FC020E030E0A9016DE0CE01F2
:10BFC0003EDF811103C01ADF882311F086E1EECF36
:10BFD000CE010ADF812FDF91CF911F910F9108953C
:10BFE000EF92FF920F931F93CF93DF93EC017901B0
:10BFF0008C81833039F089E0440F551F661F771F0D
:10C000008A95D1F79A01AB0161E1CE0118DF88234F
:10C0100011F084E013C00E940D358B01EFDE8B839D
:10C020008F3F49F40E940D35601B710B6D327140DA
:10C03000A8F381E103C08E3F31F08FE08983CE0108
:10C04000D3DE80E019C08FEF8EBDF701D701A1507C
:10C05000BE4F0DB407FEFDCF9EB591938EBDEA177E
:10C06000FB07B9F70DB407FEFDCF8EB58C93C6DE86
:10C07000C5DECE01B9DE81E0DF91CF911F910F9136
:10C08000FF90EF9008952F923F924F925F926F92A0
:10C090007F928F929F92AF92BF92CF92DF92EF9258
:10C0A000FF920F931F93CF93DF9300D01F92CDB7D2
:10C0B000DEB79C838B834B015A01DC0113968C9174
:10C0C000811103C08FEF9FEFEAC0EB81FC8181817A
:10C0D00080FFF8CFAB81BC8151960D911D912D91C0
:10C0E0003C91549718964D915D916D917C911B9761
:10C0F000C501A0E0B0E068017901C41AD50AE60ADA
:10C10000F70A8C159D05AE05BF0518F05801A41A55
:10C11000B50A75018B819C8104969A838983612C71
:10C1200092E0792EE114F10409F48BC0AB81BC815B
:10C1300018964D915D916D917C911B976A01B1E0CC
:10C14000DB22EB81FC8123811A012B0189E05694CB
:10C150004794379427948A95D1F7818D928D223018
:10C1600061F4FC01828D938DA48DB58DBC01CD0150
:10C17000620D731D841D951D4AC0DC0114961C912F
:10C1800011501221C114D10401F511111EC0452B0B
:10C19000462B472B59F4EB81FC8185899689A78929
:10C1A000B08D84839583A683B7830FC0AB81BC8198
:10C1B00014964D915D916D917C91179729813A81EB
:10C1C0000E94B573882309F47DCFEB81FC81218D1A
:10C1D000328D84819581A681B7810297A109B10929
:10C1E000F901058404C0880F991FAA1FBB1F0A9478
:10C1F000D2F74685578560897189840F951FA61FE0
:10C20000B71FBC01CD01610F711D811D911D9301EF
:10C210002C193D0987012E153F0508F489010115E8
:10C22000F2E01F0771F520916E0F30916F0F409172
:10C23000700F5091710F621773078407950719F4F7
:10C2400020C0C5012CC09401AB01BC018091770FC7
:10C250009091780FC5DE882309F434CF800E911EAB
:10C26000EB81FC8180859185A285B385800F911F2C
:10C27000A11DB11D80879187A287B387E01AF10ABB
:10C2800051CF40E00E94EC72882309F41BCFB60125
:10C290006259724FA801C4010E945AC9DFCF0F90A2
:10C2A0000F900F900F90DF91CF911F910F91FF9002
:10C2B000EF90DF90CF90BF90AF909F908F907F9046
:10C2C0006F905F904F903F902F9008954F925F92A4
:10C2D0006F927F929F92AF92BF92CF92DF92EF9236
:10C2E000FF920F931F93CF93DF931F92CDB7DEB7CB
:10C2F0008C017B016A01A22EDB0159968D919C91E4
:10C300005A97F801928F818F40E050E0BA01C7013F
:10C310006FDB912CF70180859185A285B3854189DA
:10C3200052896389748984179507A607B70708F0AF
:10C3300063C025E0B695A795979587952A95D1F77F
:10C34000F82FFF70BF2ED70113968C91823008F41E
:10C3500069C041E050E0BE016F5F7F4FC70193DECF
:10C36000019719F4898190E002C08FEF9FEF019649
:10C3700009F458C0F70180859185A285B3854F9651
:10C38000A11DB11D80879187A287B387F0E2BF9E70
:10C39000C0011124BC016259724F6115710509F485
:10C3A00041C0DB012C91222319F0253ED1F47CC140
:10C3B00091100EC040916E0F50916F0F6091700FF1
:10C3C0007091710FF8014487558766877787B08A27
:10C3D000FC01E259F24F8081882361F09924939403
:10C3E00099CF4BE050E0C6010E944DC9892B09F05E
:10C3F00091CF1AC0992493948A2D8274823491F437
:10C40000992009F49CC0D8015096BC9050971C9676
:10C410006D917D918D919C911F9741E00E94EC72EE
:10C42000811180C080E043C1A7FCFCCFF0E2BF9E39
:10C43000A00111249A012259324FD9011B968C91E7
:10C44000817121F08A2D827109F068C080916E0F90
:10C4500090916F0FA091700FB091710FF8018487C8
:10C460009587A687B787B08AFA01E259F24F4489C7
:10C47000558960E070E0BA0155274427D8015596E8
:10C480004D935D936D937C935897828D938DA0E02F
:10C49000B0E0482B592B6A2B7B2BD80155964D9336
:10C4A0005D936D937C935897D9011B968C918871FD
:10C4B00059F4848D958DA68DB78DF801818B928B63
:10C4C000A38BB48B81E010C0803141F598012F5EC1
:10C4D0003F4FD80159968D919C915A970E9436747E
:10C4E0008823E1F084E0F80183838A2D8F70D801DE
:10C4F00011968C931197F801148215821682178277
:10C5000018961D921D921D921C921B97A4FEC0C0EE
:10C51000C8010E942C288111BBC084CFD80113967A
:10C520001C9280CFF8016089F0E26F9FB001112466
:10C530006259724F6115710509F08AC073CFD70136
:10C5400013968C911397823009F46CCF51968D918C
:10C550009D910D90BC91A02D803E9F4FAF41B105A4
:10C5600008F060CFC70136DB882309F45BCF0E9457
:10C57000AC72882309F456CFD70159962D913C917E
:10C580005A9714968D919D910D90BC91A02D029774
:10C59000A109B109F901058404C0880F991FAA1FD8
:10C5A000BB1F0A94D2F74684578460887188480E6E
:10C5B000591E6A1E7B1E81E08093760F40926E0F9B
:10C5C00050926F0F6092700F7092710F80E092E046
:10C5D000EEE6FDE0DF019C011D9221503040E1F7C5
:10C5E000BB24B394D7015996ED91FC915A9784815D
:10C5F000B81690F42EE63DE0B301A2014B0D511D9B
:10C60000611D711D8091770F9091780F87DC8823D1
:10C6100009F408CFB394E6CF80E092E0A0E0B0E068
:10C62000058404C0880F991FAA1FBB1F0A94D2F764
:10C63000F7014189528963897489840F951FA61F68
:10C64000B71F818B928BA38BB48B6EE67DE0B12CF0
:10C6500080E2DB011D928A95E9F78BE0F601DB01B0
:10C6600001900D928A95E1F781E298E2FB01918BAE
:10C67000808B20E038E037872687938B828B918FE1
:10C68000808F378B268B0E94AC728111CFCECACEA1
:10C69000A5FE08C0F8014189528963897489C801DF
:10C6A000A7D905C081E003C0911098CE83CE0F902A
:10C6B000DF91CF911F910F91FF90EF90DF90CF907E
:10C6C000BF90AF909F907F906F905F904F90089534
:10C6D0002F923F924F925F926F927F928F929F9292
:10C6E000AF92BF92CF92DF92EF92FF920F931F9380
:10C6F000CF93DF93CDB7DEB7C554D1090FB6F89409
:10C70000DEBF0FBECDBF3C015B018A01322E1C8E05
:10C710001F8E19821C82672B11F410E0A6C0FC0149
:10C7200083818111FACFFA0180818F3261F4CA01CD
:10C730008C010196F80120812F32D1F3F50183811C
:10C740008250823010F475010AC0618D728DCE0165
:10C750000196E4D9882309F3CE0101967C016E018C
:10C760009CE1C90ED11C26014E01E7E38E0E911CFF
:10C77000FBE0F80D2596FFAF2597CE010196249694
:10C780009FAF8EAF24972696CFAE26972D2C35C01F
:10C7900080E2819325969FAD25979E13F9CFD8010E
:10C7A00090E027E04A2F3B2F8D91811128C08FA95F
:10C7B000803209F4B2CF842F932F8C01FC012081A9
:10C7C00001962F32D1F3222309F449C021E0A401BC
:10C7D000B701C6017BDD882309F49FCFEA14FB046F
:10C7E00011F0C701EED9C414D50491F126969FAD7E
:10C7F0002697822D7601C92ED82EF401C9CF8F320B
:10C80000B1F28E3219F0EBE9FFE00AC02A3009F4E8
:10C8100084CF98E02AE0C6CF3196381709F47DCF4F
:10C8200034913111F9CF291708F477CF3FED380F44
:10C830003E3508F072CF31E0390FF401E90FF11DF8
:10C840009FE9980F9A3108F480528083932FAACFE2
:10C8500023969FAD239724968FAD2497CBCF232D7E
:10C86000A401B701C30132DD182FCE010196B7DA5A
:10C87000CE014C96B4DA812FCB5BDF4F0FB6F89424
:10C88000DEBF0FBECDBFDF91CF911F910F91FF9003
:10C89000EF90DF90CF90BF90AF909F908F907F9060
:10C8A0006F905F904F903F902F9008954F925F92BE
:10C8B0006F927F928F929F92AF92BF92CF92DF92B0
:10C8C000EF92FF920F931F93CF93DF931F92CDB7F9
:10C8D000DEB75C016B014A01390144244A94542CAF
:10C8E000E12CF12C87010F5F1F4F0815190564F526
:10C8F00041E050E0BE016F5F7F4FC501C4DB2C01FA
:10C9000081E04816510401F569816D3099F0F60116
:10C91000EE0DFF1D60836114710419F46A3059F43F
:10C920000DC0062E000C770BC3010E947FC9892B16
:10C9300011F004C087017801D5CF8701F601E00F1F
:10C94000F11F1082C80104C057FEF7CF8FEF9FEF91
:10C950000F90DF91CF911F910F91FF90EF90DF909B
:10C96000CF90BF90AF909F908F907F906F905F908F
:10C970004F9008951F920F920FB60F9211240BB68D
:10C980000F922F933F934F936F937F938F939F9328
:10C99000EF93FF934091C6002091C10B3091C20BE1
:10C9A000C90101968F7799276091C30B7091C40BD1
:10C9B0008617970741F0F901EF5BF44F408390939E
:10C9C000C20B8093C10BFF91EF919F918F917F914B
:10C9D0006F914F913F912F910F900BBE0F900FBE13
:10C9E0000F901F90189580E090E00E9401288FEF33
:10C9F0009FEF0E9401288FEF9FEF0E9401288FEF89
:10CA00009FEF0C9401288FEF9FEF0E9401288FEF7A
:10CA10009FEF0E9401288FEF9FEF0C9401280C9448
:10CA200006280E9406288FEF9FEF0E9401288FEFB3
:10CA30009FEF0E9401288FEF9FEF0C9401281F9217
:10CA40000F920FB60F9211240BB60F92CF92DF9276
:10CA5000EF92FF920F931F932F933F934F935F9308
:10CA60006F937F938F939F93AF93BF93CF93DF93F6
:10CA7000EF93FF930E94EC9E81110C94776DDCB0D4
:10CA8000809149020E947B332CB139B15D2D5295C2
:10CA90005695577041E054275170C52F40E0D42F70
:10CAA00041E050E060914702709148028617970775
:10CAB00011F440E050E0C40FD51F22952F7081E0A3
:10CAC0002827022F017010E00C0F1D1F3695369598
:10CAD0003695832780FBEE24E0F8F12CE801CE0D9B
:10CAE000DF1D80917418909175188C179D07ECF4D8
:10CAF00080913E1090913F100197B9F080910C19F0
:10CB0000811108C080910B19811104C080910A190C
:10CB1000882359F00E940D35609370187093711836
:10CB200080937218909373181198C0907018D090D9
:10CB30007118E0907218F0907318C114D104E104D8
:10CB4000F104A1F00E940D35DC01CB018C199D0987
:10CB5000AE09BF0987399105A105B10538F080916B
:10CB60003E1090913F10019709F0E2C1D0937518E3
:10CB7000C0937418E091AA18F091AB18309709F09F
:10CB800080C19091AD188091AC18981769F0E09130
:10CB9000AC186DE4E69FF0011124E459FC4EDF016E
:10CBA000A45BBF4F81E08C93F093AB18E093AA187D
:10CBB000309709F460C1DF01A45BBF4F21E02C93E3
:10CBC00010926C1810926D1810926E1810926F18C7
:10CBD00080AD91AD81347CE9970728F481323EE441
:10CBE000930748F002C080E49CE996958795969556
:10CBF000879524E007C0813147E2940730F096958D
:10CC0000879522E020936B1807C020936B18803221
:10CC1000910510F480E290E08097811568E0960716
:10CC2000E8F0E92FFF27EE0FFF1FEE0FFF1F9F0118
:10CC300025553C4EF901329665917491AA27879F3C
:10CC4000A001869F410D5A1F06944A1F5A1F1124A6
:10CC5000F90125913491241B350B20C09C01369598
:10CC600027952C7F2555304FF90145915491F901B5
:10CC70003296A591B491BC0167707727A69F900169
:10CC8000A79F300DB69F300D112463E03695279590
:10CC90006A95E1F7BA01621B730B9B0124363105DB
:10CCA00080F4EFE9F7E02191222339F03091C000C0
:10CCB00035FFFCCF2093C600F6CF0E94182824E64B
:10CCC00030E030936A182093691880916B18082E11
:10CCD000000C990B9093681880936718E091AA183C
:10CCE000F091AB1884AD95AD90936618809365185C
:10CCF00081347CE9970728F481322EE4920748F0CA
:10CD000002C080E49CE9969587959695879524E0E6
:10CD100007C0813137E2930730F09695879522E07E
:10CD200020936B1808C021E020936B188032910586
:10CD300010F480E290E08097811548E09407E8F0D5
:10CD4000E92FFF27EE0FFF1FEE0FFF1F9F01255555
:10CD50003C4EF901329665917491AA27879FA001F4
:10CD6000869F410D5A1F06944A1F5A1F1124F9012C
:10CD700025913491241B350B20C09C0136952795B5
:10CD80002C7F2555304FF90145915491F901329688
:10CD9000A591B491BC0167707727A69F9001A79FCA
:10CDA000300DB69F300D1124B3E036952795BA9516
:10CDB000E1F7BA01621B730B9B012436310580F445
:10CDC000EFE9F7E02191222339F03091C00035FFDF
:10CDD000FCCF2093C600F6CF0E94182824E630E04E
:10CDE000C901A0E0B0E08093611890936218A0930D
:10CDF0006318B09364183093890020938800E09101
:10CE0000AA18F091AB1880899189A289B389B69547
:10CE1000A79597958795B095A095909581959F4FEB
:10CE2000AF4FBF4F80935D1890935E18A0935F182B
:10CE3000B09360188093591890935A18A0935B1878
:10CE4000B0935C188093551890935618A093571878
:10CE5000B09358188093511890935218A093531878
:10CE6000B093541810924D1810924E1810924F18FB
:10CE70001092501806C080ED97E09093890080933F
:10CE80008800E091AA18F091AB18309709F42FC6EA
:10CE900020A120934C18809111029091120220FF42
:10CEA00012C08230910511F4899808C0039719F4D3
:10CEB0008998439A06C081A1882311F0439801C044
:10CEC00089988FEF11C08230910511F4899A08C0BA
:10CED000039719F4899A439806C081A1882311F019
:10CEE000439A01C0899A81E080931502C0914C1841
:10CEF0001C2F127060914602C1FF08C080914B0246
:10CF00000E94A3338FEF8093160208C0D1E06D27F3
:10CF100080914B020E94A333D093160280910C198A
:10CF2000C0FF03C08111F9C40DC0811137C531C5DF
:10CF30001092701810927118109272181092731843
:10CF4000119A14CE8091AE188111E7C41123D9F043
:10CF500080910B19811104C08091AE18882399F03B
:10CF6000809149020E947B3321E040914702509119
:10CF700048028417950709F47AC5809149188111F0
:10CF800049C5209349189FB7C2FF1DC0F8948091EE
:10CF90000B018D7F80930B019FBF80912E19909183
:10CFA0002F19019741F09FB7F894809108018F7E67
:10CFB000809308019FBF8FEF8093170280910A1919
:10CFC00081115CC556C5F89480910B0182608093F5
:10CFD0000B019FBF80912E1990912F19019741F05D
:10CFE0009FB7F894809108018061809308019FBFEA
:10CFF00081E08093170220914C188091110290914A
:10D000001202029723FF13C0029710F48C9A07C0F4
:10D01000E091AA18F091AB1881A1813011F4169813
:10D0200001C08C9A8FEF80931802C0E0FEC0029777
:10D0300010F48C9807C0E091AA18F091AB1881A168
:10D04000813011F4169A01C08C9881E0ECCF809168
:10D05000C00087FDF0C0E091AA18F091AB18409194
:10D060005D1850915E1860915F1870916018808112
:10D070009181A281B381840F951FA61FB71F809352
:10D080005D1890935E18A0935F18B09360181816FF
:10D0900019061A061B060CF4E9C0E091AA18F091D3
:10D0A000AB18C0905918D0905A18E0905B18F090C7
:10D0B0005C1884819581A681B781C80ED91EEA1EAD
:10D0C000FB1EC0925918D0925A18E0925B18F09249
:10D0D0005C181C141D041E041F04CCF561E0809133
:10D0E0004D020E94A333E091AA18F091AB188089F9
:10D0F0009189A289B389C81AD90AEA0AFB0AC0929F
:10D100005918D0925A18E0925B18F0925C188091EE
:10D11000160240910C1350910D1360910E137091F3
:10D120000F13082E000C990BAA0BBB0B840F951F35
:10D13000A61FB71F80930C1390930D13A0930E138B
:10D14000B0930F1360E080914D020E94A333E091F1
:10D15000AA18F091AB18409155185091561860914B
:10D1600057187091581880859185A285B385840FD2
:10D17000951FA61FB71F8093551890935618A0931C
:10D180005718B0935818181619061A061B060CF4EF
:10D19000C7C0E091AA18F091AB1840915118509176
:10D1A0005218609153187091541884859585A685FE
:10D1B000B785840F951FA61FB71F809351189093B2
:10D1C0005218A0935318B0935418181619061A063B
:10D1D0001B060CF40AC180914D1890914E18A09135
:10D1E0004F18B09150180196A11DB11D80934D1894
:10D1F00090934E18A0934F18B093501840914D182B
:10D2000050914E1860914F1870915018E091AA18E3
:10D21000F091AB1880899189A289B3894817590781
:10D220006A077B0708F071C1CF5F80916B18C81740
:10D230000CF40DCF6AC14091C6002091C10B309112
:10D24000C20BC90101968F7799276091C30B70912A
:10D25000C40B8617970709F4FECEF901EF5BF44F74
:10D2600040839093C20B8093C10BF5CE8091110245
:10D27000909112020297029710F4889A03C081A13C
:10D28000813011F4419A03C0811101C0889AE09164
:10D29000AA18F091AB1880915D1890915E18A0913A
:10D2A0005F18B09160184089518962897389841B25
:10D2B000950BA60BB70B80935D1890935E18A09307
:10D2C0005F18B09360188091150240910813509137
:10D2D000091360910A1370910B13082E000C990B1F
:10D2E000AA0BBB0B840F951FA61FB71F80930813B3
:10D2F00090930913A0930A13B0930B13809111021A
:10D30000909112020297029710F4889803C081A1AD
:10D31000813011F44198C1CE8111BFCE8898BDCE25
:10D320009FB7F89480910B01886080930B019FBF99
:10D3300080912E1990912F19019741F09FB7F89481
:10D34000809108018860809308019FBFE091AA182E
:10D35000F091AB188091551890915618A0915718DC
:10D36000B09158184089518962897389841B950B43
:10D37000A60BB70B8093551890935618A093571887
:10D38000B0935818809117024091101350911113C7
:10D390006091121370911313082E000C990BAA0BB5
:10D3A000BB0B840F951FA61FB71F8093101390937C
:10D3B0001113A0931213B09313139FB7F894809195
:10D3C0000B01877F80930B019FBF80912E19909155
:10D3D0002F19019709F4DDCE9FB7F89480910801C9
:10D3E000877F809308019FBFD4CE80914018811120
:10D3F0000FC086B590E0A0E0B0E080933C18909319
:10D400003D18A0933E18B0933F1881E080934018D8
:10D4100080911102909112020297029710F48B9A58
:10D4200003C081A1813011F4149A01C08B9A4091FC
:10D430003C1850913D1860913E1870913F1886B588
:10D4400090E0A0E0B0E0841B950BA60BB70BE3E0E7
:10D45000880F991FAA1FBB1FEA95D1F74C97A1050A
:10D46000B10568F386B590E0A0E0B0E080933C1889
:10D4700090933D18A0933E18B0933F18E091AA18DE
:10D48000F091AB188091511890915218A0915318B7
:10D49000B09154184089518962897389841B950B16
:10D4A000A60BB70B8093511890935218A093531862
:10D4B000B093541880911802409114135091151391
:10D4C0006091161370911713082E000C990BAA0B7C
:10D4D000BB0B840F951FA61FB71F80931413909347
:10D4E0001513A0931613B093171380911102909106
:10D4F00012020297029710F48B9803C081A1813029
:10D5000011F4149868CE8B9866CE40914D185091C6
:10D510004E1860914F1870915018E091AA18F09130
:10D52000AB1884899589A689B78984179507A607BA
:10D53000B70708F4D6C04091611850916218609105
:10D54000631870916418048D158D268D378DAA2768
:10D55000419FB12D529FC001629F900D619F800D30
:10D56000911D429FB00D811D9A1F519FB00D811DCD
:10D570009A1F609FB00D811D9A1F509FB10D8A1F89
:10D580009A1FB6958A1F9A1F112424AD35AD820FBC
:10D59000931F909366188093651840AD51AD62ADAE
:10D5A00073ADA0E0B0E0481759076A077B0720F485
:10D5B000509366184093651880916518909166188D
:10D5C00081347CE9970728F481322EE4920748F0F1
:10D5D00002C080E49CE9969587959695879524E00E
:10D5E00007C0813137E2930730F09695879522E0A6
:10D5F00020936B1808C021E020936B1880329105AE
:10D6000010F480E290E08097811548E09407E8F0FC
:10D61000E92FFF27EE0FFF1FEE0FFF1F9F0125557C
:10D620003C4EF901329665917491AA27879FA0011B
:10D63000869F410D5A1F06944A1F5A1F1124F90153
:10D6400025913491241B350B20C09C0136952795DC
:10D650002C7F2555304FF90145915491F9013296AF
:10D66000A591B491BC0167707727A69F9001A79FF1
:10D67000300DB69F300D112413E0369527951A957D
:10D68000E1F7BA01621B730B9B012436310580F46C
:10D69000EFE9F7E02191222339F03091C00035FF06
:10D6A000FCCF2093C600F6CF0E94182824E630E075
:10D6B00030938900209388008091611890916218BE
:10D6C000A0916318B0916418820F931FA11DB11D22
:10D6D0008093611890936218A0936318B0936418B4
:10D6E000F4C040914D1850914E1860914F187091B0
:10D6F0005018808D918DA28DB38D84179507A60744
:10D70000B70708F0D6C040916C1850916D18609121
:10D710006E1870916F18048D158D268D378DAA2780
:10D72000419FB12D529FE001629FD00D619FC00DBE
:10D73000D11D429FB00DC11DDA1F519FB00DC11DFB
:10D74000DA1F609FB00DC11DDA1F509FB10DCA1FB7
:10D75000DA1FB695CA1FDA1F1124809165189091BF
:10D760006618E05CFF4F8C179D0718F4808191814B
:10D7700002C08C1B9D0B40815181628173818C01A1
:10D7800020E030E0041715072607370708F4CA0120
:10D7900081347CE9970728F481322EE4920748F01F
:10D7A00002C080E49CE9969587959695879524E03C
:10D7B00007C0813137E2930730F09695879522E0D4
:10D7C00020936B1808C021E020936B1880329105DC
:10D7D00010F480E290E08097811548E09407E8F02B
:10D7E000E92FFF27EE0FFF1FEE0FFF1F9F012555AB
:10D7F0003C4EF901329665917491AA27879FA0014A
:10D80000869F410D5A1F06944A1F5A1F1124F90181
:10D8100025913491241B350B20C09C01369527950A
:10D820002C7F2555304FF90145915491F9013296DD
:10D83000A591B491BC0167707727A69F9001A79F1F
:10D84000300DB69F300D112463E0369527956A950B
:10D85000E1F7BA01621B730B9B012436310580F49A
:10D86000EFE9F7E02191222339F03091C00035FF34
:10D87000FCCF2093C600F6CF0E94182824E630E0A3
:10D88000309389002093880080916C1890916D18D6
:10D89000A0916E18B0916F18820F931FA11DB11D3A
:10D8A00080936C1890936D18A0936E18B0936F18B6
:10D8B0000CC08091691890916A18909389008093A8
:10D8C00088008091671880936B1840914D18509193
:10D8D0004E1860914F1870915018E091AA18F0916D
:10D8E000AB1880899189A289B389481759076A07BB
:10D8F0007B0708F4FCC01092AB181092AA18909104
:10D90000AD188091AC18981709F4F1C08091AC184B
:10D910008F5F8F708093AC18EAC0E091AA18F091E5
:10D92000AB1881A1811112CB8CB191E085FB8827C6
:10D9300080F9892759F120914B18222339F1408130
:10D940005181628173811416150616061706F4F4C8
:10D95000409108135091091360910A1370910B13B1
:10D960004093CF0B5093D00B6093D10B7093D20B9D
:10D9700090930919408951896289738940934D18A0
:10D9800050934E1860934F187093501880934B1813
:10D99000DDCA8091AE18882309F4D8CAE091AA188C
:10D9A000F091AB1881A1882309F4D0CA8CB191E021
:10D9B00082958170892759F120914A18222339F1E3
:10D9C000408151816281738114161506160617066F
:10D9D000F4F4409108135091091360910A13709167
:10D9E0000B134093CF0B5093D00B6093D10B7093DC
:10D9F000D20B9093091940895189628973894093A8
:10DA00004D1850934E1860934F1870935018809390
:10DA10004A189CCAE091AA18F091AB1884819581AC
:10DA2000A681B781181619061A061B060CF0A9CA9A
:10DA300080910C1390910D13A0910E13B0910F13C0
:10DA40008093D30B9093D40BA093D50BB093D60BAC
:10DA50002093081980899189A289B38980934D18F0
:10DA600090934E18A0934F18B09350188ACA20E094
:10DA700088CA8091AE18882309F4BDCA89B191E0A3
:10DA800083FB882780F9892779F120914818222380
:10DA900059F1E091AA18F091AB1840855185628543
:10DAA00073851416150616061706F4F44091101324
:10DAB0005091111360911213709113134093D70B6F
:10DAC0005093D80B6093D90B7093DA0B909307198E
:10DAD000408951896289738940934D1850934E183B
:10DAE00060934F18709350188093481884CAFF9120
:10DAF000EF91DF91CF91BF91AF919F918F917F91E6
:10DB00006F915F914F913F912F911F910F91FF90D6
:10DB1000EF90DF90CF900F900BBE0F900FBE0F9045
:10DB20001F9018954F925F926F927F92AF92BF9223
:10DB3000CF92DF92EF92FF920F931F93CF93DF93D9
:10DB40008C01EB01FC0146A057A060A471A4AEA01B
:10DB5000BFA0C8A4D9A49501A601C301B2010E9427
:10DB6000A1BE87FF3FC0A3019201C301B2010E9481
:10DB7000FEB82B013C01F80182A993A9A4A9B5A97B
:10DB8000BC01CD0190589B01AC010E9479C4F80101
:10DB900026A537A540A951A90E94FEB89B01AC015A
:10DBA000C301B2010E9478C40E94AFC77B018C01FF
:10DBB0009B01AC01B501C6010E94A1BE87FF02C056
:10DBC000750186019701A801B501C6010E94A1BE99
:10DBD000882341F0A701B8014EA35FA368A779A7E6
:10DBE00081E08EABDF91CF911F910F91FF90EF906D
:10DBF000DF90CF90BF90AF907F906F905F904F90ED
:10DC00000895CF92DF92EF92FF920F931F93CF93DD
:10DC1000DF9300D01F92CDB7DEB78CE5C82E83E12D
:10DC2000D82E98E3E92E93E1F92E0CE413E1F601E6
:10DC300061917191819191916F01F70121913191E0
:10DC4000419151917F0129833A834B835C830E94E8
:10DC5000A5BE29813A814B815C810E94FEB80E9459
:10DC6000DEC5F80161937193819391938F01FCE676
:10DC7000CF16F3E1DF06D9F60F900F900F900F90BB
:10DC8000DF91CF911F910F91FF90EF90DF90CF9098
:10DC90000895089580E090E00895CF93DF93CDB785
:10DCA000DEB72A970FB6F894DEBF0FBECDBF2FEFB9
:10DCB00089EF90E0215080409040E1F700C00000E3
:10DCC00083EB97E00E940F656091FE127091FF1246
:10DCD0004AE0CE0101960E94DC8F89819A810E94E0
:10DCE0000F65CE0101960E947C8F0E9403652FEF85
:10DCF00089EF90E0215080409040E1F700C00000A3
:10DD000020E030E048EC52E460911B1070911C1050
:10DD100080911D1090911E100E94FEB80E94D8C5DF
:10DD2000AB01BC0189EC97E04F83588769877A87FC
:10DD30000E940F652AE04F81588569857A85CE015A
:10DD400001960E94B08F89819A810E940F65CE0151
:10DD500001960E947C8F0E9403652FEF89EF90E06F
:10DD6000215080409040E1F700C0000020E030E00A
:10DD700048EC52E46091371070913810809139105E
:10DD800090913A100E94FEB80E94D8C5AB01BC0128
:10DD90008AED97E04F83588769877A870E940F65DD
:10DDA0002AE04F81588569857A85CE0101960E94C7
:10DDB000B08F89819A810E940F65CE0101960E94E1
:10DDC0007C8F0E9403652FEF89EF90E02150804007
:10DDD0009040E1F700C0000020E030E048EC52E461
:10DDE0006091300B7091310B8091320B9091330B1D
:10DDF0000E94FEB80E94D8C5AB01BC018BEE97E033
:10DE00004F83588769877A870E940F652AE04F8180
:10DE1000588569857A85CE0101960E94B08F8981E7
:10DE20009A810E940F65CE0101960E947C8F0E940C
:10DE300003652FEF89EF90E0215080409040E1F79B
:10DE400000C0000020E030E048EC52E4609138135C
:10DE50007091391380913A1390913B130E94FEB850
:10DE60000E94D8C5AB01BC018CEF97E04F83588767
:10DE700069877A870E940F652AE04F8158856985F6
:10DE80007A85CE0101960E94B08F89819A810E9485
:10DE90000F65CE0101960E947C8F0E9403652FEFD3
:10DEA00089EF90E0215080409040E1F700C00000F1
:10DEB00020E030E048EC52E460913C1370913D1357
:10DEC00080913E1390913F130E94FEB80E94D8C5E6
:10DED000AB01BC018DE098E04F83588769877A8752
:10DEE0000E940F652AE04F81588569857A85CE01A9
:10DEF00001960E94B08F89819A810E940F65CE01A0
:10DF000001960E947C8F0E9403652FEF89EF90E0BD
:10DF1000215080409040E1F700C0000020E030E058
:10DF200048EC52E460914013709141138091421388
:10DF3000909143130E94FEB80E94D8C5AB01BC016A
:10DF40008EE198E04F83588769877A870E940F6532
:10DF50002AE04F81588569857A85CE0101960E9415
:10DF6000B08F89819A810E940F65CE0101960E942F
:10DF70007C8F0E9403652FEF89EF90E02150804055
:10DF80009040E1F700C0000020E030E048EC52E4AF
:10DF900060914413709145138091461390914713FB
:10DFA0000E94FEB80E94D8C5AB01BC018FE298E088
:10DFB0004F83588769877A870E940F652AE04F81CF
:10DFC000588569857A85CE0101960E94B08F898136
:10DFD0009A810E940F65CE0101960E947C8F0E945B
:10DFE00003652FEF89EF90E0215080409040E1F7EA
:10DFF00000C000004091961850919718052E000C13
:10E00000660B770B80E498E04F83588769877A879F
:10E010000E940F652AE04F81588569857A85CE0177
:10E0200001960E94B08F89819A810E940F65CE016E
:10E0300001960E947C8F0E9403652FEF89EF90E08C
:10E04000215080409040E1F700C0000040919418BA
:10E0500050919518052E000C660B770B82E598E021
:10E060004F83588769877A870E940F652AE04F811E
:10E07000588569857A85CE0101960E94B08F898185
:10E080009A810E940F65CE0101960E947C8F0E94AA
:10E0900003652FEF89EF90E0215080409040E1F739
:10E0A00000C0000020E030E040E251E460911B102D
:10E0B00070911C1080911D1090911E100E94FEB84E
:10E0C0000E94D8C5AB01BC0184E698E04F83588715
:10E0D00069877A870E940F652AE04F815885698594
:10E0E0007A85CE0101960E94B08F89819A810E9423
:10E0F0000F65CE0101960E947C8F0E9403652FEF71
:10E1000089EF90E0215080409040E1F700C000008E
:10E1100084E798E00E940F652AE040E85CE060E058
:10E1200070E0CE0101960E94B08F89819A810E9491
:10E130000F65CE0101960E947C8F0E9403652FEF30
:10E1400089EF90E0215080409040E1F700C000004E
:10E1500084E898E00E940F652AE040E15EE060E01C
:10E1600070E0CE0101960E94B08F89819A810E9451
:10E170000F65CE0101960E947C8F0E9403652FEFF0
:10E1800089EF90E0215080409040E1F700C000000E
:10E1900040912C0B50912D0B052E000C660B770B2C
:10E1A00084E998E04F83588769877A870E940F65D2
:10E1B0002AE04F81588569857A85CE0101960E94B3
:10E1C000B08F89819A810E940F65CE0101960E94CD
:10E1D0007C8F0E9403652FEF89EF90E021508040F3
:10E1E0009040E1F700C000004091AF185091B01886
:10E1F000052E000C660B770B87EA98E04F83588753
:10E2000069877A870E940F652AE04F815885698562
:10E210007A85CE0101960E94B08F89819A810E94F1
:10E220000F65CE0101960E947C8F0E9403652FEF3F
:10E2300089EF90E0215080409040E1F700C000005D
:10E240008091380B882319F08EEF94E002C08DEB9B
:10E2500098E00E9411652FEF89EF90E021508040F7
:10E260009040E1F700C000004091360B5091370B11
:10E27000052E000C660B770B8DEC98E04F835887CA
:10E2800069877A870E940F652AE04F8158856985E2
:10E290007A85CE0101960E94B08F89819A810E9471
:10E2A0000F65CE0101960E947C8F0E9403652FEFBF
:10E2B00089EF90E0215080409040E1F700C00000DD
:10E2C00040912E0B50912F0B052E000C660B770BF7
:10E2D00083EE98E04F83588769877A870E940F659D
:10E2E0002AE04F81588569857A85CE0101960E9482
:10E2F000B08F89819A810E940F65CE0101960E949C
:10E300007C8F0E9403652FEF89EF90E021508040C1
:10E310009040E1F700C0000088E694E00E9411659B
:10E3200082E090E0909301138093001367EF78E010
:10E33000CE0101960E940F9083E099E00E940F6544
:10E3400084E199E00E940F658091380B882319F0D1
:10E3500088E199E002C08FE194E00E940F652FEF01
:10E3600089EF90E0215080409040E1F700C000002C
:10E370008EE199E00E940F6588E299E00E940F65A6
:10E3800088EB94E00E9411652FEF89EF90E0215017
:10E3900080409040E1F700C00000099A119ACE0138
:10E3A00001960E947C8F2A960FB6F894DEBF0FBEAE
:10E3B000CDBFDF91CF910895CF93DF93CDB7DEB777
:10E3C000A0970FB6F894DEBF0FBECDBF40E250E07D
:10E3D000BE016F5F7F4F0E943855CE0101960E94AB
:10E3E0008DBDA0960FB6F894DEBF0FBECDBFDF91F6
:10E3F000CF9108956F927F928F929F92AF92BF922A
:10E40000CF92DF92EF92FF920F931F93CF93DF9300
:10E410008C01842E6901EB01EC80FD80C70101971E
:10E42000E0E0F0E02FEF3FEF40E050E0A0E0B0E0B0
:10E43000BE2EAF2E8E179F076CF1CA16DB0634F185
:10E44000EE15FF0558F4EB016880798061147104C2
:10E4500029F0E301CE0FDF1F988001C0912CEF015E
:10E460002196981431F0E817F90719F0B22EA32E6F
:10E4700009C01196A9014F5F5F4FE817F90711F422
:10E48000BC2EAD2EFE012B2D3A2DD2CFC8010E94FD
:10E49000239008C0CA16DB06CCF368E374E0C80119
:10E4A0000E940F90C801DF91CF911F910F91FF90B3
:10E4B000EF90DF90CF90BF90AF909F908F907F9024
:10E4C0006F900895FC01CB01BA012491222341F001
:10E4D0003091C00035FFFCCF2093C6003196F5CFB8
:10E4E0004AE00C94F626FC01CB01BA0124912223C8
:10E4F00041F03091C00035FFFCCF2093C60031962B
:10E50000F5CF42E00C947D27FC0120E03EE2DB01E8
:10E510004C91403241F0283011F430833196DB01C8
:10E520004C91408331962F5F6F5F7F4F2B3079F78F
:10E53000108208952FEB32E0FC0131832083049692
:10E540000C94EF5EFC0114821782138212828FEB0F
:10E5500092E0918380830895CF938091760F8823F2
:10E56000B9F140916E0F50916F0F6091700F7091E3
:10E57000710F2EE63DE08091770F9091780F0E9409
:10E580008E5FC82F811102C0C0E023C04091720F7E
:10E590005091730F6091740F7091750F4115510573
:10E5A0006105710591F02EE63DE08091770F909125
:10E5B000780F0E948E5F882339F31092720F1092A9
:10E5C000730F1092740F1092750F1092760F01C096
:10E5D000C1E08C2FCF910895CF92DF92EF92FF92FE
:10E5E000CF936B017C01C42F80916E0F90916F0FC0
:10E5F000A091700FB091710F8C159D05AE05BF05F0
:10E60000C9F0AADF811102C080E018C02EE63DE00B
:10E61000B701A6018091770F9091780F0E94F05F6B
:10E62000882391F3C0926E0FD0926F0FE092700F1B
:10E63000F092710F81E0C1118093760FCF91FF901E
:10E64000EF90DF90CF9008954F925F926F927F92FC
:10E650008F929F92AF92BF92CF92DF92EF92FF92F2
:10E660000F931F93CF93DF93EC016A017B01280185
:10E670003901423051056105710510F480E064C034
:10E6800089859A85AB85BC850196A11DB11D84172E
:10E690009507A607B70790F38F89803149F48D2C31
:10E6A0009E2CAF2CBB248B899C89AD89BE890FC061
:10E6B000803221F78B889C88AD88BE88DB01CA0137
:10E6C00057E0B695A795979587955A95D1F7880EF7
:10E6D000991EAA1EBB1E41E0C501B4017DDF88233F
:10E6E00069F29F89903161F4DD24EE24FF249601C4
:10E6F000220F331FF901E259F24F5182408211C0BB
:10E70000E894C7F8DD24EE24FF249601220F331F7E
:10E71000220F331FF901E259F24F40825182628287
:10E7200073829A89923080F04D815E816F81788505
:10E73000840E951EA61EB71E8092720F9092730FC4
:10E74000A092740FB092750FDF91CF911F910F912E
:10E75000FF90EF90DF90CF90BF90AF909F908F9001
:10E760007F906F905F904F900895CF92DF92EF92DD
:10E77000FF920F931F93CF93DF93FC0181859285C6
:10E78000A385B4850196A11DB11D84179507A60721
:10E79000B70710F480E061C08789803149F4BB2756
:10E7A000A72F962F852FC388D488E588F6880FC0B9
:10E7B000803281F783899489A589B6896A017B01B2
:10E7C000C7E0F694E794D794C794CA95D1F78C0D17
:10E7D0009D1DAE1DBF1DE9016A017B018F014091A6
:10E7E0006E0F50916F0F6091700F7091710F8417C1
:10E7F0009507A607B70799F4F80187898031B1F426
:10E80000B701A601552766277727440F551FFA0140
:10E81000E259F24F80819181A0E0B0E019C040E060
:10E82000BC01CD01D9DE8111E7CFB4CFB701A6017C
:10E830004F77552766277727440F551F440F551FDD
:10E84000FA01E259F24F80819181A281B381BF70B8
:10E8500088839983AA83BB8381E0DF91CF911F9145
:10E860000F91FF90EF90DF90CF9008954F925F92BD
:10E870006F927F92AF92BF92CF92DF92EF92FF9210
:10E880000F931F93CF93DF9300D01F92CDB7DEB7C6
:10E890008C0149835A836B837C835901C12CD12C11
:10E8A0007601412C82E0582E612C712C49815A81CD
:10E8B0006B817C819E012F5F3F4FC80156DF88230B
:10E8C00041F1D301C201F801058404C0880F991FEA
:10E8D000AA1FBB1F0A94D2F7C80ED91EEA1EFB1E40
:10E8E00049815A816B817C818789803139F481E04B
:10E8F000483F5F4F6105710538F4D8CF81E0483F4C
:10E900005F4F6F4F7F4090F2F501C082D182E2826B
:10E91000F3820F900F900F900F90DF91CF911F9186
:10E920000F91FF90EF90DF90CF90BF90AF907F90CE
:10E930006F905F904F900895DF92EF92FF920F9348
:10E940001F93CF93DF938C01EB017A018DE0D82EDA
:10E9500040E250E0BE01C8010E9443608032910550
:10E9600039F021E0892B09F420E0822F819547C0FE
:10E9700028812223C1F0253E59F32E3249F33B85ED
:10E980003F733F3061F4E114F10449F04A8D5B8D2F
:10E99000452B29F42F713FEF320F323030F02B85A9
:10E9A00023FDD6CF2CC080E02AC030E021503109B1
:10E9B000D29EC001D39E900D1124F701E80FF91FDC
:10E9C000298120832B8121832D8122832F81238301
:10E9D000298524832E852583288926832A892783D0
:10E9E0002C8920872E892187288D22872C8D2387AB
:10E9F0002E8D2487288126FFD2CF1586D0CFDF9198
:10EA0000CF911F910F91FF90EF90DF900895CF93DA
:10EA1000DF93EC018B818823A9F1898187FF2FC0C7
:10EA20006C857D858E859F8541E0D6DD882351F1FB
:10EA3000E88980E2E89FF0011124DF01A259B24F7A
:10EA4000109701F18C91853EE9F08B81823050F472
:10EA500049895A896B897C895C964D935D936D9346
:10EA60007C935F978D899E89AF89B88DE259F24F6B
:10EA7000938F828FB58BA48B89818F778983DF9168
:10EA8000CF916ACD81E0888380E0DF91CF910895B6
:10EA90002F923F924F925F926F927F928F929F92AE
:10EAA000AF92BF92CF92DF92EF92FF920F931F939C
:10EAB000CF93DF9300D01F92CDB7DEB78C014B010F
:10EAC0001A01DC0113968C9113978130C9F41196C9
:10EAD0008C9181FF15C082FF19C0F80141895289CC
:10EAE0006389748980859185A285B385841795078C
:10EAF000A607B70759F0C8010E94F85C811106C04B
:10EB000081E0F80180838FEF9FEF2CC1610185C008
:10EB1000D80159968D919C915A97FC0124812150DE
:10EB20002A013B0139E076946794579447943A95CB
:10EB3000D1F7722E74207A01F1E0FF22772009F4D8
:10EB400078C080E092E08E199F0956018C159D05D2
:10EB500008F45C01D80159962D913C915A9714966E
:10EB60008D919D910D90BC91A02D0297A109B109A5
:10EB7000F901058404C0880F991FAA1FBB1F0A94BE
:10EB8000D2F74685578560897189840F951FA61F26
:10EB9000B71F9C01AD01270D311D411D511D2901DC
:10EBA0003A01A11432E0B30609F089C080916E0FDA
:10EBB00090916F0FA091700FB091710F8415950512
:10EBC000A605B70569F41092760F8FEF9FEFDC0171
:10EBD00080936E0F90936F0FA093700FB093710F8F
:10EBE0009401B301A2018091770F9091780F0E9458
:10EBF0008E5F882309F484CFF80180859185A285F2
:10EC0000B3858A0D9B1DA11DB11D80879187A287A9
:10EC1000B3878A0C9B1CCA18DB08D80118964D9143
:10EC20005D916D917C911B97C114D10409F070CF57
:10EC30007AC0E114F10409F084CF14964D915D91EE
:10EC40006D917C911797411551056105710559F436
:10EC500055968D919D910D90BC91A02D0097A10589
:10EC6000B10539F520C09E012F5F3F4F7EDD88231F
:10EC700009F446CF89819A81AB81BC81F801218D4D
:10EC8000328DF9012789203139F4883FFFEF9F0742
:10EC9000A105B10540F40DC0883F2FEF9207A207F0
:10ECA0002FE0B20730F0C8010E94EA5D811149CF20
:10ECB00027CFF80184839583A683B78342CFE114DD
:10ECC000F10411F5D80118964D915D916D917C91EB
:10ECD0001B9751968D919D910D90BC91A02D481739
:10ECE00059076A077B0780F037DC882309F408CFCF
:10ECF00081E08093760F40926E0F50926F0F60927A
:10ED0000700F7092710F07C041E0C301B20164DC63
:10ED1000882309F4F5CEA501B401C7018259924FA9
:10ED20000E945AC969CF51968D919D910D90BC91C9
:10ED3000A02D84179507A607B70740F4F801418B6B
:10ED4000528B638B748B818180688183D80111968B
:10ED50008C9183FD02C0C10105C0C80158DE81113C
:10ED6000FACFCECE0F900F900F900F90DF91CF91F2
:10ED70001F910F91FF90EF90DF90CF90BF90AF90D9
:10ED80009F908F907F906F905F904F903F902F90CB
:10ED90000895CF93DF931F92CDB7DEB7698341E02B
:10EDA00050E0BE016F5F7F4F049672DE0F90DF91DF
:10EDB000CF910895CF93DF93EC0168E374E00E9454
:10EDC0000F908AE79FE00E94548C892B79F08AE7A4
:10EDD0009FE00E94328C682FCE010E94068F62E075
:10EDE00070E080E090E00E94D534EBCFCE01DF915F
:10EDF000CF9108958F929F92AF92BF92CF92DF9260
:10EE0000EF92FF920F931F93CF93DF93CDB7DEB7AF
:10EE10006E970FB6F894DEBF0FBECDBF69EC76E0FB
:10EE2000CE0107960E940F9020E030E040E251E4CE
:10EE3000609118137091191380911A1390911B13FC
:10EE40000E94FEB80E94D8C5AB01BC012AE0CE01E9
:10EE500001960E94B08FBE01695F7F4FCE010D9673
:10EE60000E940790BE016F5F7F4FCE010D960E94FA
:10EE7000F58E61E479E00E94DE8EBC01CE0107963A
:10EE80000E942E8FCE010D960E947C8F20E030E0F4
:10EE900040E251E460911C1370911D1380911E1388
:10EEA00090911F130E94FEB80E94D8C5AB01BC010F
:10EEB0002AE0CE010D960E94B08FBE01635F7F4FA6
:10EEC000CE0101960E94438FCE010D960E947C8F49
:10EED000BE01695F7F4FCE010D960E940790BE0173
:10EEE0006F5F7F4FCE010D960E94F58E61E479E051
:10EEF0000E94DE8EBC01CE0107960E942E8FCE01AD
:10EF00000D960E947C8F20E030E040E251E4609159
:10EF100020137091211380912213909123130E944A
:10EF2000FEB80E94D8C5AB01BC012AE0CE010D9607
:10EF30000E94B08FBE01635F7F4FCE0101960E9499
:10EF4000438FCE010D960E947C8FBE01695F7F4F7B
:10EF5000CE010D960E940790BE016F5F7F4FCE01DC
:10EF60000D960E94F58E61E479E00E94DE8EBC0170
:10EF7000CE0107960E942E8FCE010D960E947C8FA7
:10EF800020E030E040E251E46091241370912513B9
:10EF900080912613909127130E94FEB80E94D8C535
:10EFA000AB01BC012AE0CE010D960E94B08FBE01DC
:10EFB000635F7F4FCE0101960E94438FCE010D9675
:10EFC0000E947C8FBE01695F7F4FCE010D960E942B
:10EFD0000790BE016F5F7F4FCE010D960E94F58EA8
:10EFE00061E479E00E94DE8EBC01CE0107960E94AA
:10EFF0002E8FCE010D960E947C8F6091F912709138
:10F00000FA12072E000C880B990B0E94A7BE20E075
:10F0100030E040E05FE30E9479C40E94D8C5AB01B4
:10F02000770F660B770B2AE0CE010D960E94B08F0A
:10F03000BE01635F7F4FCE0101960E94438FCE01D8
:10F040000D960E947C8FBE01695F7F4FCE010D96A9
:10F050000E940790BE016F5F7F4FCE010D960E9408
:10F06000F58E61E479E00E94DE8EBC01CE01079648
:10F070000E942E8FCE010D960E947C8F20E030E002
:10F0800040E05FE3609157127091581280915912DD
:10F0900090915A120E9479C40E94D8C5AB01770F93
:10F0A000660B770B2AE0CE010D960E94B08FBE0151
:10F0B000635F7F4FCE0101960E94438FCE010D9674
:10F0C0000E947C8FBE01695F7F4FCE010D960E942A
:10F0D0000790BE016F5F7F4FCE010D960E94F58EA7
:10F0E00061E479E00E94DE8EBC01CE0107960E94A9
:10F0F0002E8FCE010D960E947C8F6091FB12709135
:10F10000FC12072E000C880B990B0E94A7BE20E072
:10F1100030E040E05FE30E9479C40E94D8C5AB01B3
:10F12000770F660B770B2AE0CE010D960E94B08F09
:10F13000BE01635F7F4FCE0101960E94438FCE01D7
:10F140000D960E947C8FBE01695F7F4FCE010D96A8
:10F150000E940790BE016F5F7F4FCE010D960E9407
:10F16000F58E61E479E00E94DE8EBC01CE01079647
:10F170000E942E8FCE010D960E947C8F20E030E001
:10F1800040E05FE360915B1270915C1280915D12D0
:10F1900090915E120E9479C40E94D8C5AB01770F8E
:10F1A000660B770B2AE0CE010D960E94B08FBE0150
:10F1B000635F7F4FCE0101960E94438FCE010D9673
:10F1C0000E947C8FBE01695F7F4FCE010D960E9429
:10F1D0000790BE016F5F7F4FCE010D960E94F58EA6
:10F1E00061E479E00E94DE8EBC01CE0107960E94A8
:10F1F0002E8FCE010D960E947C8F6091DE0B709158
:10F20000DF0B072E000C880B990B0E94A7BE20E095
:10F2100030E040E05FE30E9479C40E94D8C5AB01B2
:10F22000770F660B770B2AE0CE010D960E94B08F08
:10F23000BE01635F7F4FCE0101960E94438FCE01D6
:10F240000D960E947C8FBE01695F7F4FCE010D96A7
:10F250000E940790BE016F5F7F4FCE010D960E9406
:10F26000F58E61E479E00E94DE8EBC01CE01079646
:10F270000E942E8FCE010D960E947C8F20E030E000
:10F2800040E05FE36091471270914812809149120B
:10F2900090914A120E9479C40E94D8C5AB01770FA1
:10F2A000660B770B2AE0CE010D960E94B08FBE014F
:10F2B000635F7F4FCE0101960E94438FCE010D9672
:10F2C0000E947C8FBE01695F7F4FCE010D960E9428
:10F2D0000790BE016F5F7F4FCE010D960E94F58EA5
:10F2E00061E479E00E94DE8EBC01CE0107960E94A7
:10F2F0002E8FCE010D960E947C8F4091A8185091C0
:10F30000A918052E000C660B770B2AE0CE010D968E
:10F310000E94B08FBE01635F7F4FCE0101960E94B5
:10F32000438FCE010D960E947C8FBE01695F7F4F97
:10F33000CE010D960E940790BE016F5F7F4FCE01F8
:10F340000D960E94F58E61E479E00E94DE8EBC018C
:10F35000CE0107960E942E8FCE010D960E947C8FC3
:10F360004091610250916202052E000C660B770BF2
:10F370002AE0CE010D960E94B08FBE01635F7F4FE1
:10F38000CE0101960E94438FCE010D960E947C8F84
:10F39000BE01695F7F4FCE010D960E940790BE01AE
:10F3A0006F5F7F4FCE010D960E94F58E61E479E08C
:10F3B0000E94DE8EBC01CE0107960E942E8FCE01E8
:10F3C0000D960E947C8F80913E1090913F1081306D
:10F3D000910509F063C0BE01695F7F4FCE010D96B4
:10F3E0000E9407906FE279E0CE010D960E94DE8EBA
:10F3F000BC01CE0107960E942E8FCE010D960E9471
:10F400007C8F40911612442329F1809170109091C5
:10F410007110A0917210B09173100097A105B10501
:10F42000C1F0BC01CD016D597F4F8F4F9F4F24E636
:10F4300030E040E050E00E943DC460916C1070915B
:10F440006D1080916E1090916F100E943DC4422FFC
:10F4500001C040E050E060E070E02AE0CE010D968F
:10F460000E94B08FBE01635F7F4FCE0101960E9464
:10F47000438FCE010D960E947C8FBE01695F7F4F46
:10F48000CE010D960E940790BE016F5F7F4FCE01A7
:10F490000D960E94F58E61E479E019C0009751F451
:10F4A000BE01695F7F4FCE010D960E94079062E317
:10F4B00079E00BC00297B1F4BE01695F7F4FCE01C6
:10F4C0000D960E94079067E379E0CE010D960E94A9
:10F4D000DE8EBC01CE0107960E942E8FCE010D96C6
:10F4E0000E947C8F4091061350E060E070E02AE0BB
:10F4F000CE010D960E94B08FBE01635F7F4FCE019B
:10F5000001960E94438FCE010D960E947C8FBE0112
:10F51000695F7F4FCE010D960E940790BE016F5F1D
:10F520007F4FCE010D960E94F58E61E479E00E9436
:10F53000DE8EBC01CE0107960E942E8FCE010D9665
:10F540000E947C8F4091130250911402052E000CF2
:10F55000660B770B2AE0CE010D960E94B08FBE019C
:10F56000635F7F4FCE0101960E94438FCE010D96BF
:10F570000E947C8FBE01695F7F4FCE010D960E9475
:10F580000790BE016F5F7F4FCE010D960E94F58EF2
:10F5900061E479E00E94DE8EBC01CE0107960E94F4
:10F5A0002E8FCE010D960E947C8F80913E109091FF
:10F5B0003F10019709F086C00E940D3520E6822E8B
:10F5C0002AEE922EA12CB12CA50194010E943DC4DB
:10F5D00069017A016091390B70913A0B80913B0B74
:10F5E00090913C0BA50194010E943DC4C601821B71
:10F5F000930B6CE370E00E9408C87B010AE010E006
:10F60000B8010E941CC8282FCB01B8010E941CC859
:10F61000805D80937618205D20937718109278187B
:10F6200066E778E1CE0149960E940F90C7019927BD
:10F63000B8010E941CC8282FCB01B8010E941CC829
:10F64000805D80937618205D20937718109278184B
:10F6500066E778E1CE010D960E940F90BE01635FD0
:10F660007F4FCE0143960E94079067EA73E0CE0178
:10F6700043960E94DE8EBE01675E7F4F0E94F58E2C
:10F68000BC01CE0101960E942E8FCE0143960E94AE
:10F690007C8FCE010D960E947C8FCE0149960E94F0
:10F6A0007C8FBE01695F7F4FCE010D960E9407904F
:10F6B000BE016F5F7F4FCE010D960E94F58E61E413
:10F6C00079E00BC0BE01695F7F4FCE010D960E94AD
:10F6D00007906CE379E0CE010D960E94DE8EBC01AE
:10F6E000CE0107960E942E8FCE010D960E947C8F30
:10F6F00080911612BE01695F7F4F882339F0CE01D9
:10F700000D960E9407906FE279E006C0CE010D963B
:10F710000E94079060E479E0CE010D960E94DE8E93
:10F72000BC01CE0107960E942E8FCE010D960E943D
:10F730007C8F6091F9127091FA12072E000C880BE1
:10F74000990B0E94A7BE20915712309158124091F8
:10F75000591250915A120E94C4C6BE01695F7F4F70
:10F7600018163CF4CE010D960E9407906FE279E0E6
:10F7700006C0CE010D960E94079060E479E0CE01AC
:10F780000D960E94DE8EBC01CE0107960E942E8F40
:10F79000CE010D960E947C8F6091FB127091FC123D
:10F7A000072E000C880B990B0E94A7BE20915B12BC
:10F7B00030915C1240915D1250915E120E94C4C65D
:10F7C000BE01695F7F4F18163CF4CE010D960E9472
:10F7D00007906FE279E006C0CE010D960E94079077
:10F7E00060E479E0CE010D960E94DE8EBC01CE0170
:10F7F00007960E942E8FCE010D960E947C8F6091FD
:10F80000DE0B7091DF0B072E000C880B990B0E940A
:10F81000A7BE209147123091481240914912509151
:10F820004A120E94C4C6BE01695F7F4F18163CF49D
:10F83000CE010D960E9407906FE279E006C0CE01DE
:10F840000D960E94079060E479E0CE010D960E942B
:10F85000DE8EBC01CE0107960E942E8FCE010D9642
:10F860000E947C8FBE01695F7F4FCE010D960E9482
:10F87000079068EB74E0CE010D960E94DE8EBC010D
:10F88000CE0107960E942E8FCE010D960E947C8F8E
:10F890008F8198850E9411652FEF80E792E02150BB
:10F8A00080409040E1F700C000008CED96E00E949F
:10F8B0001165809100139091011397FD0EC080FF98
:10F8C00002C0119801C0119A809100139091011308
:10F8D0000197909301138093001380917E188111FA
:10F8E00005C00E944D6E81E080937E18CE01019686
:10F8F0000E947C8FCE0107960E947C8F6E960FB679
:10F90000F894DEBF0FBECDBFDF91CF911F910F9155
:10F91000FF90EF90DF90CF90BF90AF909F908F902F
:10F9200008954F925F926F927F928F929F92AF92C3
:10F93000BF92CF92DF92EF92FF920F931F93CF93DC
:10F94000DF93CDB7DEB768970FB6F894DEBF0FBE72
:10F95000CDBF7C0183E50E94E4AD882349F00E947D
:10F960000AAE0E94D8C57093DF0B6093DE0B16C001
:10F9700082E50E94E4AD882359F00E940AAE0E94FD
:10F98000D8C57093DF0B6093DE0B1092350209C06F
:10F99000F7FC07C0F092DF0BE092DE0B81E0809372
:10F9A00035020E940D352B013C016091DE0B7091F8
:10F9B000DF0B072E000C880B990B0E94A7BEFF24BB
:10F9C000F39420914712309148124091491250917E
:10F9D0004A120E94C4C618160CF0F12CF092A3181B
:10F9E00081E080933B108BECE82E87E1F82E97ECBA
:10F9F000C92E97E1D92E23ECA22E27E1B22E3AE0B0
:10FA0000932E8091A3186091DE0B7091DF0B8823F9
:10FA100009F479C1072E000C880B990B0E94A7BE30
:10FA200020914712309148124091491250914A1248
:10FA30000E94C4C618160CF080C10E940D35DC016E
:10FA4000CB0184199509A609B709893E9340A10500
:10FA5000B10508F447C1E091061384E0E89FF00186
:10FA60001124E95AFD4E6081718182819381F701F1
:10FA70002491EBECF7E1222349F03091C00035FFEF
:10FA8000FCCF2093C60031962491F5CF42E00E942E
:10FA90007D27F6018491E7ECF7E1882349F0909106
:10FAA000C00095FFFCCF8093C60031968491F5CFBE
:10FAB0006091061370E080E090E00E946B27F501F2
:10FAC0008491E3ECF7E1882349F09091C00095FF21
:10FAD000FCCF8093C60031968491F5CF6091471298
:10FAE000709148128091491290914A1241E00E940F
:10FAF0007D278091C00085FFFCCF9092C6000E94B8
:10FB00000D352B013C01CE010D9654D9CE010D9639
:10FB10000E94BE28882309F4E1C068E374E0CE01A6
:10FB200007960E940F906CE275E0CE0101960E944C
:10FB30000F90AE01495F5F4FBE016F5F7F4FCE01F7
:10FB40000D960E944B8DCE0101960E947C8FCE01B6
:10FB500007960E947C8F68E374E0CE0107960E94AE
:10FB60000F9067E374E0CE0101960E940F90AE0102
:10FB7000495F5F4FBE016F5F7F4FCE010D960E94C0
:10FB80004B8DCE0101960E947C8FCE0107960E947C
:10FB90007C8FBE01635F7F4FCE0101960E9407906C
:10FBA00020E030E040E2BE016F5F7F4FCE0107965C
:10FBB0000E94FA71CE0101960E947C8F63E479E085
:10FBC000CE0107960E94928E882309F44AC0BE0196
:10FBD000635F7F4FCE0143960E94079021E030E0A3
:10FBE00040E2BE016D5E7F4FCE0101960E94FA7128
:10FBF000CE0143960E947C8F21E030E040E050E04F
:10FC0000BE016F5F7F4FCE0143960E94239068E450
:10FC100079E0CE0143960E94928E882ECE014396C3
:10FC20000E947C8F8820A1F02D813E8141E050E030
:10FC3000BE016F5F7F4FCE0143960E942390CE019D
:10FC400043960E942C8D8B01CE0143960E947C8F9F
:10FC50001093DF0B0093DE0BCE0101960E947C8F88
:10FC600039C06AE479E0CE010D960E94928E882315
:10FC700019F00E9447542EC060E579E0CE010D9640
:10FC80000E94928E882329F080E090E00E942B9BB6
:10FC900021C066E579E0CE010D960E94928E811119
:10FCA00019C025E030E040E050E0BE01635F7F4FC7
:10FCB000CE0101960E9423906FE579E0CE01019676
:10FCC0000E94928E882ECE0101960E947C8F811018
:10FCD0000E947854CE0107960E947C8FCE010D962B
:10FCE0000E947C8F0E9403A58091DD0B882331F058
:10FCF0000E94E25610923F1010923E100E94AC9D5E
:10FD00000E9481327ECE072E000C880B990B0E9438
:10FD1000A7BE20914712309148124091491250914C
:10FD20004A120E94A1BE87FF08C08091350281114E
:10FD300004C080911612811180CE10923B100E9457
:10FD40000D35609340197093411980934219909337
:10FD5000431968960FB6F894DEBF0FBECDBFDF9192
:10FD6000CF911F910F91FF90EF90DF90CF90BF90B8
:10FD7000AF909F908F907F906F905F904F9008957D
:10FD80002F923F924F925F926F927F928F929F92AB
:10FD9000AF92BF92CF92DF92EF92FF920F931F9399
:10FDA000CF93DF93CDB7DEB728970FB6F894DEBFB9
:10FDB0000FBECDBF2B013C0129833A834B835C836B
:10FDC000ED82FE820F83188785E40E94E4AD8823CC
:10FDD00009F4F7C020E83FE443EC57ECC601B50155
:10FDE0000E94C4C618160CF4ECC087EC882E82E082
:10FDF000982E98E1292E93E1392E2DE0E22E29E16B
:10FE0000F22E10E0F40181914F010E94E4AD8823AD
:10FE100021F1133051F40E940AAEF1016083718325
:10FE2000828393830E94EF5918C00E940AAEF701A3
:10FE300020813181428153810E9479C4F101608324
:10FE400071838283938324E233E140E253E16CE1E6
:10FE500073E188E193E10E94E0441F5FF4E02F0E1C
:10FE6000311C84E0E80EF11C143061F620E83FE418
:10FE700043EC57ECC601B5010E94C4C6181654F4F1
:10FE8000A0922413B0922513C0922613D092271368
:10FE90000E94EF5920E83FE443EC57ECC301B20164
:10FEA0000E94C4C61816F4F420910D1930910E1951
:10FEB00040910F1950911019C301B2010E9479C4E9
:10FEC000609318137093191380931A1390931B1354
:10FED00024E233E140E253E16CE173E188E193E134
:10FEE0000E94E04420E83FE443EC57EC69817A81CA
:10FEF0008B819C810E94C4C61816FCF420911119B4
:10FF000030911219409113195091141969817A8115
:10FF10008B819C810E9479C460931C1370931D1384
:10FF200080931E1390931F1324E233E140E253E1C8
:10FF30006CE173E1CB010E94E04420E83FE443EC34
:10FF400057EC6D817E818F8198850E94C4C61816FA
:10FF5000DCF520911519309116194091171950911F
:10FF600018196D817E818F8198850E9479C4609374
:10FF7000201370932113809322139093231324E270
:10FF800033E140E253E16CE173E188E193E12896CB
:10FF90000FB6F894DEBF0FBECDBFDF91CF911F919A
:10FFA0000F91FF90EF90DF90CF90BF90AF909F9018
:10FFB0008F907F906F905F904F903F902F900C9418
:10FFC000E0440E9428A911CF28960FB6F894DEBF0E
:10FFD0000FBECDBFDF91CF911F910F91FF90EF909A
:10FFE000DF90CF90BF90AF909F908F907F906F9059
:10FFF0005F904F903F902F9008954F925F926F9235
:020000021000EC
:100000007F928F929F92AF92BF92CF92DF92EF92A8
:10001000FF920F931F93CF93DF93009709F0EAC0ED
:10002000209106132223E1F1822F90E00E9489ADF6
:10003000609318137093191380931A1390931B13E2
:100040001092250210922602109227021092280286
:100050000091231010912410D0912510C0912610EA
:10006000C0901B10D0901C10E0901D10F0901E103E
:100070009601A701B8018D2F9C2F0E94C4C61816A7
:100080001CF08601DE2DCF2DC801AD2FBC2F809333
:10009000190290931A02A0931B02B0931C02EEC0A7
:1000A000209113023091140222503109223031057F
:1000B00008F0A0C08EEA9EE00E94B5AD20910D1917
:1000C00030910E1940910F19509110190E9479C466
:1000D000609318137093191380931A1390931B1342
:1000E00087EB97E10E94B5AD20910D1930910E1963
:1000F00040910F19509110190E9479C46093250204
:100100007093260280932702909328028BEA97E14E
:100110000E94B5AD20910D1930910E1940910F1923
:10012000509110190E9479C42B013C0100912310B9
:1001300010912410D0912510C0912610C0901B1052
:10014000D0901C10E0901D10F0901E109601A70199
:10015000B8018D2F9C2F0E94C4C618162CF0BC2D00
:10016000AD2DFE2DEF2D03C0B02FA12FFE018090ED
:10017000040290900502A0900602B0900702A5012B
:1001800094016B2F7A2F8F2F9E2F0E9478C49B0192
:10019000AC01C301B2010E94A1BE87FF0FC08BEA70
:1001A00097E10E94B5AD20910D1930910E19409143
:1001B0000F19509110190E9479C413C09601A7011C
:1001C000B8018D2F9C2F0E94C4C618161CF0860102
:1001D000DE2DCF2DA5019401B8018D2F9C2F0E94FB
:1001E00078C46093190270931A0280931B02909353
:1001F0001C0244C0EC01CC0FDD1FCC0FDD1FCE0173
:100200008255914F0E94B5AD9E01285E3C4E79010A
:100210008E01035F164EF8012081318142815381A6
:100220000E9479C4F7016083718382839383CE0136
:100230008954984E0E94B5AD9E012B5D3D4F7901CA
:10024000F80120813181428153810E9479C4F701F4
:100250006083718382839383CE018555984E0E947B
:10026000B5ADC75EDD4FF8012081318142815381F8
:100270000E9479C4688379838A839B83DF91CF91BD
:100280001F910F91FF90EF90DF90CF90BF90AF90B4
:100290009F908F907F906F905F904F9008954F92B6
:1002A0005F926F927F92BF92CF92DF92EF92FF9216
:1002B0000F931F93CF93DF93CDB7DEB728970FB679
:1002C000F894DEBF0FBECDBF209111023091120213
:1002D000225031092230310508F44DC38F3F2FEFF2
:1002E000920739F40E940AAE0E94DEC56093A018FE
:1002F00002C08093A0188091A018823090F1E6E7A8
:10030000F8E08491882341F09091C00095FFFCCFE4
:100310008093C6003196F5CFECE7F5E08191882314
:1003200039F09091C00095FFFCCF8093C600F6CFC6
:100330008091A0189091C00095FFFCCF8093C600DB
:10034000E5E6F9E08191882339F09091C00095FFAE
:10035000FCCF8093C600F6CF8091C00085FFFCCF14
:100360008DC286E40E94E4AD8823E1F00E940AAECB
:100370006B017C0160937F187093801880938118C3
:100380009093821820E030E0A9010E94C4C618169C
:100390005CF4C0926302D0926402E0926502F09233
:1003A000660202C0B12C02C0BB24B3949091A01885
:1003B00080910613981709F43DC28091181390910B
:1003C0001913A0911A13B0911B13809330199093B5
:1003D0003119A0933219B093331980911C13909165
:1003E0001D13A0911E13B0911F1380933419909385
:1003F0003519A0933619B093371980912013909135
:100400002113A0912213B091231380933819909354
:100410003919A0933A19B0933B1980912413909104
:100420002513A0912613B091271380933C19909324
:100430003D19A0933E19B0933F1980913E109091C1
:100440003F10019749F081E080930C1980E090E023
:100450000E945D5210920C1980910713811122C0E5
:1004600080911A1990911B19A0911C19B0911D1916
:10047000892B8A2B8B2B09F005C2C0901813D090C2
:100480001913E0901A13F0901B138091061390E05B
:100490000E9489AD9B01AC01C701B6010E94A1BEBB
:1004A0008111F0C1C0903710D0903810E090391011
:1004B000F0903A1020E030E0A901C701B6010E9497
:1004C000A1BE87FD0AC020E030E040E251E4C70150
:1004D000B6010E94C4C6181664F480E090E0A0E95A
:1004E000B0E48093371090933810A0933910B093F4
:1004F0003A10C090300BD090310BE090320BF0905E
:10050000330B20E030E0A901C701B6010E94A1BE73
:1005100087FD0AC020E030E040E850E4C701B601A2
:100520000E94C4C6181664F480E090E0A0E0B0E435
:100530008093300B9093310BA093320BB093330B1D
:1005400010922F1010923010109231101092321021
:1005500020E030E040EA50E46091371070913810AC
:100560008091391090913A100E9478C460932B10BA
:1005700070932C1080932D1090932E102091300B9F
:100580003091310B4091320B5091330B60E070E0B1
:1005900080E090E40E9478C460933310709334102C
:1005A00080933510909336100091061310E0D09090
:1005B000A018ED2CF12CF801EE0FFF1FEE0FFF1F1E
:1005C000E95DFF4E208131814281538160911C138E
:1005D00070911D1380911E1390911F130E9478C477
:1005E000F701EE0FFF1FEE0FFF1FE95DFF4E2081A9
:1005F0003181428153810E9479C460931C137093AE
:100600001D1380931E1390931F13000F111F000FD3
:10061000111FD801A15DBF4E2D913D914D915C916F
:1006200060912013709121138091221390912313D4
:100630000E9478C4F701EE0FFF1FEE0FFF1FE15D70
:10064000FF4E20813181428153810E9479C46093A1
:100650002013709321138093221390932313D0922D
:10066000061380E090E0C9DC80911302909114029F
:10067000009709F58091171090911810A09119100A
:10068000B0911A108093181390931913A0931A1312
:10069000B0931B138091301990913119A0913219A8
:1006A000B09133198093171090931810A0931910DC
:1006B000B0931A10ADC09C0122503109223031058F
:1006C00008F04BC081E090910613911180E0809377
:1006D0001919882389F08091171090911810A09112
:1006E0001910B0911A108093181390931913A093B6
:1006F0001A13B0931B131AC0209104023091050203
:1007000040910602509107026091301970913119A1
:1007100080913219909133190E9479C46093181313
:100720007093191380931A1390931B1380913019AF
:1007300090913119A0913219B0913319809317100B
:1007400090931810A0931910B0931A1081E090E0C4
:1007500090931202809311025BC0019709F058C078
:100760008091181390911913A0911A13B0911B1333
:1007700080931E1990931F19A0932019B0932119EB
:1007800080911C1390911D13A0911E13B0911F1303
:100790008093221990932319A0932419B0932519BB
:1007A0006091201370912113809122139091231353
:1007B00000912413109125132091261330912713B3
:1007C00000932A1910932B1920932C1930932D196B
:1007D00020E030E0A9010E9479C46093261970934B
:1007E0002719809328199093291981E0809319196A
:1007F00010921A1910921B1910921C1910921D199F
:1008000080930C1980E090E00E945D5210920C19C8
:1008100024E233E140E253E16CE173E188E193E1EA
:100820000E94E044BB2031F080910713811102C087
:100830000E94C394E6E7F8E08491882341F0909108
:10084000C00095FFFCCF8093C6003196F5CFE6E758
:10085000F9E08191882339F09091C00095FFFCCF99
:100860008093C600F6CF6091061370E080E090E0C0
:100870000E946B278091C00085FFFCCF8AE08093A7
:10088000C60079C04090BD125090BE126090BF1259
:100890007090C01220E030E0A901609120137091A7
:1008A000211380912213909123130E9479C46983AC
:1008B0007A838B839C8386E0C82E83E1D82E8301C4
:1008C000720124E233E1AE014F5F5F4F6CE173E1EF
:1008D00088E193E10E9483454090B5125090B61292
:1008E0006090B7127090B81220E030E0A9016091DA
:1008F00020137091211380912213909123130E9451
:1009000079C46D837E838F8398878091061390E0EE
:100910000E9489AD69837A838B839C8383017201F2
:1009200024E233E1AE014B5F5F4F6CE173E1CE0136
:1009300001960E9483454090BD125090BE12609077
:10094000BF127090C0128091061390E00E9489AD92
:1009500069837A838B839C838301720124E233E170
:1009600040E253E16CE173E1CE0101960E948345C0
:100970000E9428A997CD28960FB6F894DEBF0FBE27
:10098000CDBFDF91CF911F910F91FF90EF90DF903E
:10099000CF90BF907F906F905F904F9008952F926F
:1009A0003F924F925F926F927F928F929F92AF92FF
:1009B000BF92CF92DF92EF92FF920F931F93CF934C
:1009C000DF93CDB7DEB7C75CD1400FB6F894DEBF7A
:1009D0000FBECDBF8091401068E374E0811106C066
:1009E000CE01815E9E4F0E940F90A5C2CE01875816
:1009F0009E4F0E940F90CE0193950E94A272C12C2F
:100A0000DD24D394CC0EDD1E84E0C80ED11C21E081
:100A100046E755E068E770E1C6010E9468638823F5
:100A200009F449C0CB5EDE4FE880F980C551D14062
:100A30009FEFE91AF90A8AE090E0CB5DDE4F9983D7
:100A40008883C552D1409E012B5D3E4FA7018E0188
:100A50000F5F1F4FB801C6010E94566468E374E03F
:100A6000CE01815E9E4F0E940F906801C601801BDF
:100A7000910B8E159F055CF4D6016D916D01662377
:100A8000A9F3CE01815E9E4F0E94068FEFCFCE016B
:100A9000815E9E4F0E94BE28882341F0BE01615EA8
:100AA0007E4FCE0187589E4F0E942E8FCE01815ED1
:100AB0009E4F0E947C8F80E091E08C0F9D1F0496DA
:100AC0000E94E15DCE0187589E4F0E94BE28882378
:100AD00009F410C268E374E0CE018D589E4F0E9465
:100AE0000F9068E374E0CE0183599E4F0E940F90EF
:100AF0008CE291E0CD56DE4F99838883C359D14073
:100B000044E0BE0161577E4FCE018D569E4F0E943C
:100B1000393E42E0BE0163567E4FCE018D569E4F58
:100B20000E94393E42E0BE0165567E4FCE018D5691
:100B30009E4F0E94393E42E0BE0167567E4FCE0175
:100B40008D569E4F0E94393E44E0BE0165577E4F50
:100B5000CE018D569E4F0E94393E44E0BE0169573A
:100B60007E4FCE018D569E4F0E94393E8EE591E01C
:100B7000CD56DE4F99838883C359D14042E0BE01F0
:100B800069567E4FCE018D569E4F0E94393E42E0FF
:100B9000BE016B567E4FCE018D569E4F0E94393E50
:100BA00044E0BE016D577E4FCE018D569E4F0E9490
:100BB000393E44E0BE0161587E4FCE018D569E4FB6
:100BC0000E94393EC158DE4F488159816A817B813C
:100BD000CF57D14022E0CE01815E9E4F0E94818F8F
:100BE000CD57DE4F488159816A817B81C358D140FE
:100BF00022E0CE018B5D9E4F0E94818FCB56DE4F4F
:100C000068817981C559D1404AE0CE01855D9E4F0A
:100C10000E94DC8FC956DE4F68817981C759D14067
:100C20004AE0CE018F5C9E4F0E94DC8F22E040E0C4
:100C300050E0BA01CE01895C9E4F0E94818F22E074
:100C400040E050E0BA01CE01835C9E4F0E94818F4C
:100C50004AE068EC70E0CE018D5B9E4F0E94DC8F15
:100C6000C957DE4F488159816A817B81C758D1407D
:100C700022E0CE01875B9E4F0E94818FC557DE4FD9
:100C8000488159816A817B81CB58D14022E0CE01D5
:100C9000815B9E4F0E94818FC756DE4F68817981AC
:100CA000C959D1404AE0CE018B5A9E4F0E94DC8F39
:100CB000C556DE4F68817981CB59D1404AE0CE01DB
:100CC000855A9E4F0E94DC8FC356DE4F6881798122
:100CD000CD59D1404AE0CE018F599E4F0E94DC8F02
:100CE000C157DE4F688179818A819B81CF58D1407D
:100CF000C959DE4F19821882C756D140C759DE4FF5
:100D000019821882C956D140C559DE4F19821882FE
:100D1000CB56D1402AE0AE014F5F5F4F0E9438BEF4
:100D2000BE016F5F7F4FCE0189599E4F0E94198F80
:100D3000BE0169597E4FCE0101960E94079061E481
:100D400079E0CE0101960E94DE8EBE016F597E4F82
:100D50000E94F58E61E479E00E94DE8EBE01655A44
:100D60007E4F0E94F58E61E479E00E94DE8EBE0126
:100D70006B5A7E4F0E94F58E61E479E00E94DE8E10
:100D8000BE01615B7E4F0E94F58E61E479E00E94B6
:100D9000DE8EBE01675B7E4F0E94F58E61E479E0D6
:100DA0000E94DE8EBE016D5B7E4F0E94F58E61E477
:100DB00079E00E94DE8EBE01635C7E4F0E94F58E5C
:100DC00061E479E0FBD7BE01695C7E4F0E94F58E3D
:100DD00061E479E0F3D7BE016F5C7E4F0E94F58E2F
:100DE00061E479E0EBD7BE01655D7E4FFED761E43B
:100DF00079E0E4D7BE016B5D7E4FF7D761E479E01F
:100E0000DDD7BE01615E7E4FF0D7BC01CE018359B4
:100E10009E4F0E942E8FCE0101960E947C8FCE01A4
:100E200089599E4F0E947C8FCE018F599E4F0E9400
:100E30007C8FCE01855A9E4F0E947C8FCE018B5AAB
:100E40009E4F0E947C8FCE01815B9E4F0E947C8FC3
:100E5000CE01875B9E4F0E947C8FCE018D5B9E4FA3
:100E60000E947C8FCE01835C9E4F0E947C8FCE01BE
:100E7000895C9E4F0E947C8FCE018F5C9E4F0E94AA
:100E80007C8FCE01855D9E4F0E947C8FCE018B5D55
:100E90009E4F0E947C8FCE01815E9E4F0E947C8F70
:100EA000BE0163597E4FCE018D589E4FECD7CE01C7
:100EB00083599E4F0E947C8FBE0167587E4FCE01A2
:100EC00001960E94079061E479E0CE01019676D701
:100ED000BE016D587E4F89D7BC01CE0187589E4F09
:100EE000BDD7CE0101960E947C8FCE018D589E4FBA
:100EF0000E947C8FC15EDE4F19821882CF51D14093
:100F0000CF5DDE4F19821882C152D140CD5DDE4FD8
:100F100019821882C352D140BE0167587E4FCE015C
:100F2000815E9E4FB0D7CE0193950E949A72CE01FA
:100F300087589E4FE1D7BE01615E7E4FCE0101967C
:100F40000E94079020E030E04CE7BE016F5F7F4FCA
:100F5000CE0193950E94FA71CE010196CDD7BE01C4
:100F6000615E7E4FCE018B5D9E4F0E94079021E017
:100F700030E04CE7BE016B5D7E4FCE0101960E94D2
:100F8000FA71CE018B5D9E4FB7D7CE01815E9E4F29
:100F90000E94BE28882309F420C4BE01615E7E4FF2
:100FA000CE018B5D9E4F0E94079022E030E04CE71F
:100FB000BE016B5D7E4FCE01855D9E4F0E94FA7132
:100FC000C55DDE4F88819981CB52D1400E9490BD92
:100FD0006B017C01CE01855D9E4F8ED7CE018B5D6E
:100FE0009E4F8AD7BE01615E7E4FCE018B5D9E4FC4
:100FF0000E94079023E030E04CE7BE016B5D7E4F1E
:10100000CE01855D9E4F0E94FA71CE01855D9E4F97
:1010100023D5C156DE4F688379838A839B83CF595A
:10102000D140C156DE4FE881F981CF59D140C15539
:10103000DE4FF983E883CF5AD140CE01855D9E4FC4
:101040005BD7CE018B5D9E4F57D7BE01615E7E4F51
:10105000CE018B5D9E4FDBD724E030E04CE7BE0134
:101060006B5D7E4FCE01855D9E4F0E94FA71CE0171
:10107000855D9E4FF1D4CF54DE4F688379838A8398
:101080009B83C15BD140CF54DE4FA880B980C15B48
:10109000D140CE01855D9E4F2FD7CE018B5D9E4FF7
:1010A0002BD7BE01615E7E4FCE018B5D9E4FAFD7C9
:1010B00025E030E04CE7BE016B5D7E4FCE01855DE3
:1010C0009E4F0E94FA71CE01855D9E4FC5D4C754D4
:1010D000DE4F6883C95BD1404B01CE01855D9E4FD9
:1010E0000BD7CE018B5D9E4F07D7BE01615E7E4F51
:1010F000CE018B5D9E4F8BD726E030E04CE7BE01E2
:101100006B5D7E4FCE01855D9E4F0E94FA71CE01D0
:10111000855D9E4F0E94DC71C955DE4F68837983DF
:101120008A839B83C75AD140CE01855D9E4FE4D60A
:10113000CE018B5D9E4FE0D6BE01615E7E4FCE013B
:101140008B5D9E4F64D727E030E04CE7BE016B5DBE
:101150007E4FCE01855D9E4F0E94FA71CE01855D66
:101160009E4F0E94DC712B013C01CE01855D9E4F9C
:10117000C3D6CE018B5D9E4FBFD6BE01615E7E4F52
:10118000CE018B5D9E4F43D728E030E04CE7BE0197
:101190006B5D7E4FCE01855D9E4F0E94FA71CE0140
:1011A000855D9E4F59D4C654DE4F688379838A8308
:1011B0009B83CA5BD140CE01855D9E4F9DD6CE01FB
:1011C0008B5D9E4F99D6BE01615E7E4FCE018B5DD9
:1011D0009E4F1DD729E030E04CE7BE016B5D7E4F8E
:1011E000CE01855D9E4F0E94FA71CE01855D9E4FB6
:1011F0000E94DC71CD55DE4F688379838A839B839F
:10120000C35AD140CE01855D9E4F76D6CE018B5D0F
:101210009E4F72D6BE01615E7E4FCE018B5D9E4FAA
:10122000F6D62AE030E04CE7BE016B5D7E4FCE0182
:10123000855D9E4F0E94FA71CE01855D9E4F0E9492
:10124000DC71C254DE4F688379838A839B83CE5BD3
:10125000D140CE01855D9E4F4FD6CE018B5D9E4F16
:101260004BD6BE01615E7E4FCE018B5D9E4FCFD6C9
:101270002BE030E04CE7BE016B5D7E4FCE01855D1B
:101280009E4F0E94FA71CE01855D9E4FE5D3CB54EF
:10129000DE4F688379838A839B83C55BD140CE010F
:1012A000855D9E4F29D6CE018B5D9E4F25D6BE0112
:1012B000615E7E4FCE018B5D9E4FA9D62CE030E063
:1012C0004CE7BE016B5D7E4FCE01855D9E4F0E9457
:1012D000FA71CE01855D9E4FBFD3C555DE4F688341
:1012E00079838A839B83CB5AD140C555DE4F888151
:1012F0009981CB5AD140CE53DE4F99838883C25C0B
:10130000D140CE01855D9E4FF7D5CE018B5D9E4FBE
:10131000F3D5BE01615E7E4FCE018B5D9E4F77D6C9
:101320002DE030E04CE7BE016B5D7E4FCE01855D68
:101330009E4F0E94FA71CE01855D9E4F0E94DC7126
:10134000CC53DE4F688379838A839B83C45CD1400E
:10135000CE01855D9E4FD0D5CE018B5D9E4FCCD505
:1013600091E0C91698E0D906E104F10408F435C209
:10137000CB54DE4F28803980C55BD14089819A816A
:101380009701860141E0BC010E94EE5668E879E0D1
:10139000CE018B5D9E4F43D6BE017395CE018B5D12
:1013A0009E4F23D568EB74E009D5BC01CE010196B0
:1013B00055D5CE018B5D9E4F9FD589819A810E9424
:1013C000116581EA99E00E94116580E090E0AAE74A
:1013D000B5E48093630290936402A0936502B09396
:1013E000660282E090E090933F1080933E101214CA
:1013F000130444F4CB54DE4F88819981C55BD140FE
:101400000E94917CC555DE4FA881B981CB5AD1404D
:10141000B0931402A0931302C155DE4FE881F98105
:10142000CF5AD1401E161F0634F56D01F2E0CF1AD7
:10143000D10882E0C816D10458F41092A018C15601
:10144000DE4F88819981CF59D1400E94379F13C0C8
:10145000CE53DE4FA881B981C25CD140119709F00B
:10146000C1C1C156DE4FE881F981CF59D140F09317
:10147000FA12E093F9121A141B0484F480911302F7
:1014800090911402019751F4C156DE4F88819981E1
:10149000CF59D1409093FC128093FB12809113029C
:1014A00090911402019739F5C155DE4FA881B98199
:1014B000CF5AD1401A161B0664F48114910449F4E2
:1014C00010920613C156DE4F88819981CF59D140C1
:1014D00010C01A141B047CF4B1E08B16910459F46B
:1014E00081E080930613CF54DE4F88819981C15BE0
:1014F000D1400E94379F80E090E00E94FD7F809164
:10150000130290911402029781F4CC53DE4F88812C
:101510009981AA81BB81C45CD140809304029093DD
:101520000502A0930602B093070291E08916910488
:1015300031F520E030E040E85FE3CD55DE4F6881D3
:1015400079818A819B81C35AD1400E94A1BE87FFC5
:1015500016C020E030E040E752E460911B1070912B
:101560001C1080911D1090911E100E9478C4CD55C2
:10157000DE4F688379838A839B83C35AD140C654E4
:10158000DE4FA881B981CA5BD140B093A918A0935E
:10159000A81863015201C955DE4FE880F9800A811D
:1015A0001B81C75AD14020E030E0A901CA01B9012E
:1015B0000E94C07E20E030E040E751E4C955DE4F94
:1015C000688179818A819B81C75AD1400E9479C400
:1015D000C156DE4F688379838A839B83CF59D1407C
:1015E0007B018C0120E83FE443EC57ECCA01B901D0
:1015F0000E94195A61E070E081E090E00E9435A9F4
:1016000080911302909114020197D1F5C754DE4FD7
:10161000B881C95BD140B09306138A948928E9F454
:1016200020E030E040EA50E46091371070913810CB
:101630008091391090913A100E9478C49B01AC01BE
:101640000E9479C49B01AC0160911B1070911C1029
:1016500080911D1090911E1007C060E070E088E43A
:1016600092EC20E030E0A90163015201C156DE4F47
:10167000E880F9800A811B81CF59D1400E94C07E49
:10168000812C912C54017501640100E010E020E0F0
:1016900030E040E050E060E070E0CB010E94994211
:1016A0001092481363015201C955DE4FE880F9805A
:1016B0000A811B81C75AD140C254DE4F288139812B
:1016C0004A815B81CE5BD140CD55DE4F6881798107
:1016D0008A819B81C35AD1400E94195ABE01615E22
:1016E0007E4FCE018B5D9E4F92D42DE030E04CE7D3
:1016F000BE016B5D7E4FCE01855D9E4F0E94FA71EB
:10170000CE01855D9E4F0E94DC71609363027093F1
:1017100064028093650290936602CE01855D9E4FC0
:10172000EBD3CE018B5D9E4FE7D320E030E04AEF54
:1017300054E460916302709164028091650290911B
:1017400066020E94A1BE87FF0CC080E090E0AAE77D
:10175000B5E48093630290936402A0936502B09312
:10176000660210923F1010923E1080914010882324
:1017700031F081E090E090933F1080933E100E9402
:101780000D356093390B70933A0B80933B0B90931C
:101790003C0BCE010196B0D3CE019395ADD3CE01D3
:1017A000815E9E4FA9D3C953DE4F0FB6F894DEBFBA
:1017B0000FBECDBFDF91CF911F910F91FF90EF90A2
:1017C000DF90CF90BF90AF909F908F907F906F9061
:1017D0005F904F903F902F9008958CE695E00E9487
:1017E0001165D7CF1A141B040CF448CE84CE08958B
:1017F000CF92DF92EF92FF920F931F93CF93DF93DD
:101800006C017A018B01C0E0D0E0CE15DF0589F0D4
:10181000D8016D918D01D601ED91FC910190F0817F
:10182000E02DC6011995892B11F47E0102C0219685
:10183000ECCFC701DF91CF911F910F91FF90EF90F7
:10184000DF90CF900895FC01538D448D252F30E01B
:10185000842F90E0821B930B541710F0CF960895BD
:1018600001970895FC01918D828D981761F0828D0A
:10187000DF01A80FB11D5D968C91928D9F5F9F73C4
:10188000928F90E008958FEF9FEF0895FC01918D66
:10189000828D981731F0828DE80FF11D858D90E0D3
:1018A00008958FEF9FEF0895FC01918D228D892F70
:1018B00090E0805C9F4F821B91098F739927089558
:1018C0008AE79FE0F1DF21E0892B09F420E0822FF5
:1018D00008950E9441C90F931F93CF93DF93EC01AA
:1018E00088819981009729F02A813B812617370743
:1018F00088F48B016F5F7F4F0E9459C8009761F099
:10190000998388831B830A832C813D81232B11F4C7
:10191000FC01108281E001C080E0DF91CF911F9136
:101920000F910895CF93DF93EC01888199810097FF
:1019300011F00E9466BA198218821D821C821B82D5
:101940001A82DF91CF910895EF92FF920F931F9328
:10195000CF93DF93EC017B018A01BA01BCDF8111D7
:1019600003C0CE01DFDF07C01D830C83B701888170
:1019700099810E9493C9CE01DF91CF911F910F9160
:10198000FF90EF900895EF92FF920F931F93CF93E4
:10199000DF93EC0181E0888F9B8D8C8D981305C0BF
:1019A000E889F989808185FD24C0F62E0B8D10E031
:1019B0000F5F1F4F0F731127E02E8C8DE8120CC0A4
:1019C0000FB607FCFACFE889F989808185FFF5CF4A
:1019D000CE010E945A33F1CF8B8DFE01E80FF11D2D
:1019E000E35AFF4FF0820B8FEA89FB898081806286
:1019F00007C0EE89FF896083E889F9898081806466
:101A0000808381E090E0DF91CF911F910F91FF9053
:101A1000EF900895CF93DF93EC01888D8823C9F070
:101A2000EA89FB89808185FD05C0A889B9898C91E7
:101A300086FD0FC00FB607FCF5CF808185FFF2CF82
:101A4000A889B9898C9185FFEDCFCE010E945A33C8
:101A5000E7CFDF91CF910895FC01808191810097BC
:101A600011F00C9490BD60E070E0CB010895CF932D
:101A7000DF93FC01C081D181209751F088818823B8
:101A800039F0082E000C990B0E9445C98993F6CFB6
:101A9000DF91CF9108952F923F924F925F926F9274
:101AA0007F928F929F92AF92BF92CF92DF92EF92EE
:101AB000FF920F931F93CF93DF9300D01F92CDB768
:101AC000DEB7FC01448055804114510409F413C170
:101AD000FB01648075806114710409F40CC17A0102
:101AE0006B019C838B83FA01A480B580A618B7088C
:101AF000FC0100811181A114B104C1F4F6016081DF
:101B00007181C8010E94B7C95C01892B09F4F3C037
:101B1000F7016081718144815581C5010E945AC9D4
:101B2000F701048115810A0D1B1DE8CFB7FE02C025
:101B3000480106C0FB01208031804201C80148C035
:101B4000F60160817181C4010E94B7C92C01892B03
:101B500029F1320168187908A301B401C8010E9473
:101B60005AC9060D171DF7016081718144815581A5
:101B7000C8010E945AC9F70184819581080F191F75
:101B8000F60184809580840C951CEB81FC81848116
:101B900095818A0D9B1D95838483D2CFB401C801A2
:101BA0000F900F900F900F90DF91CF911F910F9199
:101BB000FF90EF90DF90CF90BF90AF909F908F906D
:101BC0007F906F905F904F903F902F900C9493C9AF
:101BD000B1010E94B7C9009729F0860D971D8A0CA4
:101BE0009B1CF6CF8414950409F485C0EB81FC811D
:101BF000828193818815990578F4B4016F5F7F4FD6
:101C0000C8010E9459C8009709F475C0EB81FC8196
